:020000040800F2
:1000000000060020E1010008E3010008E301000808
:10001000E3010008E3010008E3010008E301000830
:10002000E3010008E3010008E30100089D2F000838
:10003000E3010008E3010008E3010008E301000810
:10004000E3010008E3010008E3010008E301000800
:10005000E3010008E3010008453200086D320008A2
:1000600095320008BD320008E5320008E3010008BF
:10007000E3010008E3010008E3010008E3010008D0
:10008000E3010008E3010008E3010008E3010008C0
:10009000E3010008E3010008E30100080D33000854
:1000A000E3010008E3010008E3010008E3010008A0
:1000B000E1330008E3010008E3010008E301000860
:1000C000E3010008E3010008E3010008E301000880
:1000D000E3010008E3010008E3010008E301000870
:1000E00071330008E3010008E3010008E3010008A0
:1000F000E3010008E3010008E3010008E301000850
:10010000E3010008E3010008E3010008E30100083F
:10011000E3010008E3010008E3010008E30100082F
:10012000E3010008E3010008E3010008E30100081F
:10013000E3010008E3010008E3010008E30100080F
:10014000E3010008E3010008E3010008512700086B
:10015000E3010008E3010008E3010008E3010008EF
:10016000E3010008E3010008E3010008E3010008DF
:10017000E3010008E3010008E3010008E3010008CF
:10018000E3010008E3010008E3010008E3010008BF
:10019000E3010008E3010008E3010008E3010008AF
:1001A000E3010008E3010008E3010008E30100089F
:1001B000E3010008E3010008E3010008E30100088F
:1001C000E3010008E3010008E3010008E30100087F
:1001D000E3010008E3010008E3010008E30100086F
:1001E00002E000F000F8FEE772B6374880F30888B6
:1001F000364880F3098836483649086040F20000E6
:10020000CCF200004EF63471CEF200010860BFF36C
:100210004F8FBFF36F8F40F20000C0F2F0004EF638
:100220008851CEF200010860BFF34F8FBFF36F8F8C
:100230004FF00000E1EE100A4EF63C71CEF20001E4
:100240000860062080F31488BFF36F8F01F048FF29
:1002500002F042FE4FF055301F491B4A91423CBF0D
:1002600041F8040BFAE71D49184A91423CBF41F896
:10027000040BFAE71A491B4A1B4B9A423EBF51F83E
:10028000040B42F8040BF8E700201849184A914281
:100290003CBF41F8040BFAE701F026FF02F070FEC4
:1002A000144C154DAC4203DA54F8041B8847F9E7A7
:1002B00000F042F8114C124DAC4203DA54F8041B22
:1002C0008847F9E701F00EBF000600200022002059
:1002D0000000000808ED00E00000002000060020FB
:1002E000A8370008002200204022002040220020E1
:1002F000602E0020E0010008E0010008E001000895
:10030000E00100082DE9F04F2DED108AC1F80CD066
:10031000C3689D46BDEC108ABDE8F08F002383F3CF
:1003200011882846A047002001F08AFAFEE701F074
:1003300019FA00DFFEE7000038B500F0BFFB01F05E
:100340009FFE054601F0C2FE0446C8B90E4B9D4211
:1003500018D001339D4218BF044641F2883504BFCE
:1003600001240025002001F095FE0CB100F074F886
:1003700000F018FD284600F0C3F800F06DF8F9E72A
:100380000025EFE70546EDE7010007B008B500F0EE
:1003900067FBA0F120035842584108BD07B541F260
:1003A0001203022101A8ADF8043000F077FB03B07E
:1003B0005DF804FB38B5302383F3118817480368D0
:1003C0000BB101F009FB164A144800234FF47A716F
:1003D00001F0F8FA002383F31188124C236813B15B
:1003E0002368013B2360636813B16368013B63606A
:1003F0000D4D2B7833B963687BB9022000F034FCD3
:10040000322363602B78032B07D163682BB902205A
:1004100000F02AFC4FF47A73636038BD402200205C
:10042000B50300086023002058220020084B1870F4
:1004300003280CD8DFE800F008050208022000F0CD
:1004400003BC022000F0F0BB024B00225A60704750
:100450005822002060230020244B254A10B51C465A
:100460001968013140D004339342F9D16268214BBD
:100470009A4239D9204B9B6803F1006303F580331E
:100480009A4231D2002000F033FB0220FFF7CEFF6A
:100490001A4B1A6C00221A64196E1A66196E596C7E
:1004A0005A64596E5A665A6E5A6942F080025A610D
:1004B0005A6922F080025A615A691A6942F0005260
:1004C0001A611A6922F000521A611B6972B64FF064
:1004D000E0233021C3F8084DD4E9003281F31188BC
:1004E0009D4683F30888104710BD00BF0000010837
:1004F00020000108FFFF0008002200200038024011
:100500002DE9F04F93B0AA4B00902022FF210AA8BA
:100510009D6800F0F1FBA74A1378A3B9A648012112
:1005200003601170302383F3118803680BB101F06D
:1005300053FAA24AA04800234FF47A7101F042FA1C
:10054000002383F31188009B13B19D4B009A1A601E
:100550009C4A009C1378032B1EBF00231370984AFB
:100560004FF0000A18BF5360D3465646D1460120CB
:1005700000F06AFB24B1924B1B68002B00F0118243
:10058000002000F06DFA0390039B002BF2DB0120AA
:1005900000F04AFB039B213B162BE8D801A252F83E
:1005A00023F000BF0106000829060008BD06000868
:1005B0006F0500086F0500086F0500084707000871
:1005C000170900083108000893080008BB08000854
:1005D000E10800086F050008F30800086F0500082F
:1005E00065090008A10600086F050008A9090008B0
:1005F0000D060008A10600086F0500089308000812
:100600000220FFF7C3FE002840F0F581009B022185
:10061000BAF1000F08BF1C4605A841F21233ADF82D
:10062000143000F03BFAA2E74FF47A7000F018FAA9
:10063000071EEBDB0220FFF7A9FE0028E6D0013FF2
:10064000052F00F2DA81DFE807F0030A0D101336F8
:1006500005230593042105A800F020FA17E054486B
:100660000421F9E758480421F6E758480421F3E744
:100670004FF01C08404600F03DFA08F104080590D0
:10068000042105A800F00AFAB8F12C0FF2D10120DC
:1006900000FA07F747EA0B0B5FFA8BFB4FF00009F4
:1006A00000F076FB26B10BF00B030B2B08BF0024E8
:1006B000FFF774FE5BE746480421CDE7002EA5D086
:1006C0000BF00B030B2BA1D10220FFF75FFE0746B7
:1006D00000289BD0012000F00BFA0220FFF7A6FEB5
:1006E00000261FFA86F8404600F012FA044690B140
:1006F0000021404600F01CFA01360028F1D1BA462C
:10070000044641F21213022105A8ADF814303E460A
:1007100000F0C4F92BE70120FFF788FE2546244BA3
:100720009B68AB4207D9284600F0E4F9013040F05D
:1007300067810435F3E7234B00251D70204BBA4633
:100740005D603E46ACE7002E3FF460AF0BF00B035C
:100750000B2B7FF45BAF0220FFF768FE322000F026
:100760007FF9B0F10008FFF651AF18F003077FF4EE
:100770004DAF0F4A926808EB050393423FF646AF30
:10078000B8F5807F3FF742AF124B0193B84523DDA8
:100790004FF47A7000F064F90390039A002AFFF690
:1007A00035AF019B039A03F8012B0137EDE700BF3A
:1007B000002200205C23002040220020B503000816
:1007C000602300205822002004220020082200205C
:1007D0000C2200205C220020C820FFF7D7FD07462E
:1007E00000283FF413AF1F2D11D8C5F12002424558
:1007F0000AAB25F0030028BF424683490192184402
:1008000000F054FA019A8048FF2100F075FA4FEA8F
:10081000A8037D490193C8F38702284600F074FAC3
:10082000064600283FF46DAF019B05EB830537E7D3
:100830000220FFF7ABFD00283FF4E8AE00F0A4F97A
:1008400000283FF4E3AE0027B846704B9B68BB42DC
:1008500018D91F2F11D80A9B01330ED027F003039C
:1008600012AA134453F8203C05934046042205A9DC
:1008700000F0C2FA04378046E7E7384600F03AF95C
:100880000590F2E7CDF81480042105A800F006F9E0
:1008900006E70023642104A8049300F0F5F800287B
:1008A0007FF4B4AE0220FFF771FD00283FF4AEAE36
:1008B000049800F051F90590E6E70023642104A8AC
:1008C000049300F0E1F800287FF4A0AE0220FFF7C7
:1008D0005DFD00283FF49AAE049800F04DF9EAE778
:1008E0000220FFF753FD00283FF490AE00F05CF9C2
:1008F000E1E70220FFF74AFD00283FF487AE05A993
:10090000142000F057F904210746049004A800F0D1
:10091000C5F83946B9E7322000F0A2F8071EFFF605
:1009200075AEBB077FF472AE384A926807EB0903D5
:1009300093423FF66BAE0220FFF728FD00283FF4FC
:1009400065AE27F003074F44B9453FF4A9AE4846CA
:1009500000F0D0F80421059005A800F09FF809F1F7
:100960000409F1E74FF47A70FFF710FD00283FF417
:100970004DAE00F009F9002844D00A9B01330BD09A
:1009800008220AA9002000F0BFF900283AD020224E
:10099000FF210AA800F0B0F9FFF700FD1C4800F0A5
:1009A00055FF13B0BDE8F08F002E3FF42FAE0BF0D3
:1009B0000B030B2B7FF42AAE0023642105A80593BB
:1009C00000F062F8074600287FF420AE0220FFF70F
:1009D000DDFC804600283FF419AEFFF7DFFC41F252
:1009E000883000F033FF059800F004FA464600F026
:1009F000CFF93C46BBE5064652E64FF0000905E656
:100A0000BA467EE637467CE65C22002000220020C3
:100A1000A086010070B50F4B1B780133DBB2012BB0
:100A20000C4611D80C4D29684FF47A730E6AA2FB5C
:100A30000332014622462846B047844204D1074B80
:100A400000221A70012070BD4FF4FA7000F0FEFE13
:100A50000020F8E710220020082600209423002020
:100A600007B50023024601210DF107008DF807307C
:100A7000FFF7D0FF20B19DF8070003B05DF804FB3D
:100A80004FF0FF30F9E700000A4608B50421FFF7F0
:100A9000C1FF80F00100C0B2404208BD30B4054C37
:100AA0002368DD69044B0A46AC460146204630BC4B
:100AB000604700BF08260020A086010070B501F045
:100AC000E5F9094E094D30800024286833888342B7
:100AD00008D901F0D5F92B6804440133B4F5803FFF
:100AE0002B60F2D370BD00BF962300206823002046
:100AF00001F07ABA00F1006000F5803000687047BC
:100B000000F10060920000F5803001F005BA0000AD
:100B1000054B1A68054B1B889B1A834202D9104467
:100B200001F0AEB900207047682300209623002012
:100B300038B5084D044629B128682044BDE838403E
:100B400001F0BEB92868204401F0A2F90028F3D0D2
:100B500038BD00BF6823002010F003030AD1B0F5B0
:100B6000047F05D200F10050A0F51040D0F8003805
:100B7000184670470023FBE700F10050A0F5104035
:100B8000D0F8100A70470000064991F8243033B1BC
:100B90000023086A81F824300822FFF7B1BF012042
:100BA000704700BF6C230020014B1868704700BFDE
:100BB000002004E070B5194B1D68194B0138C5F3CE
:100BC0000B0408442D0C04221E88A6420BD15C683D
:100BD0000A46013C824213460FD214F9016F4EB10E
:100BE00002F8016BF6E7013A03F10803ECD1814208
:100BF0000B4602D22C2203F8012B0A4A0524168840
:100C0000AE4204D1984284BF967803F8016B013C50
:100C100002F10402F3D1581A70BD00BF002004E0B5
:100C2000C4340008B0340008022804D1054B4FF04A
:100C300080429A6170470128FCD1024B4FF000526C
:100C4000F7E700BF00000240022804D1054B4FF433
:100C500080429A6170470128FCD1024B4FF4005248
:100C6000F7E700BF00000240022805D1064A536999
:100C700083F48043536170470128FCD1024A5369D1
:100C800083F40053F6E700BF0000024070B504464D
:100C90004FF47A764CB1412C254628BF412506FBFE
:100CA00005F000F0D3FD641BF4E770BD10B5002320
:100CB000934203D0CC5CC4540133F9E710BD00006B
:100CC00010B5013810F9013F3BB191F900409C4249
:100CD00003D11AB10131013AF4E71AB191F90020B8
:100CE000981A10BD1046FCE703460246D01A12F9C6
:100CF000011B0029FAD1704702440346934202D0F7
:100D000003F8011BFAE770472DE9F8431F4D14461D
:100D100095F824200746884652BBDFF870909CB3B4
:100D200095F824302BB92022FF2148462F62FFF787
:100D3000E3FF95F82400C0F10802A24228BF224632
:100D4000D6B24146920005EB8000FFF7AFFF95F861
:100D50002430A41B1E44F6B2082E17449044E4B27B
:100D600085F82460DBD1FFF70FFF0028D7D108E01A
:100D70002B6A03EB82038342CFD0FFF705FF0028E5
:100D8000CBD10020BDE8F8830120FBE76C230020D5
:100D9000024B1A78024B1A70704700BF9423002050
:100DA0001022002010B5104C104800F0B5F8214674
:100DB0000E4800F0DDF82468626DD2F8043843F084
:100DC0000203C2F804384FF47A70FFF75FFF084956
:100DD000204600F0D3F9626DD2F8043823F0020304
:100DE000C2F8043810BD00BF903500080826002066
:100DF000983500087047000030B5094D0A4491420B
:100E00000DD011F8013B5840082340F30004013B8A
:100E10002C4013F0FF0384EA5000F6D1EFE730BD19
:100E20002083B8ED026843681143016003B118479D
:100E30007047000013B5446BD4F894341A681178E5
:100E4000042915D1217C022912D119791289012393
:100E50008B4013420CD101A904F14C0001F0F8FEC3
:100E6000D4F89444019B21790246206800F0D0F91F
:100E700002B010BD143001F07BBE00004FF0FF3314
:100E8000143001F075BE00004C3001F04DBF000081
:100E90004FF0FF334C3001F047BF0000143001F039
:100EA00049BE00004FF0FF31143001F043BE000096
:100EB0004C3001F019BF00004FF0FF324C3001F010
:100EC00013BF00000020704710B5D0F894341A68A2
:100ED00011780429044617D1017C022914D15979CB
:100EE000528901238B4013420ED1143001F0DCFDF6
:100EF000024648B1D4F894444FF480736179206875
:100F0000BDE8104000F072B910BD0000406BFFF763
:100F1000DBBF0000704700007FB5124B0360002369
:100F20004360C0E90233012502260F4B05740446D5
:100F30000290019300F18402294600964FF48073D9
:100F4000143001F08DFD094B0294CDE9006304F5E6
:100F500023724FF48073294604F14C0001F054FED3
:100F600004B070BDE43400080D0F0008350E000811
:100F70000B68302282F311880A7903EB82029061B8
:100F80004A79093243F822008A7912B103EB8203CD
:100F900098610223C0F894140374002080F3118830
:100FA0007047000038B5037F044613B190F8543001
:100FB000ABB9201D01250221FFF734FF04F1140015
:100FC00025776FF0010100F069FC84F8545004F1BA
:100FD0004C006FF00101BDE8384000F05FBC38BD47
:100FE00010B5012104460430FFF71CFF00232377CE
:100FF00084F8543010BD000038B504460025143084
:1010000001F046FD04F14C00257701F015FE201D8E
:1010100084F854500121FFF705FF2046BDE8384011
:10102000FFF752BF90F8443003F06003202B07D144
:1010300090F84520212A4FF0000303D81F2A06D834
:1010400000207047222AFBD1C0E90E3303E0034A97
:1010500082630722C26303640120704711220020CB
:1010600037B5D0F894341A681178042904461AD197
:10107000017C022917D11979128901238B4013426F
:1010800011D100F14C05284601F096FE58B101A996
:10109000284601F0DDFDD4F89444019B21790246F5
:1010A000206800F0B5F803B030BD0000F0B500EBEB
:1010B000810385B09E6904460D46FEB1302383F35B
:1010C000118804EB8507301D0821FFF7ABFEFB6894
:1010D0005B691B6806F14C001BB1019001F0C6FD75
:1010E000019803A901F0B4FD024648B1039B2946CB
:1010F000204600F08DF8002383F3118805B0F0BD81
:10110000FB685A691268002AF5D01B8A013B13401C
:10111000F1D104F14402EAE7093138B550F8214031
:10112000DCB1302383F31188D4F894241368527906
:1011300003EB8203DB689B695D6845B1042160189D
:10114000FFF770FE294604F1140001F0B7FC2046B9
:10115000FFF7BAFE002383F3118838BD7047000003
:1011600001F016B8012303700023C0E90133C36105
:1011700083620362C36243620363704738B5044607
:10118000302383F311880025C0E90355C0E90555D4
:10119000416001F00DF80223237085F31188284681
:1011A00038BD000070B500EB810305465069DA6078
:1011B0000E46144618B110220021FFF79DFDA069CC
:1011C00018B110220021FFF797FD31462846BDE8EF
:1011D000704001F0B7B80000826802F0011282602E
:1011E0000022C0E90422826101F038B9F0B400EBBA
:1011F00081044789E4680125A4698D403D43458108
:1012000023600023A2606360F0BC01F053B90000CA
:10121000F0B400EB81040789E468012564698D401E
:101220003D43058123600023A2606360F0BC01F0B0
:10123000CDB9000070B50223002504460370C0E953
:101240000255C0E90455C564856180F8345001F049
:1012500015F863681B6823B129462046BDE8704035
:10126000184770BD0378052B10B504460AD080F8E6
:1012700050300523037043681B680BB10421984765
:101280000023A36010BD00000178052906D190F865
:101290005020436802701B6803B118477047000074
:1012A00070B590F83430044613B1002380F8343020
:1012B00004F14402204601F0F3F863689B68B3B977
:1012C00094F8443013F0600535D00021204601F039
:1012D00093FB0021204601F085FB63681B6813B176
:1012E000062120469847062384F8343070BD2046F6
:1012F00098470028E4D0B4F84A30E26B9A4288BF9D
:10130000E36394F94430E56B002B4FF0300380F237
:101310000381002D00F0F280092284F8342083F349
:1013200011880021D4E90E232046FFF771FF002326
:1013300083F31188DAE794F8452003F07F0343EA4A
:10134000022340F20232934200F0C58021D8B3F567
:10135000807F48D00DD8012B3FD0022B00F0938026
:10136000002BB2D104F14C02A2630222E263236497
:10137000C1E7B3F5817F00F09B80B3F5407FA4D136
:1013800094F84630012BA0D1B4F84C3043F002035E
:1013900032E0B3F5006F4DD017D8B3F5A06F31D060
:1013A000A3F5C063012B90D8636894F846205E686B
:1013B00094F84710B4F848302046B047002884D04D
:1013C0004368A3630368E3631AE0B3F5106F36D094
:1013D00040F6024293427FF478AF5C4BA363022352
:1013E000E3630023C3E794F84630012B7FF46DAF2D
:1013F000B4F84C3023F00203C4E90E55A4F84C3085
:10140000256478E7B4F84430B3F5A06F0ED194F8B2
:10141000463084F84E30204600F088FF63681B6831
:1014200013B1012120469847032323700023C4E908
:101430000E339CE704F14F03A3630123C3E7237832
:10144000042B10D1302383F311882046FFF7C4FE0C
:1014500085F311880321636884F84F5021701B685D
:101460000BB12046984794F84630002BDED084F824
:101470004F300423237063681B68002BD6D00221F1
:1014800020469847D2E794F848301D0603F00F0134
:1014900020460AD500F0F6FF012804D002287FF488
:1014A00014AF2B4B9AE72B4B98E700F0DDFFF3E7E7
:1014B00094F84630002B7FF408AF94F8483013F0CE
:1014C0000F01B3D01A06204602D501F0A9FAADE704
:1014D00001F09CFAAAE794F84630002B7FF4F5AEB1
:1014E00094F8483013F00F01A0D01B06204602D517
:1014F00001F082FA9AE701F075FA97E7142284F86E
:10150000342083F311882B462A4629462046FFF7CC
:101510006DFE85F31188E9E65DB1152284F834206B
:1015200083F311880021D4E90E232046FFF75EFEE5
:10153000FDE60B2284F8342083F311882B462A46DB
:1015400029462046FFF764FEE3E700BF1435000894
:101550000C3500081035000838B590F834300446D2
:10156000002B3ED0063BDAB20F2A34D80F2B32D8EC
:10157000DFE803F037313108223231313131313196
:1015800031313737C56BB0F84A309D4214D2C36849
:101590001B8AB5FBF3F203FB12556DB9302383F3BD
:1015A00011882B462A462946FFF732FE85F311881B
:1015B0000A2384F834300EE0142384F834303023C6
:1015C00083F3118800231A4619462046FFF70EFEC2
:1015D000002383F3118838BD036C03B198470023BF
:1015E000E7E70021204601F007FA0021204601F03C
:1015F000F9F963681B6813B1062120469847062352
:10160000D7E7000010B590F83430142B044629D0E9
:1016100017D8062B05D001D81BB110BD093B022BF2
:10162000FBD80021204601F0E7F90021204601F017
:10163000D9F963681B6813B1062120469847062331
:1016400019E0152BE9D10B2380F83430302383F3D4
:10165000118800231A461946FFF7DAFD002383F3A9
:101660001188DAE7C3689B695B68002BD5D1036CEE
:1016700003B19847002384F83430CEE70023037584
:10168000826803691B6899689142FBD25A680360BB
:1016900042601060586070470023037582680369D8
:1016A0001B6899689142FBD85A68036042601060D9
:1016B0005860704708B50846302383F311880B7DC6
:1016C000032B05D0042B0DD02BB983F3118808BD53
:1016D0008B6900221A604FF0FF338361FFF7CEFF62
:1016E0000023F2E7D1E9003213605A60F3E700000B
:1016F000FFF7C4BF054BD9680875186802681A60FF
:10170000536001220275D860FEF7FCBD98230020CB
:1017100030B50C4BDD684B1C87B004460FD02B4610
:10172000094A684600F04EF92046FFF7E3FF009BA8
:1017300013B1684600F050F9A86907B030BDFFF753
:10174000D9FFF9E798230020B5160008044B1A6862
:10175000DB6890689B68984294BF00200120704726
:1017600098230020084B10B51C68D86822681A60BE
:10177000536001222275DC60FFF78EFF0146204690
:10178000BDE81040FEF7BEBD9823002038B5074CD9
:1017900007490848012300252370656001F044FBD8
:1017A0000223237085F3118838BD00BF0026002076
:1017B0001C3500089823002000F044B9034A516802
:1017C00053685B1A9842FBD8704700BF001000E0D6
:1017D0008B60022308618B82084670478368A3F1FF
:1017E000840243F8142C026943F8442C426943F8FC
:1017F000402C094A43F8242CC26843F8182C0222D2
:1018000003F80C2C002203F80B2C044A43F8102C8C
:10181000A3F12000704700BF1D030008982300209B
:1018200008B5FFF7DBFFBDE80840FFF761BF000028
:10183000024BDB6898610F20FFF75CBF9823002004
:10184000302383F31188FFF7F3BF000008B501468A
:10185000302383F311880820FFF75AFF002383F316
:10186000118808BD064BDB6839B1426818605A60C0
:10187000136043600420FFF74BBF4FF0FF30704709
:10188000982300200368984206D01A6802605060CE
:1018900099611846FFF72CBF7047000038B5044621
:1018A0000D462068844200D138BD036823605C6027
:1018B0008561FFF71DFFF4E710B503689C68A2423D
:1018C0000CD85C688A600B604C6021605960996834
:1018D0008A1A9A604FF0FF33836010BD1B68121B99
:1018E000ECE700000A2938BF0A2170B504460D460E
:1018F0000A26601901F092FA01F07EFA041BA54253
:1019000003D8751C2E460446F3E70A2E04D9BDE819
:101910007040012001F0C8BA70BD0000F8B5144B4A
:101920000D46D96103F1100141600A2A19698260EC
:1019300038BF0A22016048601861A818144601F0F7
:101940005FFA0A2701F058FA431BA342064606D362
:101950007C1C281901F062FA27463546F2E70A2F67
:1019600004D9BDE8F840012001F09EBAF8BD00BFDF
:1019700098230020F8B506460D4601F03DFA0F4ABF
:10198000134653F8107F9F4206D12A46014630463F
:10199000BDE8F840FFF7C2BFD169BB68441A2C19F3
:1019A00028BF2C46A34202D92946FFF79BFF2246B7
:1019B00031460348BDE8F840FFF77EBF982300207A
:1019C000A823002010B4C0E9032300235DF8044BD2
:1019D0004361FFF7CFBF000010B5194C236998424F
:1019E0000DD0D0E90032816813605A609A680A44C9
:1019F0009A60002303604FF0FF33A36110BD2346BC
:101A0000026843F8102F53600022026022699A4254
:101A100003D1BDE8104001F0FBB9936881680B4425
:101A2000936001F0E9F92269E1699268441AA242DF
:101A3000E4D91144BDE81040091AFFF753BF00BFB5
:101A4000982300202DE9F047DFF8BC8008F110074B
:101A50002C4ED8F8105001F0CFF9D8F81C40AA68E5
:101A6000031B9A423ED81444D5E900324FF00009D6
:101A7000C8F81C4013605A60C5F80090D8F81030C0
:101A8000B34201D101F0C4F989F31188D5E90331DA
:101A900028469847302383F311886B69002BD8D0F0
:101AA00001F0AAF96A69A0EB04094A4582460DD201
:101AB000022001F0F9F90022D8F81030B34208D121
:101AC00051462846BDE8F047FFF728BF121A2244C6
:101AD000F2E712EB090938BF4A4629463846FFF7B4
:101AE000EBFEB5E7D8F81030B34208D01444211A01
:101AF000C8F81C00A960BDE8F047FFF7F3BEBDE8D9
:101B0000F08700BFA8230020982300200020704702
:101B1000FEE70000704700004FF0FF307047000004
:101B200002290CD0032904D00129074818BF00203E
:101B30007047032A05D8054800EBC20070470448E7
:101B400070470020704700BFF435000820220020B5
:101B5000A835000870B59AB00546084601A9144694
:101B600000F0C2F801A8FFF7BFF8431C5B00C5E90D
:101B700000340022237003236370C6B201AB023429
:101B80001046D1B28E4204F1020401D81AB070BDE1
:101B900013F8011B04F8021C04F8010C0132F0E7F1
:101BA00008B5302383F311880348FFF759FA00235F
:101BB00083F3118808BD00BF0826002090F8443048
:101BC00003F01F02012A07D190F845200B2A03D108
:101BD0000023C0E90E3315E003F06003202B08D189
:101BE000B0F848302BB990F84520212A03D81F2A95
:101BF00004D8FFF717BA222AEBD0FAE7034A826328
:101C00000722C26303640120704700BF182200202E
:101C100007B5052917D8DFE801F0191603191920AF
:101C2000302383F31188104A01900121FFF7BAFA9B
:101C300001980E4A0221FFF7B5FA0D48FFF7DCF9CB
:101C4000002383F3118803B05DF804FB302383F392
:101C500011880748FFF7A6F9F2E7302383F31188CC
:101C60000348FFF7BDF9EBE7483500086C3500087D
:101C70000826002038B50C4D0C4C0D492A4604F1BD
:101C80000800FFF767FF05F1CA0204F110000949D7
:101C9000FFF760FF05F5CA7204F118000649BDE8B8
:101CA0003840FFF757BF00BFD02A00202022002075
:101CB00028350008323500083D35000870B5044667
:101CC00008460D46FFF710F8C6B2204601340378E7
:101CD0000BB9184670BD32462946FEF7F1FF0028C1
:101CE000F3D10120F6E700002DE9F04705460C4648
:101CF000FEF7FAFF2B49C6B22846FFF7DFFF08B10F
:101D00000736F6B228492846FFF7D8FF08B1103643
:101D1000F6B2632E0BD8DFF88C80DFF88C90234F5F
:101D2000DFF894A02E7846B92670BDE8F0872946E2
:101D30002046BDE8F04701F09DBB252E2ED107229D
:101D400041462846FEF7BCFF70B9194B224603F105
:101D50000C0153F8040B42F8040B8B42F9D11B8899
:101D6000138007350E34DDE7082249462846FEF782
:101D7000A7FF98B90F4BA21C197809090232C95D57
:101D800002F8041C13F8011B01F00F015345C95D53
:101D900002F8031CF0D118340835C3E704F8016BCE
:101DA0000135BFE7143600083D3500082B36000822
:101DB0001C360008107AFF1F1C7AFF1FBFF34F8FDD
:101DC000024AD368DB03FCD4704700BF003C0240EA
:101DD00008B5094B1B7873B9FFF7F0FF074B1A6979
:101DE000002ABFBF064A5A6002F188325A601A6858
:101DF00022F480621A6008BD2E2D0020003C0240B3
:101E00002301674508B50B4B1B7893B9FFF7D6FF45
:101E1000094B1A6942F000421A611A6842F4805272
:101E20001A601A6822F480521A601A6842F48062BA
:101E30001A6008BD2E2D0020003C02400B28F0B592
:101E400016D80C4C0C4923787BB90C4D0E460C234C
:101E50004FF0006255F8047B46F8042B013B13F069
:101E6000FF033A44F6D10123237051F82000F0BD5E
:101E70000020FCE7602D0020302D00203C360008BB
:101E8000014B53F8200070473C3600080C20704787
:101E90000B2810B5044601D9002010BDFFF7CEFF76
:101EA000064B53F824301844C21A0BB90120F4E74A
:101EB00012680132F0D1043BF6E700BF3C3600085F
:101EC0000B2810B5044621D8FFF778FFFFF780FFF5
:101ED0000F4AF323D360C300DBB243F4007343F033
:101EE00002031361136943F480331361FFF766FF44
:101EF000FFF7A4FF074B53F8241000F0D9F8FFF7C1
:101F000081FF2046BDE81040FFF7C2BF002010BD92
:101F1000003C02403C360008F8B512F001031446BC
:101F200042D18218B2F1016F57D82D4B1B6813F0C4
:101F3000010352D02B4DFFF74BFFF323EB60FFF76C
:101F40003DFF40F20127032C15D824F00104661848
:101F5000244C401A40F20117B142236900EB0105FD
:101F600024D123F001032361FFF74CFF0120F8BDCA
:101F7000043C0430E7E78307E7D12B6923F440737F
:101F80002B612B693B432B6151F8046B0660BFF357
:101F90004F8FFFF713FF03689E42E9D02B6923F0B0
:101FA00001032B61FFF72EFF0020E0E723F44073CD
:101FB000236123693B4323610B882B80BFF34F8F41
:101FC000FFF7FCFE2D8831F8023BADB2AB42C3D027
:101FD000236923F001032361E4E71846C7E700BF44
:101FE00000380240003C0240084908B50B7828B18F
:101FF0001BB9FFF7EDFE01230B7008BD002BFCD0D1
:10200000BDE808400870FFF7FDBE00BF2E2D002080
:1020100010B50244064BD2B2904200D110BD441C10
:1020200000B253F8200041F8040BE0B2F4E700BF1F
:10203000502800400F4B30B51C6F240407D41C6F90
:1020400044F400741C671C6F44F400441C670A4C81
:10205000236843F4807323600244084BD2B2904259
:1020600000D130BD441C00B251F8045B43F820504D
:10207000E0B2F4E700380240007000405028004011
:1020800007B5012201A90020FFF7C2FF019803B0A4
:102090005DF804FB13B50446FFF7F2FFA04205D03C
:1020A000012201A900200194FFF7C4FF02B010BD76
:1020B00070470000034B1A681AB9034AD2F8742813
:1020C0001A607047642D00200030024008B5FFF709
:1020D000F1FF024B1868C0F3407008BD642D00206A
:1020E00070470000FEE700000A4B0B480B4A904285
:1020F0000BD30B4BDA1C121AC11E22F003028B42C7
:1021000038BF00220021FEF7F7BD53F8041B40F84A
:10211000041BECE7E8370008602E0020602E00204A
:10212000602E002070B5D0E915439E6800224FF064
:10213000FF3504EB42135101D3F800090028BEBF5C
:10214000D3F8000940F08040C3F80009D3F8000B31
:102150000028BEBFD3F8000B40F08040C3F8000B4E
:10216000013263189642C3F80859C3F8085BE0D2FD
:102170004FF00113C4F81C3870BD0000890141F014
:102180002001016103699B06FCD41220FFF716BBF6
:1021900010B5054C2046FEF7E5FF4FF0A043636500
:1021A000024BA36510BD00BF682D002090360008CB
:1021B00070B50378012B054650D12A4B446D9842E7
:1021C0001BD1294B5A6B42F080025A635A6D42F080
:1021D00080025A655A6D5A6942F080025A615A6902
:1021E00022F080025A610E2143205B6900F022FC3C
:1021F0001E4BE3601E4BC4F800380023C4F8003EB9
:10220000C02323606E6D4FF40413A3633369002B66
:10221000FCDA012333610C20FFF7D0FA3369DB07C6
:10222000FCD41220FFF7CAFA3369002BFCDA00262F
:10223000A6602846FFF776FF6B68C4F81068DB6875
:10224000C4F81468C4F81C684BB90A4BA3614FF07A
:10225000FF336361A36843F00103A36070BD064BC5
:10226000F4E700BF682D0020003802404014004011
:1022700003002002003C30C0083C30C0F8B5446D7B
:10228000054600212046FFF779FFA96D00234FF096
:1022900001128F68C4F834384FF00066C4F81C2867
:1022A0004FF0FF3004EB431201339F42C2F8006944
:1022B000C2F8006BC2F80809C2F8080BF2D20B682A
:1022C0006A6DEB65636210231361166916F01006E0
:1022D000FBD11220FFF772FAD4F8003823F4FE6322
:1022E000C4F80038A36943F4402343F01003A3610A
:1022F0000923C4F81038C4F814380A4BEB604FF0C7
:10230000C043C4F8103B084BC4F8003BC4F8106944
:10231000C4F80039EB6D03F1100243F48013EA6551
:10232000A362F8BD6C36000840800010426D90F842
:102330004E10D2F8003823F4FE6343EA0113C2F8CA
:10234000003870472DE9F84300EB8103456DDA68EA
:10235000166806F00306731E022B05EB41130C46AC
:1023600080460FFA81F94FEA41104FF00001C3F89F
:10237000101B4FF0010104F1100398BFB60401FADD
:1023800003F391698EBF334E06F1805606F5004681
:1023900000293AD0578A04F15801490137436F5058
:1023A000D5F81C180B43C5F81C382B180021C3F8AE
:1023B000101953690127611EA7409BB3138A928BA2
:1023C0009B08012A88BF5343D8F85C20981842EA3A
:1023D000034301F1400205EB8202C8F85C0021468C
:1023E00053602846FFF7CAFE08EB8900C3681B8AC2
:1023F00043EA8453483464011E432E51D5F81C38F7
:102400001F43C5F81C78BDE8F88305EB4917D7F8DA
:10241000001B21F40041C7F8001BD5F81C1821EA65
:102420000303C0E704F13F0305EB83030A4A5A6044
:1024300028462146FFF7A2FE05EB4910D0F80039E7
:1024400023F40043C0F80039D5F81C3823EA070705
:10245000D7E700BF0080001000040002826D126800
:10246000C265FFF75FBE00005831436D49015B58FC
:1024700013F4004004D013F4001F0CBF022001200D
:10248000704700004831436D49015B5813F4004028
:1024900004D013F4001F0CBF02200120704700007D
:1024A00000EB8101CB68196A0B6813604B685360BD
:1024B0007047000000EB810330B5DD68AA6913683E
:1024C000D36019B9402B84BF402313606B8A146812
:1024D000426D1C44013CB4FBF3F46343033323F02B
:1024E000030302EB411043EAC44343F0C043C0F886
:1024F000103B2B6803F00303012B09B20ED1D2F875
:10250000083802EB411013F4807FD0F8003B14BF71
:1025100043F0805343F00053C0F8003B02EB4112FC
:10252000D2F8003B43F00443C2F8003B30BD00004A
:102530002DE9F041244D6E6D06EB40130446D3F8AF
:10254000087BC3F8087B38070AD5D6F81438190772
:1025500006D505EB84032146DB6828465B6898476F
:10256000FA071FD5D6F81438DB071BD505EB840313
:10257000D968CCB98B69488A5A68B2FBF0F600FB7F
:1025800016228AB91868DA6890420DD2121AC3E985
:102590000024302383F311880B482146FFF78AFF7C
:1025A00084F31188BDE8F081012303FA04F26B89FA
:1025B00023EA02036B81CB68002BF3D0214602484B
:1025C000BDE8F041184700BF682D002000EB8103F3
:1025D00070B5DD68436D6C692668E6604A0156BBDC
:1025E0001A444FF40020C2F810092A6802F00302CE
:1025F000012A0AB20ED1D3F8080803EB421410F4F2
:10260000807FD4F8000914BF40F0805040F00050A3
:10261000C4F8000903EB4212D2F8000940F004406C
:10262000C2F80009D3F83408012202FA01F101438B
:10263000C3F8341870BD19B9402E84BF4020206003
:1026400020682E8A8419013CB4FBF6F440EAC440A9
:1026500040F000501A44C6E72DE9F8433B4D6E6D3B
:1026600006EB40130446D3F80889C3F8088918F02C
:10267000010F4FEA40171AD0D6F81038DB0716D5ED
:1026800005EB8003D9684B691868DA68904230D24C
:10269000121A4FF000091A60C3F80490302383F334
:1026A000118821462846FFF791FF89F3118818F019
:1026B000800F1CD0D6F834380126A640334216D0FD
:1026C00005EB84036D6DD3F80CC0DCF814200134E5
:1026D000E4B2D2F800E005EB04342F4451687145B0
:1026E00015D3D5F8343823EA0606C5F83468BDE8B2
:1026F000F883012303FA04F22B8923EA02032B81D6
:102700008B68002BD3D0214628469847CFE7BCF8EA
:102710001000AEEB0103834228BF0346D7F8180927
:1027200080B2B3EB800FE2D89068A0F1040959F8A9
:10273000048FC4F80080A0EB09089844B8F1040F96
:10274000F5D818440B4490605360C7E7682D00200B
:102750002DE9F74FA24C656D6E69AB691E4016F40A
:1027600080586E6107D02046FEF764FD03B0BDE8D7
:10277000F04F00F047BC002E12DAD5F8003E984822
:102780009B071EBFD5F8003E23F00303C5F8003EAB
:10279000D5F8043823F00103C5F80438FEF774FDBA
:1027A000370505D58E48FFF7BDFC8D48FEF75AFD6D
:1027B000B0040CD5D5F8083813F0060FEB6823F4F5
:1027C00070530CBF43F4105343F4A053EB60310734
:1027D0001BD56368DB681BB9AB6923F00803AB61E9
:1027E0002378052B0CD1D5F8003E7D489A071EBFF3
:1027F000D5F8003E23F00303C5F8003EFEF744FD84
:102800006368DB680BB176489847F30274D4B7026B
:1028100027D5D4F85490DFF8C8B100274FF0010A4B
:1028200009EB4712D2F8003B03F44023B3F5802FA5
:1028300011D1D2F8003B002B0DDA62890AFA07F3B6
:1028400022EA0303638104EB8703DB68DB6813B1CF
:10285000394658469847A36D01379B68FFB29F429F
:10286000DED9F00617D5676D3A6AC2F30A1002F096
:102870000F0302F4F012B2F5802F00F08580B2F55C
:10288000402F08D104EB83030022DB681B6A07F5A5
:10289000805790426AD13003D5F8184813D5E10328
:1028A00002D50020FFF744FEA20302D50120FFF766
:1028B0003FFE630302D50220FFF73AFE270302D54D
:1028C0000320FFF735FE75037FF550AFE00702D513
:1028D0000020FFF7C1FEA10702D50120FFF7BCFED3
:1028E000620702D50220FFF7B7FE23077FF53EAF50
:1028F0000320FFF7B1FE39E7636DDFF8E4A0019331
:1029000000274FF00109A36D9B685FFA87FB9B4589
:102910003FF67DAF019B03EB4B13D3F8001901F495
:102920004021B1F5802F1FD1D3F8001900291BDAFF
:10293000D3F8001941F09041C3F80019D3F80019F9
:102940000029FBDB5946606DFFF718FC218909FA65
:102950000BF321EA0303238104EB8B03DB689B6801
:1029600013B15946504698470137CCE7910708BF45
:10297000D7F80080072A98BF03F8018B02F1010203
:1029800098BF4FEA182884E7023304EB830207F567
:1029900080575268D2F818C0DCF80820DCE9001C27
:1029A000A1EB0C0C002188420AD104EB830463687C
:1029B0009B699A6802449A605A6802445A606AE7BE
:1029C00011F0030F08BFD7F800808C4588BF02F8CC
:1029D000018B01F1010188BF4FEA1828E3E700BF2E
:1029E000682D0020436D03EB4111D1F8003B43F407
:1029F0000013C1F8003B7047436D03EB4111D1F860
:102A0000003943F40013C1F800397047436D03EBFC
:102A10004111D1F8003B23F40013C1F8003B70478B
:102A2000436D03EB4111D1F8003923F40013C1F8D1
:102A30000039704700F1604303F561430901C9B2F1
:102A400083F80013012200F01F039A4043099B0002
:102A500003F1604303F56143C3F880211A607047B6
:102A600030B5039C0172043304FB0325C0E906530F
:102A7000049B03630021059BC160C0E90000C0E91D
:102A80000422C0E90842C0E90A11436330BD0000D6
:102A9000416A0022C0E90411C0E90A22C2606FF055
:102AA0000101FEF7FBBE0000D0E90432934201D1E0
:102AB000C2680AB9181D7047002070470369196081
:102AC000C2680132C260C2691344826903619342E1
:102AD00024BF436A03610021FEF7D4BE38B5044623
:102AE0000D46E3683BB16269131D1268A36213448B
:102AF000E362002007E0237A33B929462046FEF737
:102B0000B1FE0028EDDA38BD6FF00100FBE70000F0
:102B1000C368C269013BC36043691344826943616E
:102B2000934224BF436A436100238362036B03B172
:102B30001847704770B53023044683F31188866ABE
:102B40003EB9FFF7CBFF054618B186F3118828463A
:102B500070BDA36AE26A13F8015BA362934202D3D9
:102B60002046FFF7D5FF002383F31188EFE700002D
:102B70002DE9F84F04460E46174698464FF03009A7
:102B800089F311880025AA46D4F828B0BBF1000FBC
:102B900009D141462046FFF7A1FF20B18BF31188F0
:102BA0002846BDE8F88FD4E90A12A7EB050B521AA4
:102BB000934528BF9346BBF1400F1BD9334601F123
:102BC000400251F8040B43F8040B9142F9D1A36A77
:102BD00040334036A3624035D4E90A239A4202D3F7
:102BE0002046FFF795FF8AF31188BD42D8D289F3BA
:102BF0001188C9E730465A46FEF758F8A36A5B4485
:102C00005E44A3625D44E7E710B5029C01720433A1
:102C100003FB0421C0E906130023C0E90A33039B28
:102C20000363049BC460C0E90000C0E90422C0E95A
:102C30000842436310BD0000026AC260426AC0E9F4
:102C400004220022C0E90A226FF00101FEF726BE2D
:102C5000D0E904239A4201D1C26822B9184650F83B
:102C6000043B0B60704700231846FAE7C368C2694B
:102C70000133C3604369134482694361934224BFB3
:102C8000436A43610021FEF7FDBD000038B50446EC
:102C90000D46E3683BB123691A1DA262E269134441
:102CA000E362002007E0237A33B929462046FEF785
:102CB000D9FD0028EDDA38BD6FF00100FBE7000018
:102CC00003691960C268013AC260C269134482692B
:102CD0000361934224BF436A036100238362036B51
:102CE00003B118477047000070B530230D46044605
:102CF000114683F31188866A2EB9FFF7C7FF10B11A
:102D000086F3118870BDA36A1D70A36AE26A01335D
:102D10009342A36204D3E16920460439FFF7D0FF50
:102D2000002080F31188EDE72DE9F84F04460D46A9
:102D3000904699464FF0300A8AF311880026B34630
:102D4000A76A4FB949462046FFF7A0FF20B187F395
:102D500011883046BDE8F88FD4E90A073A1AA8EB83
:102D60000607974228BF1746402F1BD905F140039D
:102D700055F8042B40F8042B9D42F9D1A36A403347
:102D8000A3624036D4E90A239A4204D3E16920467B
:102D90000439FFF795FF8BF311884645D9D28AF3A2
:102DA0001188CDE729463A46FDF780FFA36A3B44E8
:102DB0003D44A3623E44E5E7D0E904239A4217D19B
:102DC000C3689BB1836A8BB1043B9B1A0ED013601E
:102DD000C368013BC360C3691A44836902619A42B4
:102DE00024BF436A036100238362012318467047AE
:102DF0000023FBE700F030B94FF08043586A70477A
:102E00004FF08043002258631A610222DA60704753
:102E10004FF080430022DA60704700004FF080439B
:102E200058637047FEE7000070B51B4B0163002537
:102E3000044686B0586085620E4600F0BFF804F183
:102E40001003C4E904334FF0FF33C4E90635C4E985
:102E50000044A560E562FFF7CFFF2B460246C4E9B8
:102E6000082304F134010D4A256580232046FEF72E
:102E7000AFFC0123E0600A4A037500927268019278
:102E8000B268CDE90223074B6846CDE90435FEF769
:102E9000C7FC06B070BD00BF002600209C360008AD
:102EA000A1360008252E0008024AD36A1843D062D2
:102EB000704700BF982300204B6843608B68836095
:102EC000CB68C3600B6943614B6903628B694362E2
:102ED0000B6803607047000008B5264B26481A6946
:102EE00040F2FF110A431A611A6922F4FF7222F0BC
:102EF00001021A611A691A6B0A431A631A6D0A43AE
:102F00001A651E4A1B6D1146FFF7D6FF02F11C0120
:102F100000F58060FFF7D0FF02F1380100F5806016
:102F2000FFF7CAFF02F1540100F58060FFF7C4FF0C
:102F300002F1700100F58060FFF7BEFF02F18C0125
:102F400000F58060FFF7B8FF02F1A80100F580608E
:102F5000FFF7B2FF02F1C40100F58060FFF7ACFF9C
:102F600002F1E00100F58060FFF7A6FFBDE8084030
:102F700000F0EEB80038024000000240A836000819
:102F800008B500F059FAFEF701FCFFF793F8BDE829
:102F90000840FEF76FBE000070470000EFF30983A2
:102FA00005494A6B22F001024A63683383F30988BA
:102FB000002383F31188704700EF00E0302080F396
:102FC000118862B60C4B0D4AD96821F4E0610904FE
:102FD000090C0A43DA60D3F8FC20094942F08072F8
:102FE000C3F8FC200A6842F001020A602022DA7766
:102FF00083F82200704700BF00ED00E00003FA05EF
:10300000001000E010B5302383F311880E4B5B688D
:1030100013F4006314D0F1EE103AEFF30984683C26
:103020004FF08073E361094BDB6B236684F30988FF
:10303000FEF78CFB10B1064BA36110BD054BFBE7FF
:1030400083F31188F9E700BF00ED00E000EF00E036
:103050002F030008320300080F4B1A6C42F00102E4
:103060001A641A6E42F001021A660C4A1B6E9368CB
:1030700043F0010393604FF0804353229A624FF074
:10308000FF32DA6200229A615A63DA605A600122E2
:103090005A611A60704700BF00380240002004E007
:1030A0004FF0804208B51169D3680B40D9B2C943CB
:1030B0009B07116107D5302383F31188FEF77CFB52
:1030C000002383F3118808BD1F4B1A696FEAC252AF
:1030D0006FEAD2521A611A69C2F308021A614FF0FC
:1030E000FF301A695A69586100215A6959615A6951
:1030F0001A6A62F080521A621A6A02F080521A62E8
:103100001A6A5A6A58625A6A59625A6A1A6C42F0C2
:1031100080521A641A6E42F080521A661A6E0B4A76
:10312000106840F480701060186F00F44070B0F5C3
:10313000007F1EBF4FF4803018671967536823F46F
:103140000073536000F054B9003802400070004032
:10315000334B4FF080521A64324A4FF440411160B1
:103160001A6842F001021A601A689107FCD59A6841
:1031700022F003029A602A4B9A6812F00C02FBD1EB
:10318000196801F0F90119609A601A6842F48032F6
:103190001A601A689203FCD55A6F42F001025A670E
:1031A0001F4B5A6F9007FCD51F4A5A601A6842F0AD
:1031B00080721A601B4A53685904FCD5184B1A6870
:1031C0009201FCD5194A9A60194B1A68194B9A4218
:1031D000194B21D1194A1168194A91421CD140F268
:1031E00005121A60144A136803F00F03052BFAD175
:1031F0000B4B9A6842F002029A609A6802F00C0245
:10320000082AFAD15A6C42F480425A645A6E42F447
:1032100080425A665B6E704740F20572E1E700BF7C
:10322000003802400070004008544007009488387D
:10323000002004E011640020003C024000ED00E0AA
:1032400041C20F41074A08B5536903F001035361B6
:1032500023B1054A13680BB150689847BDE8084090
:10326000FFF7D0BE003C0140E02D0020074A08B522
:10327000536903F00203536123B1054A93680BB10C
:10328000D0689847BDE80840FFF7BCBE003C01404D
:10329000E02D0020074A08B5536903F00403536189
:1032A00023B1054A13690BB150699847BDE808403E
:1032B000FFF7A8BE003C0140E02D0020074A08B5FA
:1032C000536903F00803536123B1054A93690BB1B5
:1032D000D0699847BDE80840FFF794BE003C014024
:1032E000E02D0020074A08B5536903F0100353612D
:1032F00023B1054A136A0BB1506A9847BDE80840EC
:10330000FFF780BE003C0140E02D0020164B10B5B9
:103310005C6904F478725A61A30604D5134A936A6F
:103320000BB1D06A9847600604D5104A136B0BB1F5
:10333000506B9847210604D50C4A936B0BB1D06BA8
:103340009847E20504D5094A136C0BB1506C9847B5
:10335000A30504D5054A936C0BB1D06C9847BDE822
:103360001040FFF74FBE00BF003C0140E02D0020A1
:10337000194B10B55C6904F47C425A61620504D5AE
:10338000164A136D0BB1506D9847230504D5134AA7
:10339000936D0BB1D06D9847E00404D50F4A136EBE
:1033A0000BB1506E9847A10404D50C4A936E0BB133
:1033B000D06E9847620404D5084A136F0BB1506F62
:1033C0009847230404D5054A936F0BB1D06F9847F3
:1033D000BDE81040FFF716BE003C0140E02D002084
:1033E00008B5FFF75DFEBDE80840FFF70BBE000023
:1033F000062108B50846FFF71DFB06210720FFF749
:1034000019FB06210820FFF715FB06210920FFF70D
:1034100011FB06210A20FFF70DFB06211720FFF7FD
:1034200009FB06212820FFF705FBBDE8084007211E
:103430001C20FFF7FFBA000008B5FFF745FE00F0BB
:103440000BF8FDF78DFEFDF765FDFFF7A5FDBDE867
:103450000840FFF7CFBC00000023054A194601339E
:10346000102BC2E9001102F10802F8D1704700BF29
:10347000E02D0020034611F8012B03F8012B002A50
:10348000F9D1704753544D3332463F3F3F005354B8
:103490004D3332463430780053544D333246343253
:1034A000780053544D3332463434365858000000B7
:1034B000012033000010410001105A000310590090
:1034C00007103100000000008434000813040000DD
:1034D0008E3400081904000098340008210400000C
:1034E000A234000800000000910E00087D0E0008C4
:1034F000B90E0008A50E0008B10E00089D0E0008C8
:10350000890E0008750E0008C50E000800000000B6
:1035100001000000000000006330000018350008C2
:10352000F0230020002600204172647550696C6F02
:10353000740025424F415244252D424C00255345ED
:103540005249414C2500000002000000000000002C
:10355000AD1000081911000840004000A02A00200A
:10356000B02A00200200000000000000030000005C
:10357000000000005D1100080000000010000000C5
:10358000C02A002000000000010000000000000030
:10359000682D002001010200111C0008211B0008F9
:1035A000BD1B0008A11B000843000000B035000847
:1035B00009024300020100C03209040000010202B6
:1035C0000100052400100105240100010424020269
:1035D0000524060001070582030800FF0904010015
:1035E000020A0000000705010240000007058102F1
:1035F0004000000012000000FC350008120110011C
:1036000002000040091241570002010203010000BC
:103610000403090425424F41524425004D6174655D
:103620006B463430352D57696E6700303132333494
:1036300035363738394142434445460000400000A2
:1036400000400000004000000040000000000100B9
:103650000000020000000200000002000000020062
:103660000000020000000200000002000000000054
:10367000A112000859150008051600084000400076
:10368000C82D0020C82D002001000000D82D0020EA
:103690008000000040010000030000006D61696EC1
:1036A0000069646C650000000A01A81600000000B3
:1036B000AAAAAAAA05011400FF9F00008800000022
:1036C00070A70A000000000100000000AAAAAAAA30
:1036D00000000001FFFF00000000000000000000EB
:1036E00000A0A01200000000AAAAAAAA005050112F
:1036F000FFFF0000000000880077080020000000A5
:1037000000000000AAAAAAAA10000000FFFF000003
:1037100000080000000000000000000000000000A1
:10372000AAAAAAAA00000000FFFF000000000000F3
:10373000000000000000000000000000AAAAAAAAE1
:1037400000000000FFFF000000000000000000007B
:103750000000000000000000AAAAAAAA00000000C1
:10376000FFFF00000000000000000000000000005B
:10377000000000000A00000000000000030000003C
:103780000000000000000000000000000000000039
:103790000000000000000000000000000000000029
:1037A00000000000000000007F000000000000009A
:1037B00000000F0000000000FF009600000000085D
:1037C0000096000000000800040000001036000809
:1037D00000000000000000000000000000000000E9
:1037E0000000000000000000FFFFFFFFFFFFFFFFE1
:1037F000FFFFFFFFFFFFFFFFFFFFFFFFFFFFFFFFD9
:10380000FFFFFFFFFFFFFFFFFFFFFFFFFFFFFFFFC8
:10381000FFFFFFFFFFFFFFFFFFFFFFFFFFFFFFFFB8
:10382000FFFFFFFFFFFFFFFFFFFFFFFFFFFFFFFFA8
:020000040801F1
:100000000006002099120108A5810908018109084C
:100010006D81090801810908398109089B120108CD
:100020009B1201089B1201089B120108A1FB0B08FF
:100030009B1201089B1201089B1201089B120108E8
:100040009B1201089B1201089B1201089B120108D8
:100050009B1201089B12010839070C0861070C0864
:1000600089070C08B1070C08D9070C0821AA0B084E
:1000700049AA0B0875AA0B08A1AA0B08CDAA0B0860
:10008000F5AA0B0821AB0B08A5A90B089B120108C8
:100090009B1201089B1201089B12010801080C0821
:1000A0004D090C0861090C0875090C0879090C0840
:1000B0007D090C0891090C08A5090C0879B30B08F7
:1000C0008DB30B08B1B30B08C5B30B089B12010825
:1000D0009B120108D5080C08E9080C08FD080C085B
:1000E00065080C089B1201089B120108C9090C083D
:1000F000CD090C08E1090C08E5090C084DAB0B080B
:100100009B1201089B120108B9090C089B120108F7
:1001100011090C0825090C089B1201089B12010803
:1001200079AB0B08A1AB0B08CDAB0B08F9AB0B08F7
:1001300025AC0B089B1201089B1201089B120108B9
:100140009B1201089B1201089B120108CD020C08AA
:100150004DAC0B0879AC0B08A5AC0B0839090C08A1
:100160009B1201089B1201089B1201089B120108B7
:100170009B1201089B1201089B1201089B120108A7
:100180009B1201089B1201089B1201089B12010897
:100190009B1201089B1201089B1201089B12010887
:1001A0009B1201089B1201089B1201089B12010877
:1001B0009B1201089B1201089B1201089B12010867
:1001C0009B1201089B1201089B1201089B12010857
:1001D0009B1201089B1201089B1201089B12010847
:1001E000915801086D7F020835F80308A1BA050887
:1001F000C5C0050801340608C198060885A0060890
:10020000BDA3060839090708692F0708FDEF07088D
:1002100001500808595D0808417309082578090844
:10022000818B0A0815E70A08790D0B08E5180B08F9
:1002300071480B089D4E0B080000000000000000F4
:1002400081F0004102E000BF83F0004330B54FEA87
:1002500041044FEA430594EA050F08BF90EA020FF4
:100260001FBF54EA000C55EA020C7FEA645C7FEA87
:10027000655C00F0E2804FEA5454D4EB5555B8BFAA
:100280006D420CDD2C4480EA020281EA030382EA1B
:10029000000083EA010180EA020281EA0303362DAD
:1002A00088BF30BD11F0004F4FEA01314FF4801C80
:1002B0004CEA113102D0404261EB410113F0004F92
:1002C0004FEA03334CEA133302D0524263EB430349
:1002D00094EA050F00F0A780A4F10104D5F1200EE7
:1002E0000DDB02FA0EFC22FA05F2801841F1000142
:1002F00003FA0EF2801843FA05F359410EE0A5F116
:1003000020050EF1200E012A03FA0EFC28BF4CF046
:10031000020C43FA05F3C01851EBE37101F00045FC
:1003200007D54FF0000EDCF1000C7EEB00006EEB09
:100330000101B1F5801F1BD3B1F5001F0CD3490893
:100340005FEA30004FEA3C0C04F101044FEA4452EA
:1003500012F5800F80F09A80BCF1004F08BF5FEA71
:10036000500C50F1000041EB045141EA050130BD51
:100370005FEA4C0C404141EB0101013C28BFB1F563
:10038000801FE9D291F0000F04BF01460020B1FAAE
:1003900081F308BF2033A3F10B03B3F120020CDA81
:1003A0000C3208DD02F1140CC2F10C0201FA0CF05F
:1003B00021FA02F10CE002F11402D8BFC2F1200CC4
:1003C00001FA02F120FA0CFCDCBF41EA0C0190407A
:1003D000E41AA2BF01EB0451294330BD6FEA0404C3
:1003E0001F3C1CDA0C340EDC04F11404C4F12002AE
:1003F00020FA04F001FA02F340EA030021FA04F3C0
:1004000045EA030130BDC4F10C04C4F1200220FA16
:1004100002F001FA04F340EA0300294630BD21FA54
:1004200004F0294630BD94F0000F83F4801306BF1A
:1004300081F480110134013D4EE77FEA645C18BF0E
:100440007FEA655C29D094EA050F08BF90EA020FA5
:1004500005D054EA000C04BF1946104630BD91EA9D
:10046000030F1EBF0021002030BD5FEA545C05D1A0
:100470004000494128BF41F0004130BD14F58004DF
:100480003CBF01F5801130BD01F0004545F0FE4153
:1004900041F470014FF0000030BD7FEA645C1ABF88
:1004A000194610467FEA655C1CBF0B46024650EABF
:1004B000013406BF52EA033591EA030F41F40021EB
:1004C00030BD00BF90F0000F04BF0021704730B571
:1004D0004FF4806404F132044FF000054FF0000146
:1004E00050E700BF90F0000F04BF0021704730B507
:1004F0004FF4806404F1320410F0004548BF4042DC
:100500004FF000013EE700BF42004FEAE2014FEA30
:1005100031014FEA02701FBF12F07F4393F07F4F0B
:1005200081F06051704732F07F4208BF704793F00E
:100530007F4F04BF41F40021704730B54FF4607421
:1005400001F0004521F000411CE700BF50EA010224
:1005500008BF704730B54FF000050AE050EA0102CD
:1005600008BF704730B511F0004502D5404261EB3D
:1005700041014FF4806404F132045FEA915C3FF47E
:10058000D8AE4FF003025FEADC0C18BF03325FEA1B
:10059000DC0C18BF033202EBDC02C2F1200300FACC
:1005A00003FC20FA02F001FA03FE40EA0E0021FAF1
:1005B00002F11444BDE600BF70B54FF0FF0C4CF4DF
:1005C000E06C1CEA11541DBF1CEA135594EA0C0F91
:1005D00095EA0C0F00F0DEF82C4481EA030621EACC
:1005E0004C5123EA4C5350EA013518BF52EA033507
:1005F00041F4801143F4801338D0A0FB02CE4FF0B9
:100600000005E1FB02E506F00042E0FB03E54FF0E8
:100610000006E1FB03569CF0000F18BF4EF0010EE0
:10062000A4F1FF04B6F5007F64F5407404D25FEADC
:100630004E0E6D4146EB060642EAC62141EA55518F
:100640004FEAC52040EA5E504FEACE2EB4F1FD0CD1
:1006500088BFBCF5E06F1ED8BEF1004F08BF5FEA4F
:10066000500E50F1000041EB045170BD06F0004601
:1006700046EA010140EA020081EA0301B4EB5C04AE
:10068000C2BFD4EB0C0541EA045170BD41F48011A6
:100690004FF0000E013C00F3AB8014F1360FDEBFCB
:1006A000002001F0004170BDC4F10004203C35DAA7
:1006B0000C341BDC04F11404C4F1200500FA05F32A
:1006C00020FA04F001FA05F240EA020001F00042CB
:1006D00021F0004110EBD37021FA04F642EB060141
:1006E0005EEA430E08BF20EAD37070BDC4F10C046B
:1006F000C4F1200500FA04F320FA05F001FA04F22F
:1007000040EA020001F0004110EBD37041F100011A
:100710005EEA430E08BF20EAD37070BDC4F1200525
:1007200000FA05F24EEA020E20FA04F301FA05F28D
:1007300043EA020321FA04F001F0004121FA04F235
:1007400020EA020000EBD3705EEA430E08BF20EA05
:10075000D37070BD94F0000F0FD101F0004640003F
:1007600041EB010111F4801F08BF013CF7D041EAC1
:10077000060195F0000F18BF704703F000465200C5
:1007800043EB030313F4801F08BF013DF7D043EA96
:100790000603704794EA0C0F0CEA135518BF95EA4C
:1007A0000C0F0CD050EA410618BF52EA4306D1D1D3
:1007B00081EA030101F000414FF0000070BD50EAF2
:1007C000410606BF1046194652EA430619D094EA7C
:1007D0000C0F02D150EA013613D195EA0C0F05D166
:1007E00052EA03361CBF104619460AD181EA0301BA
:1007F00001F0004141F0FE4141F470014FF0000072
:1008000070BD41F0FE4141F4780170BD70B54FF00C
:10081000FF0C4CF4E06C1CEA11541DBF1CEA13558C
:1008200094EA0C0F95EA0C0F00F0A7F8A4EB05046E
:1008300081EA030E52EA03354FEA013100F0888065
:100840004FEA03334FF0805545EA131343EA12632E
:100850004FEA022245EA111545EA10654FEA0026E3
:100860000EF000419D4208BF964244F1FD0404F59C
:10087000407402D25B084FEA3202B61A65EB0305F8
:100880005B084FEA32024FF480104FF4002CB6EBB5
:10089000020E75EB030E22BFB61A754640EA0C0035
:1008A0005B084FEA3202B6EB020E75EB030E22BF75
:1008B000B61A754640EA5C005B084FEA3202B6EBB6
:1008C000020E75EB030E22BFB61A754640EA9C0075
:1008D0005B084FEA3202B6EB020E75EB030E22BF45
:1008E000B61A754640EADC0055EA060E18D04FEA03
:1008F000051545EA16754FEA06164FEAC30343EAA3
:1009000052734FEAC2025FEA1C1CC0D111F4801F6F
:100910000BD141EA00014FF000004FF0004CB6E768
:1009200011F4801F04BF01430020B4F1FD0C88BF07
:10093000BCF5E06F3FF6AFAEB5EB030C04BFB6EB12
:10094000020C5FEA500C50F1000041EB045170BD05
:100950000EF0004E4EEA113114EB5C04C2BFD4EB32
:100960000C0541EA045170BD41F480114FF0000EB6
:10097000013C90E645EA060E8DE60CEA135594EA32
:100980000C0F08BF95EA0C0F3FF43BAF94EA0C0F35
:100990000AD150EA01347FF434AF95EA0C0F7FF4AA
:1009A00025AF104619462CE795EA0C0F06D152EAFE
:1009B00003353FF4FDAE1046194622E750EA4106E2
:1009C00018BF52EA43067FF4C5AE50EA41047FF4F3
:1009D0000DAF52EA43057FF4EBAE12E74FF0FF3C58
:1009E00006E000BF4FF0010C02E000BF4FF0010C29
:1009F0004DF804CD4FEA410C7FEA6C5C4FEA430CA2
:100A000018BF7FEA6C5C1BD001B050EA410C0CBFF0
:100A100052EA430C91EA030F02BF90EA020F002052
:100A2000704710F1000F91EA030F58BF994208BFB9
:100A300090422CBFD8176FEAE37040F00100704776
:100A40004FEA410C7FEA6C5C02D150EA013C07D1CD
:100A50004FEA430C7FEA6C5CD6D152EA033CD3D018
:100A60005DF8040B704700BF8446104662468C4612
:100A70001946634600E000BF01B5FFF7B7FF002845
:100A800048BF10F1000F01BD4DF808EDFFF7F4FF6E
:100A90000CBF012000205DF808FB00BF4DF808EDF9
:100AA000FFF7EAFF34BF012000205DF808FB00BF1C
:100AB0004DF808EDFFF7E0FF94BF012000205DF83E
:100AC00008FB00BF4DF808EDFFF7CEFF94BF0120F3
:100AD00000205DF808FB00BF4DF808EDFFF7C4FFEC
:100AE00034BF012000205DF808FB00BF4FEA410C35
:100AF0007FEA6C5C02D150EA013C0AD14FEA430C18
:100B00007FEA6C5C02D152EA033C02D14FF0000054
:100B100070474FF0010070474FEA410212F5001292
:100B200015D211D56FF47873B3EB625212D94FEA34
:100B3000C12343F0004343EA505311F0004F23FA1E
:100B400002F018BF404270474FF00000704750EA73
:100B5000013005D111F0004008BF6FF00040704730
:100B60004FF00000704700BF4A0011D212F500128A
:100B700011D20DD56FF47873B3EB62520ED44FEAF5
:100B8000C12343F0004343EA505323FA02F0704775
:100B90004FF00000704750EA013002D14FF0FF30B3
:100BA00070474FF0000070474FEA4102B2F1E04356
:100BB00024BFB3F5001CDCF1FE5C0DD901F0004C44
:100BC0004FEAC0024CEA5070B2F1004F40EB830094
:100BD00008BF20F00100704711F0804F21D113F1C0
:100BE0003872BCBF01F00040704741F480114FEAF9
:100BF0005252C2F11802C2F1200C10FA0CF320FA82
:100C000002F018BF40F001004FEAC1234FEAD3239E
:100C100003FA0CFC40EA0C0023FA02F34FEA430308
:100C2000CCE77FEA625307D150EA01331EBF4FF091
:100C3000FE4040F44000704701F0004040F0FE40AC
:100C400040F40000704700BF80F0004002E000BFA9
:100C500081F0004142001FBF5FEA410392EA030FA7
:100C60007FEA226C7FEA236C6AD04FEA1262D2EBF1
:100C70001363C1BFD218414048404140B8BF5B42F6
:100C8000192B88BF704710F0004F40F4000020F08F
:100C90007F4018BF404211F0004F41F4000121F0A5
:100CA0007F4118BF494292EA030F3FD0A2F10102EF
:100CB00041FA03FC10EB0C00C3F1200301FA03F12D
:100CC00000F0004302D5494260EB4000B0F5000F50
:100CD00013D3B0F1807F06D340084FEA310102F10F
:100CE0000102FE2A51D2B1F1004F40EBC25008BFC1
:100CF00020F0010040EA03007047490040EB00008B
:100D0000013A28BFB0F5000FEDD2B0FA80FCACF18B
:100D1000080CB2EB0C0200FA0CF0AABF00EBC250B8
:100D200052421843BCBFD0401843704792F0000FA6
:100D300081F4000106BF80F400000132013BB5E7F9
:100D40004FEA41037FEA226C18BF7FEA236C21D06F
:100D500092EA030F04D092F0000F08BF08467047D4
:100D600090EA010F1CBF0020704712F07F4F04D1A2
:100D7000400028BF40F00040704712F100723CBFB5
:100D800000F50000704700F0004343F0FE4040F4DF
:100D9000000070477FEA226216BF08467FEA23639D
:100DA0000146420206BF5FEA412390EA010F40F488
:100DB000800070474FF0000304E000BF10F00043D4
:100DC00048BF40425FEA000C08BF704743F09643BB
:100DD00001464FF000001CE050EA010208BF7047D6
:100DE0004FF000030AE000BF50EA010208BF70475D
:100DF00011F0004302D5404261EB41015FEA010C72
:100E000002BF84460146002043F0B64308BFA3F169
:100E10008053A3F50003BCFA8CF2083AA3EBC2534B
:100E200010DB01FA02FC634400FA02FCC2F120026A
:100E3000BCF1004F20FA02F243EB020008BF20F0A1
:100E40000100704702F1200201FA02FCC2F1200207
:100E500050EA4C0021FA02F243EB020008BF20EAFC
:100E6000DC7070477BB972B90029BEBF00204FF01B
:100E7000004106E008BF00281CBF6FF000414FF0A2
:100E8000FF3000F007BAADF1080C6DE904CE00297F
:100E900009DB002B1ADB00F095F8DDF804E0DDE952
:100EA000022304B07047404261EB4101002B1BDB81
:100EB00000F088F8DDF804E0DDE9022304B04042E8
:100EC00061EB4101524263EB43037047524263EBD3
:100ED000430300F077F8DDF804E0DDE9022304B015
:100EE000404261EB41017047524263EB430300F023
:100EF00069F8DDF804E0DDE9022304B0524263EB57
:100F00004303704753B94AB9002908BF00281CBFE2
:100F10004FF0FF314FF0FF3000F0BCB9ADF1080CDD
:100F20006DE904CE00F04EF8DDF804E0DDE90223BF
:100F300004B07047430803F05533C01A830803F028
:100F4000333300F03330184400EB101000F00F3052
:100F500000EB002000EB0040000E704707EE900A07
:100F6000F5EEC07AF1EE10FA01D400F00BB8F1EE14
:100F7000677A08B517EE900A00F004F8404261EB7A
:100F8000410108BDD0B5FFF7BFFA0C4B0022064661
:100F90000F46FFF711FBFFF7E7FD0446FFF792FA54
:100FA000074B0022FFF708FB02460B463046394646
:100FB000FFF74AF9FFF7D8FD2146D0BD0000F03D0C
:100FC0000000F0412DE9F047089D04468E46002BB5
:100FD0004DD18A42944669D9B2FA82F252B101FAED
:100FE00002F3C2F1200120FA01F10CFA02FC41EAFD
:100FF000030E94404FEA1C48210CBEFBF8F61FFA82
:101000008CF708FB16E341EA034306FB07F199421C
:101010000AD91CEB030306F1FF3080F01F819942CF
:1010200040F21C81023E63445B1AA4B2B3FBF8F0A9
:1010300008FB103344EA034400FB07F7A7420AD930
:101040001CEB040400F1FF3380F00A81A74240F258
:1010500007816444023840EA0640E41B00261DB1C3
:10106000D4400023C5E900433146BDE8F0878B42F8
:1010700009D9002D00F0EF800026C5E900013046B7
:101080003146BDE8F087B3FA83F6002E4AD18B4291
:1010900002D3824200F2F980841A61EB030301203B
:1010A0009E46002DE0D0C5E9004EDDE702B9FFDE27
:1010B000B2FA82F2002A40F09280A1EB0C014FEAD2
:1010C0001C471FFA8CFE0126200CB1FBF7F307FB2F
:1010D000131140EA01410EFB03F0884208D91CEBD2
:1010E000010103F1FF3802D2884200F2CB8043466F
:1010F000091AA4B2B1FBF7F007FB101144EA01444E
:101100000EFB00FEA64508D91CEB040400F1FF31DC
:1011100002D2A64500F2BB800846A4EB0E0440EACA
:1011200003409CE7C6F12007B34022FA07FC4CEAD3
:10113000030C20FA07F401FA06F31C43F9404FEAC6
:101140001C4900FA06F3B1FBF9F8200C1FFA8CFEDB
:1011500009FB181140EA014108FB0EF0884202FA2F
:1011600006F20BD91CEB010108F1FF3A80F08880F0
:10117000884240F28580A8F102086144091AA4B2AD
:10118000B1FBF9F009FB101144EA014100FB0EFE2E
:101190008E4508D91CEB010100F1FF346CD28E455D
:1011A0006AD90238614440EA0840A0FB0294A1EBEE
:1011B0000E01A142C846A64656D353D05DB1B3EB4B
:1011C000080261EB0E0101FA07F722FA06F3F1407B
:1011D0001F43C5E9007100263146BDE8F087C2F122
:1011E0002003D8400CFA02FC21FA03F3914001439A
:1011F0004FEA1C471FFA8CFEB3FBF7F007FB1036D3
:101200000B0C43EA064300FB0EF69E4204FA02F47E
:1012100008D91CEB030300F1FF382FD29E422DD9D1
:10122000023863449B1B89B2B3FBF7F607FB163306
:1012300041EA034106FB0EF38B4208D91CEB010186
:1012400006F1FF3816D28B4214D9023E6144C91A06
:1012500046EA004638E72E46284605E70646E3E616
:101260001846F8E64B45A9D2B9EB020864EB0C0E20
:101270000138A3E74646EAE7204694E74046D1E72F
:10128000D0467BE7023B614432E7304609E76444DD
:10129000023842E7704700BF02E000F000F8FEE7C6
:1012A00072B6374880F30888364880F30988364894
:1012B0003649086040F20000CCF200004EF634716E
:1012C000CEF200010860BFF34F8FBFF36F8F40F283
:1012D0000000C0F2F0004EF68851CEF20001086026
:1012E000BFF34F8FBFF36F8F4FF00000E1EE100A96
:1012F0004EF63C71CEF200010860062080F314889F
:10130000BFF36F8FAEF0AAFCADF012FD4FF0553079
:101310001F491B4A91423CBF41F8040BFAE71D49A3
:10132000184A91423CBF41F8040BFAE71A491B4A9C
:101330001B4B9A423EBF51F8040B42F8040BF8E7EE
:1013400000201849184A91423CBF41F8040BFAE7C3
:10135000AEF088FCADF040FD144C154DAC4203DA04
:1013600054F8041B8847F9E701F014F9114C124DA9
:10137000AC4203DA54F8041B8847F9E7AEF070BCBE
:1013800000060020002200200000010808ED00E017
:101390000000002000060020B09D0E080022002062
:1013A000002C0020002C0020F85E0120E001010844
:1013B0003802010838020108380201082DE9F04F0F
:1013C0002DED108AC1F80CD0C3689D46BDEC108A83
:1013D000BDE8F08F002383F311882846A047002042
:1013E000ADF02CFAFEE7ADF089F800DFFEE7000073
:1013F00001F0FF01102A2BDB10F0070F08D010F8C6
:10140000013B013A8B422DD010F0070F42B3F6D1C9
:10141000F0B441EA012141EA014122F007047FF0E2
:1014200000070023F0E80256083C85EA010586EA39
:10143000010685FA47F5A3FA87F586FA47F6A5FA75
:1014400087F68EB9EED1F0BC01F0FF0102F0070281
:1014500032B110F8013B013A83EA010313B1F8D12C
:101460000020704701387047002D06BF354603380D
:10147000073815F0010F07D1013015F4807F02BF46
:10148000013015F4C03F0130F0BC0138704700BF97
:1014900010F8012B11F8013B012A28BF9A42F7D01E
:1014A000D01A7047034613F8012B002AFBD1181AF3
:1014B0000138704738B50022002304460D46FFF777
:1014C000EDFA28B920462946BDE8384000F00AB8B0
:1014D000204605F1004100F005F8404261EB410172
:1014E00038BD00BFD0B50C4B002206460F46FFF7B3
:1014F00063F8FFF739FB0446FEF7E4FF074B0022D1
:10150000FFF75AF802460B4630463946FEF79CFE76
:10151000FFF72AFB2146D0BD0000F03D0000F0415E
:10152000036800221B68184710B503685B6804460F
:10153000984708B194F84D0010BD000038B5044636
:101540007CF0DCFF0E4B1D680146E86A02681268F9
:10155000904753F0FBFEEB6A93F89C1052F0E2FECA
:1015600094F837305BB186F053FEEB6AD3F8A030C5
:10157000C01AB0F5FA6F24BF002384F8373038BDA5
:101580000C2C002070B50E4605465FF0F5FB5FF0B1
:10159000B7FB10B90124204670BD0A4B93F9D23431
:1015A000012BF7D15FF0E8FB437A002BF2D15FF01B
:1015B000E3FB847A002CEDD1034A314628467DF0C6
:1015C000C9F9E8E7104C0020E07F0C08034BD3F882
:1015D0003C350BB97CF048BF01207047104C00200F
:1015E0002DE9F0432DED028BC47F91B006460F46E6
:1015F0008CB990F90430002B00F00681834B1D68F4
:10160000A86A03685B6B9847044650B9804A39461C
:1016100030467DF09FF9204611B0BDEC028BBDE84D
:10162000F083B3684BB933685B6B3946304611B011
:10163000BDEC028BBDE8F0431847E86AFFF774FF82
:1016400004460028E7D1394630467EF043F8DFF8FB
:10165000F4810546394630467DF0A4F908F2E442AB
:1016600008F59C6392ED007AD3ED007AB4EEE77A48
:101670002840F1EE10FAC5B209D598F9DC34032BF5
:1016800005D0644A394630467DF064F9254608F2B3
:101690008443D3ED007AB0EE088AF4EEC87AF1EE16
:1016A00010FA0BD517EE900AFEF72EFF5A4ACDE935
:1016B0000001394630467DF04DF9002508F591636B
:1016C000D3ED007AF4EEC87AF1EE10FA0BD517EEEE
:1016D000900AFEF719FF514ACDE90001394630461C
:1016E0007DF038F9002508F28C43D3ED007AB8EE8E
:1016F000087AF4EEC77AF1EE10FA0BDD17EE900AD5
:10170000FEF702FF464ACDE90001394630467DF03A
:1017100021F90025B8F97034042B07DC052200926A
:101720003946404A30467DF015F90025D8F8280F93
:101730005FF07EFB80B198F9D2346BB1D8F8283FC6
:10174000B8F9D424B3F90E309A4205DA364A39464C
:1017500030467DF0FFF80025DFF8EC903946304642
:10176000FFF710FF99F8B131002B46D100EA0504CC
:101770002E484FF4806100F0EFFE78B1D8F8283F92
:10178000B3F90C30A3F2E24292B2B2F5FA7F05D976
:10179000274A394630467DF0DDF8002499F84C3868
:1017A00053B124482DF0C6F8054628B9224A3946D7
:1017B00030467DF0CFF82C4600212E2204A80DF1F2
:1017C0000C080391B2F0A4F9D9F89C0142463221E9
:1017D00008F0CEF9054600287FF41DAFD9F89C012A
:1017E00003689B689847154ACDF800800346394640
:1017F00030467DF0AFF82C460DE7114A39463046A9
:101800007DF0A8F80024B3E7012404E70C2C0020A5
:10181000F07F0C0807800C082A800C084A800C080E
:101820006C800C088E800C08AD800C08102C0020F9
:10183000E8800C085484002010810C0848330D08FF
:10184000D3800C08104C0020107C002070B5054699
:101850000E46FFF797FE3146044628467DF0E6FD2A
:101860002040C0B270BD0000F0B591B005460E46F4
:101870007DF04EF90446D8B1102128467CF05AFE7E
:10188000B0B100212E2204A803AF0391B2F040F9B9
:1018900010F080FD32233A46012110F067F804462B
:1018A00030B9054B00973246102128467CF04AFE9D
:1018B000204611B0F0BD00BF24810C0870B505466C
:1018C0000E46B1B990F910408CB116480BF004FBEC
:1018D000DFED157AB0EEC00AB4EEE70AF1EE10FAC9
:1018E00007D4124A012128467DF034F834462046B8
:1018F00070BDAB689BB10E4B1B68D86AFFF714FE36
:10190000044630B15DF044FD0A4A042156F068FEF9
:10191000EDE731462846BDE870407DF0C5BB0124A7
:10192000E5E700BF102C00200000003430810C08D7
:101930000C2C002042810C0838B504467DF084FF51
:101940000546A8B10B4805F0AFFB38B10A490B4872
:1019500010F04CF910B1074800F0D2FD2046FFF717
:10196000EDFD0123064984F8373020467DF082FEE4
:10197000284638BD102C0020308F00205040002019
:1019800064810C08F8B505460E461746C2B12329F6
:1019900001D0012914D81D4807F050FC044668B155
:1019A00000242046F8BD95F91030022B08D05DF0D8
:1019B000EFFC174A062156F013FEF2E7002EF2D094
:1019C0003A46314628467DF0F5FF04460028E7D028
:1019D000104ED6F89C2106F168039A4203D006F611
:1019E00044002DF0DDFBD6F89C0103689B6B984703
:1019F00086F818082846FFF7A1FD4FF0FF33064987
:101A0000C6F8CC3128467DF035FECAE7102C002000
:101A100074810C08107C00208C810C08F8B50546F8
:101A20000E467CF033FE104B93F9A7740446CFB9F1
:101A30000E48BD212DF04AFB38B10D4B32464FF414
:101A4000804128467CF07EFD3C460848BC212DF0B4
:101A50003DFB38B1074B32464FF4804128467CF0BD
:101A600071FD00242046F8BD104C00205484002055
:101A7000A0810C08CC810C0800207047014800F0C0
:101A8000E7BC00BF102C002003685B68184700000B
:101A90000DF0DABB65F056BA5FF0BCB825F03ABB82
:101AA00052F0C2BD07F0FCBC50F07CBE0AF00EBD87
:101AB0000CF03CBC02F040BE4FF010BA14F034BD44
:101AC00062F036BB61F0B4BF0CF094BC46F052BE7D
:101AD0000BF080BA14F086B866F0E8BF5EF0BCBDCB
:101AE0005CF0C4BE06F010BF04F08CBA0AF030B847
:101AF0000AF056BC0CF062BA0CF036BD0BF0A2B87E
:101B00000CF082BB01F02EB900F2845016F0CCBE6E
:101B100007F038BA90F8F432B02202FB030390F8D1
:101B2000382393F8D13012B1012B28BF0123184676
:101B300070470000034808602E21117008221A60C7
:101B4000704700BF30850C0870B5044600F5C840EA
:101B50002C3004F5A255FFF7F1FC0021284610F0C7
:101B60009FFB802120460CF069FF18B127F056F941
:101B700024F0EAFE04F5005303F28C4292ED007A61
:101B8000DFED216A03F28442D2ED007A67EEA67A95
:101B9000D5ED936AFDEEE77A03F63C73F8EEE77A4B
:101BA00004F5BB5167EEA67A1831FDEEE77A05F52C
:101BB000457017EE902A43F8042CD5ED927AF0EE9A
:101BC000E77A67EE877A04F5AF46C3ED007A2AF02C
:101BD000A5F994ED467AD6ED057AE7EE007AC6EDE2
:101BE000057AB0EE670A27F087FE4FF4001186ED04
:101BF000050A20460CF022FF20B12846BDE87040BF
:101C00000EF052BE70BD00BF0000C842FFF79CBF7F
:101C100038B500F5A0450446D5F89C0103689B6BD8
:101C2000984795F8D3373BB930B104F53F501030A1
:101C3000BDE8384082F074B838BD0000FFF7E8BF57
:101C400038B54FF4801104460CF0F8FE054620B973
:101C5000012120460CF0F2FE0546022120460CF040
:101C6000EDFE40B115B9204602F00AFD04F5A25080
:101C70000EF018FD01E0002DF8D14FF48051204600
:101C80000CF0DCFE30B104F5C7402830BDE8384028
:101C900062F074BB38BD0000FFF7D2BF38B54FF417
:101CA000801104460CF0CAFE0121054620460CF0C6
:101CB000C5FE18B115B9204602F0E2FC10212046FD
:101CC0000CF0BCFE60B1204602F04EFD4FF48001E6
:101CD00020460CF0B3FE18B927F0A0F824F030FF2E
:101CE000202120460CF0AAFE28B1204602F0B0FDCB
:101CF000204602F0C9FE4FF4005120460CF09EFE33
:101D000010B1204602F0A8FE802120460CF096FE7D
:101D100028B127F083F8BDE8384024F039BE38BD3B
:101D2000FFF7BCBF00F5A04300F5C540D3F8C011D4
:101D300004307FF037BA0000FFF7F4BF10B5044657
:101D400016F0A2FE90F921308BB190F8403373B1B8
:101D500094F9A8355BB1064B1B68DB6A93F89C309D
:101D60002BB904F28450BDE8104016F0B5BB10BD8D
:101D70000C2C0020FFF7E2BF2DE9F843434B1B6812
:101D8000DB6A93F89C300446002B7CD000F5805829
:101D900098F84937002B76D007F050FA002872D017
:101DA00004F5005504F5055795F88E1238460EF0E7
:101DB0001DF8002867D004F590763046FFF7AAFE9C
:101DC000022860D994F814244FF0B00909FB0242AC
:101DD00092ED837AF1EE007AB4EEE77AF1EE10FA42
:101DE00051D495F88E1238460EF0B0FAB5F9703429
:101DF00007EE903AB8EEE77AB4EEC07AF1EE10FA58
:101E00000CDD94F8143409FB0343F8EE677A93ED84
:101E1000837AF4EEC77AF1EE10FA34DCD8F838366B
:101E2000D5F8382F002BB8BF5B4293422BDC08F269
:101E30003C63D3ED007A9FED166A05F59163D3ED0F
:101E4000006AF8EEE77A66EE866AF4EEE67AF1EE7C
:101E500010FA18DC05F63C7393ED007A27EE067A4B
:101E6000F4EEC77AF1EE10FA0DD494F81414B5F923
:101E70007224B02303FB0161384601F58271BDE88D
:101E8000F8430DF0C9BDBDE8F88300BF0C2C00205D
:101E90000000C842FFF770BF2DE9F04190F81434FC
:101EA0002D4D00EB03132F68D3F8C48100F5907615
:101EB00004463046FFF72EFE474514D0022814D9B9
:101EC00004F5A047C5F8008097F8C431012B15D858
:101ED00017D104F5C045D5F82833E3B9D5F82C332C
:101EE000CBB905230BE0022810D804F5A04393F8E2
:101EF000C4215AB1052283F8C42107E0013B87F8C9
:101F0000C43104F5C3501C3011F0C4FB2046BDE8B9
:101F1000F04109F0E5BF114B1B68D86A03685B68A4
:101F2000984780460028ECD194F81414B02303FBA2
:101F30000161DC31204605F027F9D5F80C330FCBD1
:101F400005F5447605F54C7586E80F0085E80F0029
:101F500087F8C481D5E700BF002C00200C2C00209E
:101F6000FFF79ABF10B500F5A04300F5805493F831
:101F7000D3271AB1002384F849370AE0D3F8203870
:101F8000042B07D100F5C340783082F067F984F85C
:101F9000490710BD0123EEE710B500F5A044234624
:101FA000D4F89C2168339A4208D000F5A1432C3321
:101FB0009A421CBF4FF0FF33C4F88C3704F27C7395
:101FC000074A1A6000F5AF43064A1A60FFF7CAFFD6
:101FD000D4F89C010368BDE810401B69184700BF96
:101FE0000000C8420000C8C2FFF7D6BFF7B500F531
:101FF000A0460446D6F820388B420D463FD00B1F32
:1020000000F5C347594207F1780759413846019115
:1020100082F014F80199384682F010F8042D02D1AC
:1020200018486DF0ADFBD6F82038012B18D1032DE0
:1020300016D104F5C8402C307CF06AFA40B1204635
:1020400007F0FCF820B104F53B500C306DF092FB2A
:102050002046C6F8205803B0BDE8F04002F062BC4C
:10206000072DF5D104F55B50D6F89C276423052194
:1020700092FBF3F32030044A56F0B2FAE8E703B0DB
:10208000F0BD00BFDC5A002070820C0838B500F5A6
:10209000A0450446D5F89C0103689B6B984700282F
:1020A0003FD095F81838E3BBD5F89C212B46683310
:1020B0009A4238D195F8CC372BB901212046BDE89A
:1020C0003840FFF793BFB5F88238152B29D104F5B6
:1020D000C04393F8FC1111F0010120D1D5F820285C
:1020E000072A1CD093F972320BB90421E6E7204687
:1020F0000AF0F2FEDFED0F7AB4EEE70AF1EE10FA25
:10210000F3DB04F5C340783081F0E8FF0028ECD021
:1021100004F55B50084A0621203056F061FA072189
:10212000CCE70321CAE704F5A1432C339A42F8D146
:1021300038BD00BF0000B44294820C0810B5214C99
:10214000D4F89C2104F168039A422DED028BB0EE85
:10215000408A03D00020BDEC028B10BDD4F820389B
:10216000042B25D194F8C53133B11749A1F6DC20F1
:102170002DF08EFA0028EED19FED147AF0EEC87A99
:10218000F4EEC77AF1EE10FA09D49FED110A28EEA9
:10219000008ABDEEC88A18EE103AC4F89C370D4884
:1021A00081F09CFF0028D5D0002384F8CF37D2E7F8
:1021B000B4F88218A4F5A04006F008FA0028D1D19E
:1021C000C8E700BF107C0020308F002000000034E2
:1021D0000000C842088E002010B52DED028B00F5DE
:1021E000A0430446D3F82038042B0BD104F0B6F9F1
:1021F0002046B0EE408A04F07FFA38EE400ABDEC8B
:10220000028B10BD00F5C04494EDD70AF7E700003B
:102210002DE9F0412DED028B00F58C658AB0044666
:10222000284612F03BFC002307A904F5A2500793AF
:10223000089309930FF0C0FE002800F086809DED02
:10224000090ADFED587A04F5A04505F2AC7393ED69
:10225000007A20EE270ADFED547AA7EE270A04F56C
:10226000B2403C3083ED000A66F034FE2046FFF7B2
:102270000DFFD5F89C0103689B6B984795F8D33701
:10228000002B5DD100285BD095F81838002B57D172
:10229000D5F82038042B6FD09FED448A204604F0F7
:1022A0004DFA04F5C04204F5A143C2F8E404D5F8A0
:1022B0009C11994204F500561AD192F8A033BBB98B
:1022C000B6F9043F002B04DC3949D1F8C41EC90615
:1022D0000ED5D2F80C73D2F814137F680A33C91BD9
:1022E00064277B438142ACBF5B181B18C2F8E434FF
:1022F000D5F82038D2F8E414D5F8C8210591204645
:10230000049203930CF016FEB5F9D68107462046D9
:10231000FFF762FFCDE9007806F20C5605F63C05A2
:1023200004F53F50F0EE400ADDE90332D6ED001A25
:1023300095ED001A0599B0EE480A103081F094F935
:102340000AB0BDEC028BBDE8F08104F59070FFF798
:10235000E1FB02280AD994F81434B02202FB0343AB
:1023600093F8402212B193ED8B0A6AE7284612F0E7
:102370002FFAB1EE400A64E704F5C64604F5C647F5
:102380002036303704F5C6413A461031304615F054
:10239000BFFC002880D03946304615F04DFDB0EE28
:1023A000408A7BE7CDCC4C3ECDCC4C3F00000000BA
:1023B000104C0020FFF72CBF00F5A04300F5A14012
:1023C000D3F89C21243082421FBF03F2B473012052
:1023D0001B680B6008BF00207047000010B500F5B7
:1023E000A04200F5A143D2F89C2124339A420C4626
:1023F00012D000F54050D0F8080903681B699847CF
:1024000007EE900A9FED057AF8EEE77A012067EE75
:10241000877AC4ED007A10BD0020FCE70AD7233C80
:1024200010B500F5A04200F5A143D2F89C21243359
:102430009A420C460AD000F54050D0F808090368CB
:102440005B699847012084ED000A10BD0020FCE77D
:1024500030B505460FC985B06C4684E80F0040F2E0
:1024600079322146284604F021FD0C4B03F19002FD
:10247000D3F89C3193420ED19DF8001011F0040165
:1024800002D1204615F040FA0548214604F0CAFD65
:10249000012005B030BD0020FBE700BF107C00200C
:1024A000102C002000F5A040D0F89C0103689B6C24
:1024B0001847000000F5A040D0F89C010368DB6CD1
:1024C0001847000010B500F5A25300F50050D3F8EE
:1024D00008421460D3F804320B60D0F8C43E9B0568
:1024E0000BD400F20C50D0ED006AD2ED007A9FEDD3
:1024F000037AE6EEC77AC2ED007A10BD35FA8E3C5B
:1025000038B50C4D044629460B480FF081FC04F504
:10251000A04305F13C0183F8C50104F5A25004F580
:10252000C0440FF00DFBD4EDD77AF1EE677AC4ED1D
:10253000D77A38BD308F00205040002010B50446B7
:1025400000F590701EF0C6FF2046BDE81040FFF772
:10255000D7BF0000FFF7F2BF00F50050D0F8C43E2F
:10256000194214BF012000207047000010B500F58B
:10257000A0430446D3F89C0103689B6D984701462D
:1025800004F5A1405C30BDE8104084F01DBA0000A5
:10259000FFF7ECBF38B5054B1C6823680A461D6879
:1025A000034B01462046A847002038BD0C2C0020D4
:1025B000102C002070B52DED028B0446036804F545
:1025C00000559B6D9847D5F8C43E1B0617D5B5F945
:1025D0007034B5F97214CA1A0B4402EBD27203EBD1
:1025E000D37352105B1000EE902A00EE103AF8EE12
:1025F000E00AB8EEC00A04F5A2500FF05FF85A4B9B
:10260000B5F8A2241A7004F5C84560F0A7FC2C3573
:1026100060F0F6F800212846FEF7E2FF534E012352
:10262000B0712846F3717BF069FF28B928467DF028
:1026300035F8B0FA80F040093071042120460CF0E2
:10264000FDF920B104F5B2405C3050F05DF9284648
:102650007BF054FFE0B994F8143404F5C04504EB62
:10266000031341F28832D3F8C461D5F8A433F31AC6
:1026700093420DD904F59070FFF74CFA022807D960
:10268000C5F8A463204604F00FFD0023C5F8F83117
:10269000B4F9A4301BB9B4F8A230A4F8A430B4F84B
:1026A000A430DFED338A07EE903AF8EEE77AB7EE22
:1026B000008A88EE270AD4ED2B7AF0EEE77AF4EE62
:1026C000E87AF1EE10FA09D5B4F9A23007EE903AA3
:1026D000F8EEE77A88EE277A84ED2B7AD4ED2B0A90
:1026E00027F00CF820BB51F01FF840F27D124FF498
:1026F000801150F0D1FF4EF0A7FC4EF00FF904F519
:102700004A500C30B0EE408A75F046F804F54F5050
:10271000B0EE480A283075F03FF8B0EE480ABDEC3C
:10272000028B04F554501C30BDE8704075F034B88D
:10273000D4ED2B7A94ED460AF0EEE77AF4EEE87ADF
:10274000F1EE10FA09D5B4F9A23007EE903AF8EE9E
:10275000E77A88EE277A84ED2B7AD4ED2B0A26F0DF
:10276000CDFF0028BFD0C6E75C2300209D9100204C
:1027700000000034FFF71EBF70B500F5C0460446E8
:1027800096F97032002B2ADD06F058FD38BB04F5AF
:10279000C8452C3528467CF081FF00B328467BF0E5
:1027A000ADFEE0B185F034FD04F5A0434FF47A723C
:1027B000D3F8BC37C01A96F97032534398420ED3FF
:1027C00001221C212846FFF7DDF840B104F55B50DB
:1027D000034ABDE870400621203055F001BF70BDAE
:1027E000B4820C0830B52DED028B83B0044601A9EC
:1027F00000F5A2500FF0B2FB002874D004F5AF45ED
:1028000095ED097ADDED017AB4EEE77AF1EE10FA92
:1028100005F1240507D504F5C8402C307BF078FE7F
:1028200008B1019B2B6004F500541820B4F97034F2
:10283000052BB8BF052307EE903A04F2C443D3ED4D
:10284000006AB4F9723407EE103AB8EEC77AF8EEBF
:10285000E77A37EE077AC6EE870AB6EE007AF4EE2C
:10286000470AF1EE10FAC8BFF0EE470A9FED2D7A45
:1028700067EE877A9FED2C7A86EEA71AF0EE007A43
:10288000B4EE671AF1EE10FA48BFB0EE671ADDED4C
:10289000017AF4EEC77AF1EE10FACCBF86EEA70A01
:1028A000B0EE410A27F03CF8B0EE408A1F480EF027
:1028B0003DFB90B91E484021FFF74EFE68B11D4B0D
:1028C000D3F82038012B08D1F7EE007AB4EEE78A6E
:1028D000F1EE10FA58BFB0EE678AB0EE480A03B0C6
:1028E000BDEC028B30BD04F5C8402C307BF010FEEF
:1028F000B7EE008A0028D9D046205FF0D1FDB4EEB3
:10290000C80ADFED0D7AF1EE10FAD8BFB0EE480A32
:1029100087EE800AAFF04CF82F209FED081ADFED0C
:10292000080ABFE73333333F17B7D1385040002090
:10293000102C0020107C0020000034428FC2D53FB4
:102940009A99193FF8B504465EF016FA0368DB68F9
:102950009847054610B900252846F8BD204606F0E0
:10296000FFFA04F5A0460746D6F89C0103689B6B66
:10297000984780B10E4BD3F89C0103685B6B984776
:1029800048B104F5005494F91935002BE3D0032B1A
:10299000E1D03D46E0E796F8B031002BDCD004F5FD
:1029A000005494F9DC54023D18BF0125D4E700BF60
:1029B000107C002073B500F5A0431A46D3F89C1193
:1029C00093ED790A0432914229D100F50052D2F8F0
:1029D000202FB2F90840003C18BF012400F54955EA
:1029E00000F58050D3F83468D0F8382693F83038A2
:1029F0001435B61A5BB10B488DED010A4FF4006136
:102A0000FFF7AAFD9DED010A80F00100C3B2224646
:102A10003146284602B0BDE870407DF0E7BC002496
:102A2000DCE700BF102C002010B5044605F0CCFEFA
:102A300098B104F5A042D2F8343803F58C415031F6
:102A4000C2F8341804F58051D1F838160029BEBFF9
:102A5000A3F58C43503BC2F834382046FFF7AAFF59
:102A6000BDE8104004205FF007BD00002DE9F041F3
:102A70002DED048B00F5005606F20C5393ED008A01
:102A8000DFED358A28EE288A00F5A048BDEEC88A19
:102A9000D8F8383898ED799A18EE102A1A4408EECA
:102AA000102A054646205FF0FBFC06F2B443D3ED46
:102AB000007AD8F89C01B8EEC88A4346A0EE278A6F
:102AC00004339842FDEEC87A17EE904A41D1D6F809
:102AD000243FB3F90860003E18BF012603685B6914
:102AE0009847C0B9D8F89C0103689B6B984790B988
:102AF00005F5C047D7F8DC34022B0CD128460AF084
:102B000039F840B1D7ED947A67EEA87AFDEEE77A0E
:102B100017EE903A1CB205F54E5705F580552C3747
:102B2000D5F83C36E41A98F830383BB10B484FF4EE
:102B30000061FFF711FD80F00100C3B2B0EE490A59
:102B4000BDEC048B324621463846BDE8F0417DF0AD
:102B500089B90026C2E700BF0000C842102C00203F
:102B600010B504460CF02EFB68B100B200EB40003B
:102B7000C0EB001300EE103AB8EEC00ABDE81040FA
:102B800013205FF079BC2046FFF770FFF6E70000E6
:102B900010B50E48FFF7D6FEB0B10D4C04205FF023
:102BA0007FFCD4F8200F5EF057FB04205FF064FC3C
:102BB00013205FF075FCD4F8240F5EF04DFBBDE8E8
:102BC000104013205FF058BC10BD00BF102C002037
:102BD000104C002070B52DED028B0446FFF7B2FEBD
:102BE000002875D004F5A0452A46D5F89C3114324A
:102BF00093426DD0283293426AD02432934267D0F8
:102C00001C3A934264D00832934261D0403A9342D6
:102C10005ED004F50056F6EE008AD6F8200F5EF07E
:102C2000DBF9B4EEE80AF1EE10FA3EDDB0EE087A18
:102C3000FFEE007AE0EE077AB0EE670AD6F8382F9A
:102C4000D5F8343807EE902AB8EEE77A07EE903AD6
:102C5000F8EEE77A5142E7EE007AFDEEE77A17EEFA
:102C6000900AC5F8340826F0FBFED5F89C21C5F87B
:102C7000340804F5A14308339A4222D0D6F8240F31
:102C80005EF0AAF9B4EEE80AF1EE10FAB0EE408A6E
:102C900021DCFEEE007AB4EEE70AF1EE10FA22D55E
:102CA000B0EE087AF7EE007A19E0FEEE007AB4EEA4
:102CB000E70AF1EE10FAC1D5B0EE087AF7EE007A25
:102CC000B8E726484FF48051FFF746FC0028D5D0DE
:102CD000BDEC028B70BDB0EE087AFFEE007AE8EE34
:102CE000077AB0EE678A204605F06EFD08B1B1EEB6
:102CF000488A06F59163D3ED006AD5F838389FED20
:102D0000186A06F63C7696ED007AB5EEC08A07EEB4
:102D1000903AF1EE10FACCBF28EE268A27EE488AC8
:102D2000F8EEE77A66EE866AE8EE067A27EE067A2D
:102D3000FDEEE77AFDEEE66A17EE903ABDEEC77A51
:102D400016EE902A17EE101A17EE900AC5F83838CA
:102D500026F086FEC5F83808BAE700BF102C002020
:102D60000000C84270B5044604F5A04585F050FA4D
:102D7000D5F8AC31C31AB3F5FA6F064603D9D5F8C6
:102D80009C0106F00FFF2E4BC5F8AC61D3F89C01F7
:102D9000026813689847002120460AF09DF8DFED8D
:102DA000297AB0EEC00AB4EEE70AF1EE10FA45D582
:102DB00004F5C043D3EDD77AB1EE047AF0EEE77AAA
:102DC000F4EEC77AF1EE10FA38D504F58C6011F004
:102DD000FFFCF6EE007AB0EEC00AB4EEE70AF1EEC0
:102DE00010FA2BD504F5C25595ED017AF0EE087A6C
:102DF000B4EEE77AF1EE10FA05F104051ED504F5FC
:102E0000495014307DF062FB04F54E502C307DF0BB
:102E1000D9F804F5545004307EF006F895ED007AA8
:102E2000F7EE007AB4EEE77AF1EE10FA06D504F583
:102E300059503830BDE870407DF04CBD70BD00BFCA
:102E4000107C00200000003400F5005090F9673439
:102E5000012BC3BF00F57D6090ED290ADFED047AF8
:102E60009FED040AC8BF20EE270A46205FF004BB8E
:102E70000000C842000000002DE9F0412DED028B5A
:102E800000F5A0480546D8ED798A09F091FC07467F
:102E9000D8F89C0103681B6A984705F55456043618
:102EA00098B14E4CD4F8F837002B0EDD85F0B0F910
:102EB000D4F8F837C01A40F6B733984205D8B4F9B9
:102EC000EC4730467DF0BCFF7AE005F5C04305F5E0
:102ED000005493F8D13443B1B4F9F834002B04DD35
:102EE00005F5405393F91A3513BBD8F89C3105F515
:102EF000A0450435AB426DD00021B0EE680A3046E3
:102F00007DF036FD054604205FF0CAFA2AB207EECE
:102F1000902A04F2AC43F8EEE77A93ED007AE0EE03
:102F2000077AFDEEE77A17EE904A3C4424B2C8E7F0
:102F30000121284609F014FE9FED297AB4F9F834EE
:102F4000C0EE077A08EE103AD8F834389FED250A1B
:102F5000B8EEC88A28EE278A07EE903AF8EEE77AAC
:102F600067EE807A9FED200A27EE800AAEF044FBE0
:102F7000B4F97034DFED1D7A20EE270A07EE903A9F
:102F800008F5046393ED007AF8EEE77A0021B4EED9
:102F9000E77AF1EE10FA58BFF0EE477A80EE277A22
:102FA0003046DFED137AB0EE480AA7EE270AF0EEBE
:102FB000680A7DF039FEBDEEC00A10EE103A1CB270
:102FC000BDEC028B20460B49BDE8F04141F2941262
:102FD00026F056BD391E18BF01218EE7107C002057
:102FE00000A08C450AD7233C35FA8E3C0AE81C41E8
:102FF000E02E65426CEEFFFF38B500F54053054604
:10300000D3F808090368DB689847014605F559506D
:1030100038307DF041FC04B22846FFF793FC70B1D4
:1030200007EE904A05F50055B8EEE70AD5F82C0FE3
:103030005EF012F9BDEEC00A10EE103A1CB2204646
:103040000349BDE8384041F2941226F019BD00BF93
:103050006CEEFFFF38B590F81434B02202FB030386
:1030600093ED837AF7EE007AB4EEE77AF1EE10FA98
:10307000054600F5A0441DD5002109F02DFFDFED28
:10308000427AB0EEC00AB4EEE70AF1EE10FA11D5BA
:10309000D4F82038012B0DD0072B0BD0002384F857
:1030A000903704F29474002323602846BDE838402A
:1030B00009F07EBB85F0ACF8D4F89837C4F89807CF
:1030C000C31AB3F57A7F84BF002384F8903728466B
:1030D00009F06EFBD4F82038012B07EE100A2DD032
:1030E000072B2BD0B8EEC77ADFED286AC7EE267A19
:1030F00005F50052B2F9BC2400EE102AB8EEC00A61
:1031000027EE800ADFED207AB0EEC07AB4EEE77ADF
:10311000F1EE10FA14D4002384F8903794F8903725
:1031200005F559503830DBB97DF09EFABDE83840DE
:10313000174900B241F2941226F0A2BC9FED150A85
:1031400094F89027002AE9D10122934284F890272D
:10315000E4D0072B1EBF04F2947300221A60DDE74F
:1031600004F2947494ED007ADFED0B7A67EEC77A7F
:103170009FED0A7A67EE877AFDEEE77A17EE901AEE
:103180007DF08AFBD2E700BF0000003400A08C4530
:103190006CEEFFFF00000000E02E65420000C84218
:1031A00070B52DED028B00F5C346783682B005462A
:1031B000304680F0C3FE0446E8B905F50053D3F865
:1031C000202FB2F9082082B905F5C042D2EDD77A96
:1031D00003F5976393ED007AF0EEE77AF4EEC77AA1
:1031E000F1EE10FA4CBF01240024304680F0BAFE04
:1031F000002808BF0024304680F0A0FE28BB05F55B
:10320000A043D3F88C37013319D0F4B99FED1A8A53
:103210002846FFF731FE07EE900AB8EEE70A8DED7B
:10322000010AD4B915205FF027F99DED010A1A2093
:1032300002B0BDEC028BBDE870405FF01DB9002C00
:10324000E4D02846FFF706FF02E02846FFF7D4FE49
:1032500007EE900AB8EEE78ADAE71A205FF0AEFBD5
:103260009DED010A08B9B0EE480A15205FF004F997
:10327000B0EE480ADBE700BF0000000010B500F523
:10328000005303F59162D2ED006ADFED137A9FEDF2
:10329000136A03F63C7292ED007A03F57D6366EEE5
:1032A000A76A27EE277AD3ED2A7A67EE867AFDEEB3
:1032B000E66ABDEEC77AFDEEE77A044616EE902A7E
:1032C00017EE101A17EE900A26F0CAFB04F5A04478
:1032D000C4F8380810BD00BF0000C842A00CB345B8
:1032E00010B504460BF0AEFB031E2CDB04F50052B8
:1032F00092F967249A4226DD04F5A041D1F820080E
:10330000022820D004F51354D4ED007ADFED0E6AC4
:10331000D31A66EEE76A07EE102A07EE903AB8EE87
:10332000C77AF8EEE77AD1F8383887EE876A07EE81
:10333000903AF8EEE77AE6EE867AFDEEE77A17EE57
:10334000903AC1F8383810BD0000C842F8B52DEDEC
:10335000028B00F5A0459FED440AD5F834389FED67
:10336000437A07EE903AF8EEE77A044667EE807A01
:103370009FED3F0AF0EEE76AF4EE476AF1EE10FACD
:10338000C8BFF0EE477A27EE800AADF0A5FF26F021
:10339000E9F9B7EE008AC8EE007A05F63C0704F5B5
:1033A0000056C7ED007A96F9983453B3204605F0DD
:1033B0000BFA30BBB6F97034012BB8BF012307EE0E
:1033C000903A05F50462F8EEE77AD2ED006A86EEEF
:1033D000A77AB4EEC87AF1EE10FA15D840F6C41206
:1033E0002449D5F8340826F03BFBC5F83408D6F854
:1033F000382F40F6C4139A42D4BFC6F8382FC6F807
:10340000383FBDEC028BF8BDD7ED007AB4EEE77A19
:10341000F1EE10FAF5D588EE070A20EE000AAEF0BC
:1034200015F9DFED157AD5F8340820EE270ADFED1F
:10343000137A20EE270A40F6C413FDEEC07A17EE89
:10344000904A9C42B8BF1C462246614226F008FBC7
:10345000C5F83408D6F8383FA342D4BFC6F8383F81
:10346000C6F8384FCDE700BF0AD7233C0000AA4278
:1034700035FA8E3C3CF6FFFFE02E65420000C84264
:1034800010B500F540530446D3F8080903681B68DB
:10349000984704F50053D3F8382F514226F0E0FA4C
:1034A00004F5A043C3F834082046BDE81040FFF7F8
:1034B0004DBF000070470000012070470820704792
:1034C0000120704770470000014B93F8A404704737
:1034D000104C0020034B93F9B80C003818BF0120A2
:1034E000704700BF104C0020014B93F9A6047047B1
:1034F000104C002013B5064BD3F89C014B690468AF
:10350000009308310EC9646CA04702B010BD00BF23
:10351000107C0020704700000020704770470000BA
:1035200038B5254DD5F89C0103685B6898470F288E
:1035300034D80F2839D8DFE800F008360808080822
:103540000808083836363636363610241B4B93F8C2
:10355000D92612B193F8D8360BB944F01004184BA1
:10356000D5F89C219A42A3F1080303D09A4218BFD0
:1035700044F01004134991F91915C1B19A4218D0B9
:10358000032902D1104B9A4201D144F040040F4864
:103590007AF0B4FF68B144F080040AE0182814BF40
:1035A00001241824D2E71824D0E70124CEE79A4258
:1035B000EDD144F0010038BD107C0020105C0020EB
:1035C000B47C0020104C0020787C00203C9000202F
:1035D00008B5044805F032FE00280CBF0120022087
:1035E00008BD00BF102C0020F0B52DED028B8BB074
:1035F00005460EF0CFFE4FF48071D0F8047290EDC6
:10360000828AD0F80C6204461448FEF7A5FF30B950
:10361000134BDFED147A93ED007AA7EE678A2D7CC9
:1036200084F0F6FDD4F81823D4F81C33D4F814131E
:103630000892099327221C23CDE9003203900791B9
:1036400003AA1E21284604978DED058A069655F09B
:10365000FBFF0BB0BDEC028BF0BD00BF102C0020B7
:103660001C51002035FA8E3C2DE9F041414E2DEDE4
:10367000068BD6F89C2106F1A4039A428AB073D037
:10368000A6F5005390F81080D3F80879D6F83438AE
:103690009FED399A07EE903AD6F83838B8EEE7AA97
:1036A00007EE903A3B6838469B68F8EEE79A9847F1
:1036B00007EE900AF8EEE77A384667EE897A2AEE46
:1036C00009AAFDEEE77A69EE899A17EE903A1DB2E3
:1036D0003B681B69984707EE900AF8EEE77AA6F573
:1036E000A04067EE897AFDEEE77A17EE903A1CB2B9
:1036F00006F2B473D3ED008ADFED207AF4EEE78AA8
:10370000F1EE10FA58BFF0EE678A02F07FFE3B68D8
:10371000D6ED74AADFED1A7A5B6908EE100A384616
:103720006AEEA7AA9847FCEEE88AB8EEC88A18EEB7
:10373000903AB72228EE098AADF824301A23CDE951
:1037400000323E2103AA40468DED03AACDED049A36
:103750008DED058ACDED06AA8DED070AADF8205056
:10376000ADF8224055F070FF0AB0BDEC068BBDE805
:10377000F08100BF107C00200AD7233C00FF7F4768
:103780000000C84208B502480BF05CF900B208BD61
:10379000102C002037B50D46134840F2EF2203F0FD
:1037A00085FB2C7814F004040AD0696803220F48C2
:1037B00013F0E6FF0C4803B0BDE8304002F042BD14
:1037C00001AA2146284614F0AFF80028F2D0DDED1A
:1037D000017A9FED077A67EE877A2246FDEEE77A57
:1037E00017EE901AE3E700BF102C0020408F002056
:1037F0000000C84210B5054C012384F8DB3657F0B1
:1038000025FC002384F8DB3610BD00BF105C0020CF
:103810005AF0CCBE2DE9F0412DED028B4FF000089F
:1038200082B0CDE900281E4F9FED1E8A0C4615463A
:10383000B0EE480AB1F90220D7F8201F4FF47A738E
:1038400006465BF09BF90123CDE90053B4F9002053
:10385000D7F8241FB0EE480A30464FF47A735BF075
:103860008DF9B4F90420D7F8281F9FED0F0A4346BD
:103870003046CDE900585BF081F9CDE90058B4F944
:103880000620D7F82C1FB0EE480A4FF47A73304662
:103890005BF074F902B0BDEC028BBDE8F08100BFB3
:1038A000104C00200000FA4400007A4438B5C57876
:1038B0000B46352D044628BF3525352200211846F4
:1038C000B0F026F92A4604F10C01BDE83840B0F00A
:1038D000D5B8000010B5074B93F95C2940F24D3480
:1038E00040F24D13002A08BF1C4657F0F7F9204359
:1038F00010BD00BF107C002010B5044614F044FB3E
:10390000204610BD10B50B4C002384F8CF3758F07B
:1039100097F8D4F89C2104F168039A4208D194F8EE
:1039200048382BB904F64400BDE810402BF00ABE1D
:1039300010BD00BF107C002013B5124C94F88E12FD
:1039400004F5A0700CF052FA78B194F88E1204F5D8
:10395000A0700CF0B9FC40B194F88E1204F5A07080
:1039600002B0BDE810400CF0F1BC0EF013FD01A94F
:103970000EF0F4FA18B19DED010A02B010BD9FEDF2
:10398000020AFAE7104C00200000000008B5084BBE
:10399000D3F8A82E002A03DCBDE8084057F016B97A
:1039A00003F6C85054F08CF990ED000A08BD00BF32
:1039B000104C002008B51148D0F89C2100F19C0360
:1039C0009A4214D0B0F9B4319BB990F8593783B901
:1039D00090F8B1316BB990F8093863B9A0F5A040FF
:1039E00005F02CFC00280CBF0320042008BD022099
:1039F000FCE70520FAE70620F8E700BF107C00206E
:103A000010B5214B03F1A402D3F89C31934290B03E
:103A1000044636D000231D48029313F09BFE014656
:103A200018B91A4802AA13F0E1FE247C84F0F0FBD6
:103A3000174BDDED027A9FED177AD3E9CE2305937C
:103A40000023F8EEE77A0793089309930A930B9300
:103A50000C930D930E934FF6F853ADF83C300023C2
:103A6000CDE9030267EE877A96228DF83E30332344
:103A7000CDE90032572103AA2046CDED067A55F054
:103A8000E3FD10B010BD00BF107C0020408F00206F
:103A9000108C00200AD7233C10B557F019FB0446C0
:103AA00078B90948D0F89C2180F8CF4700F1680325
:103AB0009A4206D190F848381BB900F644002BF022
:103AC00041FD204610BD00BF107C00200120704742
:103AD00008B5034BD3F89C0103685B68984708BDA1
:103AE000107C002030B587B005460EF053FC04462C
:103AF0002D7C84F081FBD4F88422D4F8883204929F
:103B0000059300211023CD22CDE9003202900391CC
:103B100002AA42F60C31284655F096FD07B030BD9A
:103B200030B52DED028B89B005460EF033FC00F563
:103B30005A7393E8070002AC84E80700DDED020A3F
:103B40009DED030A2D7CF1EE600AB1EE400AADF066
:103B5000E5FD2046B0EE408A28F0C6FDDFED0B7A89
:103B6000049B079328EE278A0C230122CDE900321B
:103B7000A82105AA28468DED058A8DED060A55F087
:103B800063FD09B0BDEC028B30BD00BFE02E654285
:103B9000282938B5054623D007D824292BD0272932
:103BA00011D01B2908D1012413E0432937D008D8AC
:103BB0004029F8D0422928D02846BDE838405BF09B
:103BC00039B95329EEE7122154F03CFF044610B9ED
:103BD0000024204638BD297C13484DF0D5FDF8E778
:103BE000162154F02FFF04460028F1D0297C0E48FE
:103BF0004DF0A4FEEDE70C2154F024FF044600280C
:103C0000E6D02846FFF78CFFE3E7102154F01AFFB7
:103C100004460028DCD02846FFF764FFD9E7017C82
:103C2000024880F089F9BEE76C850020088E0020EC
:103C3000F0B52DED028B05468DB01646B0EE408AEC
:103C40000C46002930D0007C55F094FC0746287CB7
:103C500056F094FB00F121039F4207D2287C0DB05F
:103C6000BDEC028BBDE8F04054F0DABE6369089306
:103C7000636A2269CDF82530236AA069E16807925A
:103C8000CDF829306222212327680590CDE9003242
:103C90000691287C0397192303AAC2218DED048A7B
:103CA0008DF8246055F0D0FC0DB0BDEC028BF0BD5A
:103CB00070B52D4DD5F89C2105F1A4039A42044618
:103CC00050D0A5F54056B6F84A35DB0708D5A5F51E
:103CD000005393EDE00A012203F55F71FFF7A8FF9F
:103CE000B6F84A35980708D520490B4693ED000AE7
:103CF000043902222046FFF79BFFB6F84A355907E0
:103D000008D51B490B4693ED000A043903222046CF
:103D1000FFF78EFFB6F84A351A0708D515490B4646
:103D200093ED000A043905222046FFF781FFB6F81B
:103D30004A35DB0616D5D5F82038042B12D10EF003
:103D400029FB05460C4880F027F995EDC70ADFED01
:103D50000B7A014620EE270A20460622BDE8704075
:103D6000FFF766BF70BD00BF107C0020EC60002034
:103D700060620020BC620020088E0020E02E6542B8
:103D800070B504460E461DF0E3FB90F8F412B02324
:103D900003FB0101DC31204603F0F6F9054690B142
:103DA0003EB10EF0F7FA90F87C3243F0020380F84F
:103DB0007C3204F5A04304F5A144D3F89C01A04251
:103DC00001D105F03BFE284670BD000073B51646D4
:103DD000019104460EF0DEFA01990DF007FF054649
:103DE00090B13EB10EF0D6FA90F87C3243F0020367
:103DF00080F87C3204F5A04304F5A144D3F89C017B
:103E0000A04201D105F01AFE284602B070BD0000A4
:103E100030B5054685B00C46D1E9040126F036F8E8
:103E200040B1684613F0A6FC6A46214628465AF07F
:103E300015FE08B9022067E0344840F24F32694667
:103E400003F034F8D4ED037AF4EE677AF1EE10FA69
:103E500022D69FED2F7AF0EEE77AF4EEC77AF1EEF4
:103E600010FA54BF012200229DF80030294962F364
:103E7000410368468DF8003013F0E6FD0028D9D1E3
:103E80002548694669F038FD40B951F05FFA0522CE
:103E9000162151F013F8CDE70022E5E7D4ED017AC1
:103EA000FDEEE77A17EE903ADB0706D41B4B03F1E1
:103EB0009002D3F89C31934225D11949134802222C
:103EC0000AF0D2FB9DF8001011F0040102D16846FF
:103ED00013F01AFD0D48694603F0A4F894ED020AA8
:103EE000B4EE400AF1EE10FA0BD6B5EEC00AF1EED0
:103EF00010FA06DD9DF800100948C1F3400106F0F4
:103F000019FE002000E0042005B030BD102C002078
:103F100000000034308F0020204F0020107C002053
:103F2000A07C002010B52DED028BD1ED017A91ED32
:103F3000008AFCEEE77A8AB0CDED037A9DF80C108A
:103F400005AA04465AF074FDC8B1DFED0E7A059B50
:103F5000009368EE277A0022FDEEE77A114617EE0D
:103F6000903A06A813F026FC23682046D3F8CC30FC
:103F700006A9984700200AB0BDEC028B10BD0220B4
:103F8000F9E700BF0000C84237B5124DD5F89C01D3
:103F900003681B6A0C46984740B9D5F89C2105F187
:103FA00068039A4202D0042003B030BDD4ED007AF9
:103FB000D4ED020A94ED010A0748FCEEE77ACDED54
:103FC000017A9DF8041003F093FE0028EBD0002046
:103FD000EAE700BF107C0020102C002008B5D1EDCE
:103FE000007A9FED087A0848F0EEE77AF4EEC77A97
:103FF000F1EE10FA54BF0121002104F0DFFB002094
:1040000008BD00BF00000034102C002010B5D1ED19
:10401000007AFCEEE77A17EE903A9CB2012C02D0BF
:10402000022C06D084B91148214664F0C1FE00205C
:1040300010BD0F4890F850395B0707D55BF0A8F921
:104040000C4A052154F0CCFA0420F1E790F93C39F0
:104050001BB95BF09DF9084AF3E7A0F5A04008F012
:1040600067FA002814BF00200420E1E74C850020F7
:10407000107C0020D0880C08EB880C0838B58B8B9E
:10408000C02B05460C4631D8B12B0BD8112B00F0B4
:104090009680142B00F0968021462846BDE83840D3
:1040A0005BF0BCBFB23B0E2BF6D801A151F823F058
:1040B0001F410108994001089940010899400108F1
:1040C0009940010899400108994001089940010868
:1040D000154101089940010839410108734101085F
:1040E00099400108294101080B410108D42B08D04F
:1040F000B3F5967F49D0D02BCED1BDE83840FFF73D
:1041000085BFBDE83840FFF769BF2146BDE83840AC
:10411000FFF77EBE2146BDE83840FFF703BF2146CA
:10412000BDE83840FFF730BF94ED000A2948FEF79C
:1041300005F8E0B100201BE0274C94F8C531B3B17D
:1041400004F5995104F644002BF0FAFA78B10123F2
:1041500084F87D38022204F16801A4F5A0400AF039
:1041600083FA0028E6D11C4B002283F87D28042026
:1041700038BD194C94F8C531002BF8D004F599518D
:1041800004F644002BF060FAE0E7D1ED007A9FEDF1
:10419000137AF0EEE77AF4EEC77AF1EE10FA16D55C
:1041A000D1ED017AF0EEE77AF4EEC77AF1EE10FA8B
:1041B0000DD50B49022207480AF056FABAE7094919
:1041C0000222F8E708490222A1F5A140F4E7022003
:1041D000CEE700BF102C0020107C0020000000342F
:1041E000787C0020987C0020907C0020F0B5414C29
:1041F000D4F89C2104F190039A428FB00D4677D1F8
:10420000CE78272E28BF27262722002104A8AFF02A
:104210007FFC324605F10C0104A8AFF02FFC059B92
:104220009DF836500093069B0193ED43079B029344
:10423000EDB2089B03938DF8365083F0E9FF15F03B
:10424000810F05F08707064601D1802F12D16846FD
:1042500027F0B2F9DFED287AC4F8F06720EE270ADC
:10426000DFED267A20EE270ABDEEC00A10EE103AE6
:10427000C4F8E43715F0820F01D1802F12D16846BF
:1042800027F0B4F9DFED1C7AC4F8F46720EE270AB2
:10429000DFED1A7A20EE270ABDEEC00A10EE103AC2
:1042A000C4F8E83715F0840F01D1802F12D1684689
:1042B00027F0ACF9DFED107AC4F8F86720EE270A92
:1042C000DFED0E7A20EE270ABDEEC00A10EE103A9E
:1042D000C4F8EC376B060BD5DDED0C7A9FED077A51
:1042E000C4F8006867EE877A04F2FC73C3ED007AC5
:1042F0000FB0F0BD107C0020E02E65420000C842E7
:1043000030B51F4C91B0084602A9FFF7CFFAD4F898
:104310009C2104F190039A422FD19DF83C30072B49
:104320002BD104F58054D4EDCD7ADDED056A9FEDF7
:10433000157AF8EEE77AE6EEC77AFDEEE77AC4ED95
:10434000CD7A5BF025F8D4F80C23D4F834335268D6
:104350009FED0D7A9B1A07EE903AF8EEE77A054644
:1043600067EE877A17EE900AFCF7CEF8074ACDE998
:1043700000010621284654F033F911B030BD00BFCA
:10438000107C00200000C8420AD7233C04890C0896
:1043900010B51D4B03F19002D3F89C3193420446B3
:1043A00096B008460FD108A9FFF780FA9DF854107F
:1043B00003AA20465AF03CFB38B95AF0E9FF134AE9
:1043C000042154F00DF916B010BDBDF8503023F0A3
:1043D00004039BB2002BF6D0DDED0B7A9FED0C7A37
:1043E000039B009367EE877A0022FDEEE77A114681
:1043F00017EE903A04A813F0DDF9236804A9D3F866
:10440000CC3020469847DEE7107C002018890C0845
:104410000000C84230B48D7A4B7A43EA0523CD7A46
:1044200043EA0543562B04460A461BD008D8522BB4
:1044300012D0542B13D02046114630BC5AF0C8BFBE
:1044400003F18073863B23F07F43012BF3D8017C7B
:10445000064830BC4DF03ABB30BCFFF7C7BE30BC9D
:10446000FFF74EBF30BCFFF793BF00BF6C85002045
:1044700000207047C8207047012070470020704717
:104480000020704790F89C308B4286BF283150F84E
:10449000210000207047000090F89C308B4286BFBE
:1044A000283150F821000020704700000320704799
:1044B000014B93F8A2047047104C002070B50446DD
:1044C0004C4808F003FD18B1E36A43F40003E362CB
:1044D000484808F0FBFC88B146205DF0E1FFDFEDC5
:1044E000467AB4EEE70AF1EE10FA07D8236B43F4EC
:1044F00000032363636B43F400036363E36A43F4E1
:10450000F843E3623D4BD3F89C0103685B6898472E
:104510000138172814D8DFE800F03A420C44424230
:104520004242133A3A3A3A3A3A1313131313131313
:10453000133A334A92F8D8368BB392F8D9268AB315
:10454000304B93F8F431012B3DD0022B44D02E4B4D
:104550001D68DDB12D4E284696F8121F47F0B2FFB8
:10456000A0B1E36A43F48073E36296F948351BB166
:10457000236B43F48073236396F8121F284647F099
:10458000D9FF18B1636B43F48073636370BDD4E9E2
:104590000C2342F4E04243F4E043226363630123CB
:1045A00000E00023216B41F480622263626B42F4DD
:1045B00080606063002BC3D041F4406142F44062EC
:1045C00021636263BCE7E36A43F48003E362236B25
:1045D00043F480032363BAE7E36A43F48003E362AE
:1045E000236B43F480032363636B43F480036363AF
:1045F000ADE700BF102C0020000000B4107C0020AC
:10460000105C0020108C002048920020104C0020EC
:1046100013B54FF44470CDE9002113F0ADFC04460E
:1046200028B1DDE900215BF0F5F8024B236020465C
:1046300002B010BD188B0C08002070470020704796
:10464000002070470020704700F514500430704778
:1046500000487047A0B00C0800F5A040D0F89C01BD
:1046600003685B681847000000F5A0431846D3F8BC
:104670009C3168301B1A5842584170479B20704744
:1046800030B500F5A04303F6380353F8042CDFEDF2
:10469000296A07EE902AB8EEE77AD3ED007AF8EEB1
:1046A000E77A85B027EE267A67EEA67A04460023DD
:1046B00001A900F5A25003938DED017ACDED027AA8
:1046C00004F58F550CF016F804F54D523C32692173
:1046D00028464FF007FD04F5535218326A21284648
:1046E0004FF000FD04F5405393F91A2542B903F544
:1046F000A263D3ED007AF5EEC07AF1EE10FA06DD92
:1047000004F559520C326B2128464FF0EBFC04F5AE
:104710005954383420467CF0E1F828B104F13002D5
:104720006D2128464FF0DEFC0DF034FE0DF05AFBF3
:1047300005B030BD0AD7233C10B54FF480110446B4
:104740000AF07CF910B12046FFF79AFF4FF4800180
:1047500020460AF073F928B124F060FBBDE8104050
:1047600022F0EEB910BD000070B590B0002300F546
:10477000A256029302A9002304460DF10702304617
:104780008DF807300DF0F0FB03A930460CF01EFC4D
:1047900008B92D4B03933022002104A8AFF0B8F9DB
:1047A00004F5A045A3238DF8103095238DF8113022
:1047B00083F036FDD5F83438ADF81B3004F580535E
:1047C000CDF81300D3F83826ADF81D20D3F83C36C9
:1047D000D5F83828CDF817104620ADF81F20ADF8D1
:1047E00021305DF05DFE10EE103A1520CDF823303B
:1047F0005DF056FE10EE103ACDF8273004F53F5329
:104800009FED127AD3ED2D7A67EE877A304617EE58
:10481000903ACDF82B30029BCDF82F309DF8073021
:104820008DF83330039B0D930DF0A4FDD5F8D831EE
:104830008DED0E0A302204A904F58F500F934FF02E
:104840008DFD10B070BD00BF2292CA7F0000C8422B
:1048500070B58EB03522044600216846AFF058F995
:10486000A3238DF8003095238DF80130012304F542
:10487000A0468DF8023083F0D3FC04F5405506F2D3
:10488000B473CDF803001B68D5F80809CDF80710FC
:10489000CDF80B3003681B699847ADF80F00D5F8C9
:1048A000080903689B689847ADF811001C4801F09F
:1048B000ADFDADF81300D5F8080903685B699847AA
:1048C00010EE103AD5F80809CDF8153003689B6949
:1048D000984710EE103ACDF81930D6F8D031CDF80F
:1048E0001D3004F5C0433522D3F83813CDF821101C
:1048F000D3F83C13CDF82510D3F83413D3F8E434AF
:10490000CDF82910CDF82D306946D6F8C831CDF84C
:10491000313004F58F504FF021FD0EB070BD00BF57
:10492000102C002030B587B01622044600216846BE
:10493000AFF0EEF8A3238DF8003095238DF8013009
:1049400002238DF8023083F06BFC04F5A045CDF80E
:1049500003002046CDF8071004F070FC05F6240390
:104960008DF80B001B680393124B1B68D86A90F8F4
:104970009C308DF810300368DB69984795F809384A
:104980008DF812308DF8110024F048FA23F03CFA2B
:10499000D5F820388DF813008DF81430162295F8CC
:1049A0000A388DF81530694604F58F504FF0D6FC63
:1049B00007B030BD0C2C002010B58AB02722044669
:1049C00000216846AFF0A4F8A3238DF800309523AA
:1049D0008DF8013009238DF8023083F021FCCDF8E9
:1049E00003000420CDF807105DF05AFD10EE103AD8
:1049F0001320CDF80B305DF053FD10EE103A462039
:104A0000CDF80F305DF04CFD10EE103A1520CDF8CA
:104A100013305DF045FD10EE103A0320CDF817304D
:104A20005DF04EFD10EE103A1A20CDF81B305DF00F
:104A300037FD10EE103ACDF81F3004F5A0432722C1
:104A4000D3F8E431CDF82330694604F58F504FF0A8
:104A500085FC0AB010BD000013B5044600F58F5068
:104A600001904EF0ADFF01984FF044F804F58053EB
:104A7000019893F910330BB14FF0E4F8204602B0DF
:104A8000BDE81040FFF798BF7047000010B500F573
:104A9000A0430446D3F89C0103685B68984704F57B
:104AA0000053014693F8242404F58F504FF016FE6E
:104AB00004F5A2500DF0BAFE04F59070BDE8104068
:104AC0001BF0B0BD9FED020A002245F0AFBE00BF53
:104AD0000AD7233C1C4B70B5044640F8043B5BF0FE
:104AE000CBFF1A4E1A4B6360542560195CF07AF9BB
:104AF00066513035B5F5557FF7D104F555705EF048
:104B0000C3F8144A04F5EE6002F66C3180F0B6F892
:104B100004F67C15FF2384F88C3984F894390E4907
:104B2000284646F019FA0D4B1A6812B10C4883F06A
:104B30003DFB1D60012320460A4984F8C13946F037
:104B40000BFA204670BD00BF703A00207CDB0C08D9
:104B500090DB0C087450002028180E08E89B0020F9
:104B60001CC80C0840CB0C082DE9F04100F512518F
:104B70009AB00D22203104464DF0DCFF0022BE48E1
:104B8000BE4E272145F0CAFD042100205EF056F8F4
:104B9000132101205EF052F8462102205EF04EF80B
:104BA000152103205EF04AF85DF0B4FD46F0DAFB13
:104BB000B34A138843F0040313804FF000080AAF90
:104BC000002110223846AEF0A3FF01238DF83030CB
:104BD0003388ADF8283005A973680B93384645F043
:104BE000A5FCC8B19DF91430002B15DD5CF0C4F8AC
:104BF0009DF81410036801391B68C9B2984758B171
:104C0000051D284645F030FC30B9B368ADF81830C2
:104C100006A9284647F04CF808F10608B8F12A0F13
:104C200006F10C06CCD1974800220DF10B0145F09E
:104C300003FA06AD064620B345F016FC08BB924BBE
:104C40000FCB85E80F0004A9284645F06FFC00282B
:104C500040F03A814FF004088C4B0FCB87E80F00EF
:104C600005A9384645F062FC28B105A845F0FCFBD3
:104C700008B148F0010803A930468DF80C8046F0D1
:104C8000C5FF834B0FCB85E80F0003A9284645F0ED
:104C90004DFC002846D00998002204A945F0CCF923
:104CA000064600283ED045F0DFFB0546002839D1F6
:104CB0009DF80C30013BDBB2032B96BF754A0346CF
:104CC000D35C8DF828303046394646F09FFF724855
:104CD000002205A945F0B0F9064669F04FF878B111
:104CE00069F04AF890F8302090F8281090F8483091
:104CF000114490F840200A44D34214BF01250025F6
:104D000086B130469DF90C8045F0AEFB50B91DB11F
:104D1000B8F1000518BF0125394630468DF82850F6
:104D200046F074FF04F514500022B7EE000A01218A
:104D30003C3045F07BFD04F513500022B7EE000A2D
:104D40000221183045F072FD01230093534A0023DD
:104D500004F505518E2045F0E5FC94F9DCC9BCF161
:104D6000000F1AD14E4E0FCE3D460FC50FCE0FC5C8
:104D70000FCE0FC596E80F0085E80F0062460421AC
:104D8000384645F0CBFC9FED470A474846F08CFC7F
:104D90004648B7EE000A46F087FC012504F50C51A1
:104DA000434A00950023103140F2051045F0BAFC4B
:104DB00004F5145002210C30FFF784FE04F5115065
:104DC00003213430FFF77EFE04F5115003213C30FF
:104DD000FFF778FE04F5145003210830FFF772FE48
:104DE00004F5145002211030FFF76CFE04F5125048
:104DF00002210830FFF766FE04F5125002210C3044
:104E0000FFF760FE04F5125002210430FFF75AFE4E
:104E100004F5C34078307FF025FA264A1368D90795
:104E200009D42549156004F50A5320330B6004F5B5
:104E300097531433CB6004F515501F4902221030EC
:104E4000012545F0C1FC1D4A0095002304F58F5152
:104E5000FD2045F067FC1A4B1A68D20705D4194AA1
:104E60001D6004F59B54083414601648012145F078
:104E7000C7FC1AB0BDE8F0817CC80C08ECCA0C086D
:104E80002C92002040C80C08947D0C08A47D0C08CE
:104E9000B47D0C0878C80C084BC80C08FCF00C0852
:104EA000C47D0C080000000058C80C0867C80C0836
:104EB0006C130E08042C002000220020808A0D08AC
:104EC000082C00201822002004A845F0CDFA002864
:104ED0003FF4C0AE4FF00C08BEE600BF70470000C4
:104EE0000020704700207047002070470020704766
:104EF0000020704770470000002070470020704776
:104F000084B001A880E80E0004B0002070470000C3
:104F10000020704700207047704700001020704745
:104F2000004870478CD70C08004870479CD70C0885
:104F30000020704770470000012070470120704733
:104F400000207047002343608360C36003614361B6
:104F5000002303767047000010B50446FFF7F2FF08
:104F60000023637610BD0000027E531CDBB2042BCD
:104F7000037600EB820288BF002382ED010A88BF1E
:104F80000376704710B50446FFF7EEFFD4ED017AC3
:104F90009FED107A94ED020A637E77EE877A042BF8
:104FA00077EE807A94ED030A94BF0133052377EE00
:104FB000807A94ED040A637677EE807A637E94EDCE
:104FC000050A77EE807A00EE103AB8EEC00A87EE56
:104FD000800A10BD0000000010B5044612F0D4FF96
:104FE000204610BD03F070BE03F07CB803F0D4BAC5
:104FF00003F084B801F0BEBC01F068B801F0F0B96C
:1050000001F030BAFDF7B8BBFDF740B870B5234BDF
:10501000036000F540530446D3F89C08204AC3F8C7
:10502000E02608B112F0B4FF1E4B236004F50053D4
:1050300093F8DC2042B9D3F8D8502DB1284620F09F
:10504000F7FD284612F0A0FF04F59A500C3078F0D6
:10505000B1FC04F5985010305EF01EFF04F6E465D4
:1050600004F68466B54204D0183D284620F036FA8E
:10507000F8E70D4BC4F8C83804F6282052F0FCFAC3
:1050800004F6FC1052F0F8FA04F65C1052F0F4FA50
:1050900004F5136052F0F0FA204670BD98BE0C087B
:1050A00074A50D0880830D0894430D0838B54C4B4A
:1050B000044640F8043B62F065F804F1100010F07B
:1050C000B7FE04F168004BF097FC04F590701AF0FD
:1050D00063FE04F58C600FF051FB04F2845012F073
:1050E00059FF04F6C80021F05BFE04F5666061F02C
:1050F00027FE04F5736047F00BF904F58F504FF06D
:1051000061F804F59750143067F072FD04F598507B
:1051100010305EF0A9FE04F59A500C3078F036FCA1
:1051200004F59B5008304CF029F804F59D501C30D4
:1051300063F006FA04F5805304F59F5200251046EB
:1051400083F8E053274B10301A6041F00BFF2946DB
:1051500004F5A2500BF012FC04F5D550083072F0A3
:1051600021FD04F5FB500C3075F030FC04F50250C5
:10517000043077F065FD04F50350283078F09AF993
:1051800004F505500AF05EFC04F50A50203073F077
:10519000EBF904F50B501449383045F0DDFE04F509
:1051A0000C50103068F0C0F804F50F500C3078F057
:1051B00089FF04F5005304F5105083F824540B4D77
:1051C0003C3079F0A1F82B6813B1094882F0EEFF6A
:1051D0002046084945F0C0FE2C60204638BD00BF7F
:1051E00080830D08549B00209C190E08809200209B
:1051F000A4D70C0888820D082DE9F04F2DED028B05
:1052000004469FB0FFF752FFDE4B236004F51550B4
:105210001030FFF75FFC04F53C5018307AF0EAFBE1
:1052200004F5005504F513532A33C5F8403F04F53F
:105230003D50062385F8443F2C305EF027FA04F5F4
:10524000115704F5A25304F5C34B04F54056C5F8B5
:10525000E03F24370E930BF1780B4FF40063C5F851
:10526000EC3FC5F8E47FC5F8E8BF5A2305F57D6536
:1052700086F86C304FF07E53C5F85C31C24BC5F8F0
:105280006031C24BC5F8643104F54650C04BC5F8D7
:105290006831C5F8CC312C3052F00EFD04F5465083
:1052A00004F53F59383052F007FD4FF00008B94B74
:1052B000C6F8C83109F1100986F8E08109F5FC70DB
:1052C000FFF740FEB44BB549C6F8C83186F8E18116
:1052D000484645F041FEB24BC6F8E8310E9BC6E9A0
:1052E0007B390023C6F81C32C6F8243204F5475532
:1052F000012386F82C32283504F5495012F03AFA89
:10530000A84986F85082284645F026FE04F5495003
:10531000394614307AF024FF04F54E5039462C30CB
:105320007AF082FB04F55450394604307BF0E2FAFF
:105330002C22414606F5D560AEF0EAFB04F5595043
:105340009949383004F55B5845F006FE08F120080D
:10535000964BC6F8E03608F1140081F07FFE04F5A4
:105360005C5A04F55D530AF1180A3C3350460F931A
:1053700057F044FB0F9B0AF1140A5345F6D107235B
:10538000C6F8A0380023A6F8A4384FF4CB7012F06A
:10539000F9FDC6F89C0804F56250283081F05EFEE5
:1053A00004F563502C3081F059FE814B1A680AB91C
:1053B000C3F800807F4BC6F8E03604F564504FF424
:1053C0008051C6F808590C3010F034FE04F56650D0
:1053D0000C3043F08DF904F567500C3046F01EFD9B
:1053E00004F5675020306AF05BFC04F59F407C3088
:1053F00004F006FB04F580436F4AC3F8FC2F04F564
:10540000A04004F5A045043004F0FAFA6B4B6B6041
:1054100028460C3004F0F4FA694BEB60284614304F
:1054200004F0EEFA674B6B61B7EE008A0023284662
:105430006B632B63EB6285ED0A8A3C3004F0E0FA83
:10544000614BEB632846443004F0DAFA5F4B6B643F
:1054500028464C3004F0D4FA5D4BEB6428466030AB
:1054600004F0CEFA5B4B2B662846683004F0C8FA8D
:10547000594BAB6604F5A14004F0C2FA574BC5F88E
:10548000803004F5A140083004F0BAFA544BC5F856
:10549000883004F5A140103004F5A14804F0B0FABA
:1054A00008F11C084F4BC5F89030404604F0A8FAAC
:1054B0004D4BC5F89C3004F5A140243004F0A0FA0F
:1054C0004A4BC5F8A43004F5A1402C3006F072F820
:1054D00004F5A140543004F093FA454BC5F8D4309C
:1054E000444BC5F8DC3004F5A1404FF4C0534249A9
:1054F000A5F830315C3045F02FFDFE2385F8A8314A
:10550000052385F8C4313D4B11934FF0FF3A3C4BD6
:10551000C5F8CCA104F5A3404FF40071C5E9678834
:1055200085ED798A224600936830344B10940FF051
:105530005DFF05F29C73154AC5F88CA7DA6000235D
:10554000C5F8E437C5F8E837C5F8EC37C5F8F037E3
:10555000C5F8F437C5F8F8370323C5F8203805F641
:105560003C0383ED008A274BC5F86438264BC5F809
:105570006C3804F5B140254BC5F87438C5F860485F
:1055800046E000BF98BE0C08000080BF0000B44297
:105590000000B4C210D80C0820D80C0844550E08DE
:1055A000B8520E0860520E08FC4C0E0874A50D0887
:1055B000C4950020F48B0C08F0E10C08F4E50C080D
:1055C00014E90C0838E00C0800E30C0888E30C0828
:1055D00068E20C0870E10C08ECE00C0878E50C08B7
:1055E00080E40C0808E40C0858D80C0800E50C0806
:1055F00090E80C0848D80C08D45F0E08E54F010865
:10560000C8880C08E94F0108ED4F0108F14F010867
:10561000C5F86848C5F87048083012F0ABF804F5D2
:10562000B140243012F0A6F804F5B140403012F039
:10563000A1F804F5B048794BC5F8D43808F1DC007E
:10564000A5F8D8A812F096F808F14408744B7549EB
:10565000C5F838A94046C3F8008045F07DFC4FF6F8
:10566000FF73A5F8803804F5B2406F4B6F49A5F879
:105670009CA83C30186045F06FFC04F5B2405C30EB
:105680004CF04CFE6A4BD6F808291294CDE913343D
:10569000684BCDE91534684BCDE91734674BCDE93C
:1056A0001934674BCDE91B34664B1D931EA911E9D4
:1056B00003000CAB83E80300DDE91A010AAB83E8C1
:1056C0000300DDE9180108AB83E80300DDE91601FA
:1056D00006AB83E80300DDE9140104AB83E80300B3
:1056E000DDE9120102AB83E8030004F5C046414640
:1056F000CDE900274B460E9A584604F5C5487EF082
:10570000B9FB08F10408504BC6F8843208F13C009C
:1057100012F030F84D49404645F01EFC4C4B1F68D6
:1057200017B14C4882F042FDC3F800804A4BC6F8DE
:1057300084320E9B86F8887203F51B7304F5C6400D
:10574000C6F80C3386F88D7286F8B172103012F0FC
:1057500011F804F5C640203012F00CF804F5C640EC
:10576000303012F007F81C22394606F55070AEF0C2
:10577000CFF904F5C84804F5C74008F12C082830D3
:105780005EF0C0FC404678F079FE344B3449C6F8F0
:105790002C34404645F0E0FB324A3349116004F5B1
:1057A000C84364334FF0140CB8B20CFB001201373D
:1057B000127C002AF8D12D4A10802D4A17680FB1AB
:1057C0002C48AFE704F5C8406830136078F040FE1D
:1057D000294BC6F86834294BC6F87834642386F818
:1057E0007C34274BC6F8B03404F5C840254BC6F8C6
:1057F000B4342549783045F0AFFB244BC6F87834F3
:1058000020460123C6F8D87486F8E07485F8CC37B2
:105810001FB0BDEC028BBDE8F08F00BF0000FFFFA2
:1058200070910020E0510D085C9B00202CB90D0800
:10583000F54F0108F94F0108FD4F0108015001081B
:105840000550010809500108F8D70C08DC500E0873
:105850006CA30020B8D70C08B4DB0C0828820C0815
:1058600000820C083C92002000CD0C083A920020E7
:10587000F8910020D4D70C0868820C0830D80C08A6
:1058800050ED0C08A8ED0C08A8AC0D0828EF0C088A
:1058900010B581F0C3FF064C064B18602046FFF799
:1058A000ABFC2046044A0549BDE81040ABF0EEBB16
:1058B000102C00200C2C0020C8F300200D500108F3
:1058C0000069C0F3401070470F299DBF302303FBD0
:1058D0000100503000207047014B93F9E9047047F4
:1058E000104C0020014BD3F82C0F7047104C0020B7
:1058F00008B503689B68984730B9044B93F8B60124
:10590000B0FA80F0400908BD0020FCE7107C0020C0
:1059100008B5044807F068F810B9034B93F8B001D4
:1059200008BD00BF102C0020107C0020022A10B5FA
:105930000C4605D1BDE810400948352208F06CBF7F
:10594000084BD3F89C0103685B689847A04205D1D7
:105950005BF012FABDE810405BF098B910BD00BFD3
:10596000102C0020107C0020012910B50C4614D00A
:10597000022907D0D1B90E4BC3F8D81459F008FD4D
:105980000C4A05E00A4BC3F8D81459F001FD0A4A45
:10599000BDE81040062152F023BE59F0F9FC074A39
:1059A000062152F01DFE024BC3F8D84410BD00BFC3
:1059B000108C002073D90C0848D90C085CD90C084D
:1059C000012903D0022914BF00210221014BC3F891
:1059D000AC1E7047104C0020012902D0022900D0D3
:1059E00011B9024BC3F8DC14704700BF108C0020C3
:1059F000622910B400F3888047291ADC402900F09E
:105A0000978008DC162951DC032904DD504B012462
:105A10008C40234053B95DF8044B5CF023B8A1F1EE
:105A200096040123A3404B4C2342F4D05DF8044B71
:105A30007047A1F148031A2BEDD801A454F823F0C4
:105A40002D5A0108175A0108175A0108175A010858
:105A5000175A01082D5A0108175A0108175A010848
:105A6000175A0108175A0108175A0108175A01084E
:105A7000175A0108175A0108275B0108275B01081C
:105A8000275B01082D5A0108175A0108275B0108F6
:105A90002D5A0108175A0108175A01082D5A0108F2
:105AA0002D5A0108175A01082D5A0108A1F12703A0
:105AB000112BB0D8112BAED801A454F823F000BF9D
:105AC0002D5A0108175A0108175A0108175A0108D8
:105AD0002D5A0108175A0108175A0108175A0108C8
:105AE000175A0108175A0108175A0108175A0108CE
:105AF0002D5A01082D5A0108175A0108175A010892
:105B00002D5A01082D5A0108B02904DC952986DC9C
:105B10006B2980D18AE7B52988D0A1F1D003022B67
:105B20003FF679AF82E75DF8044B00235BF06CBF72
:105B3000094B012283F8D424A3F58043D3F8280F1E
:105B400000283FF473AF5DF8044B64215BF05AB951
:105B500010004100A1008004108C002038B50B46D5
:105B60006B2B0446114600F3AA80472B14DC382B1C
:105B700000F38E80262B5FDC102B00F0CD80162BDF
:105B800000F02281042B00F0DE800A4620461946F0
:105B9000BDE838405BF0C8BCA3F14802232AF4D822
:105BA00001A050F822F000BF215D01088B5B0108C5
:105BB0008B5B01088B5B01088B5B01084B5D010867
:105BC0008B5B01088B5B01088B5B01088B5B010819
:105BD0008B5B01088B5B01088B5B01088B5B010809
:105BE0005F5D01089F5D0108575D0108C15D010807
:105BF0008B5B0108A75D0108515D01088B5B010803
:105C00008B5B0108075D0108D55D01088B5B01080E
:105C10002F5D01088B5B01088B5B01088B5B010822
:105C20008B5B01088B5B01088B5B01088B5B0108B8
:105C30008B5B0108FB5D0108A3F12702112AA4D8A0
:105C400001A050F822F000BF075D01088B5B01083E
:105C50008B5B01088B5B01080B5D01088B5B010806
:105C60008B5B01088B5B01088B5B01088B5B010878
:105C70008B5B01088B5B0108415D0108295D010810
:105C80008B5B01088B5B01083B5D0108355D0108FA
:105C9000402B7FF47AAF931E5942684C594184F8E7
:105CA000D31459F075FB664A94F8D314654B002958
:105CB00008BF1346644A062152F092FC23E09D2B54
:105CC00000F08F800BDC962B00F089809B2B7FF4FB
:105CD0005CAF022A17D15D4806F094FD13E0B52BA6
:105CE00000F09B800ADCAD2B7FF44FAF022A0AD173
:105CF0009FED570A5548FCF721FA04E0A3F1D002C2
:105D0000022A3FF642AF012454E08A1E514B514211
:105D1000514183F8A911F6E70A21FFF707FEF2E7E0
:105D20000A4601212046F8E70A460421FAE70A4616
:105D30000321F7E70A460C21F4E70A460F21F1E7B1
:105D40000A460021EEE70B21E7E70A460D21E9E7C5
:105D50000A460521E6E72046FFF732FED3E7374C37
:105D6000D1B102290DD1012384F8D034A4F5805398
:105D7000D3F89C0103685B6A984710B1334800F080
:105D800087FD59F005FB344A94F8D014334B0029B1
:105D900008BF1346324A8EE784F8D014E6E720465F
:105DA000FFF7E2FDAFE7012431B1022902D12D4B0B
:105DB00083F88C42204638BD2A4B83F88C12F9E7D1
:105DC0002046FFF709FE9EE7022A9CD11F4806F0F5
:105DD000AFFB98E75AF0D0FF5AF058FF93E707213E
:105DE0009BE701242AB1022AE4D1144B83F8D24460
:105DF000E0E7124B83F8D224DCE7022918D1154DD5
:105E0000D5F89C010368DB6B9847044648B1012133
:105E1000A5F5A04002F0D2FCCCE7134880F0B0FA20
:105E200071E759F0B5FA114A042152F0D9FB6AE73B
:105E30000648002102F0C2FC65E700BF108C00207C
:105E400088D90C082BC10C0890D90C08102C002004
:105E500000000000107C002087AC0C0860E60C08F5
:105E6000A0D90C08104C0020EC7C0020B3D90C0801
:105E700010B5084CD4F89C0103689B6B984730B967
:105E8000D4F89C01A434001B18BF012010BD0220CF
:105E9000FCE700BF107C002008B5022103205CF065
:105EA00017FE022108465CF013FE012104205CF07D
:105EB0000FFE022115205CF00BFE132002215CF086
:105EC00007FE124807F002F8A8B1002146205CF056
:105ED000FFFD002149205CF0FBFD00214A205CF021
:105EE000F7FD002101205CF0F3FD0021BDE8084032
:105EF00008465CF0EDBD012146205CF0E9FD012182
:105F000049205CF0E5FD0121E8E700BF102C0020EE
:105F100002490348052208F0A7BB00BF787C002097
:105F2000102C002038B5304B01241C7090F90A3039
:105F30002B2B0CD12D487EF093F92D4808F018F941
:105F4000BDE838402B4801220921FBF71BBD284D35
:105F50009FED290AD5ED460A642103205CF082FBFF
:105F6000D5ED460A9FED240A642102205CF07AFBFD
:105F70009FED220A03205CF07FFA9FED200A0220A9
:105F80005CF07AFA9FED1E0A04205CF075FA9FED32
:105F90001C0A15205CF070FA13209FED190A5CF0C2
:105FA0006BFA284606F092FFA0B1002146205CF073
:105FB000BDFD002149205CF0B9FD00214A205CF0C4
:105FC000B5FD002101205CF0B1FD002108465CF028
:105FD000ADFDB2E7214646205CF0A8FD21464920F0
:105FE0005CF0A4FD2146E9E724960020088E0020FD
:105FF000102C00203C900020000000000000C8424F
:1060000000A08C4500F5A040D0F89C0103681B6CF3
:106010001847000000F5145393ED027A00F5C040D4
:10602000B5EEC07AF1EE10FA03F108035DBFD0F8C7
:106030000C33DFED086AD3ED017AD0F824035FBF9B
:10604000F8EEE77AE7EE267AFDEEE77A17EE900AA9
:10605000704700BF0000C84200F5005090F84805A6
:1060600028B141F00101084214BF0120002070470F
:1060700013B50346FFF7F0FF58B103F5005191F84F
:10608000480FC00705D501F6647191ED000A02B012
:1060900010BD03F5C04412B994EDD70AF7E794F8A0
:1060A000F421022AF8D103F5B240012201A95C30A3
:1060B0004CF0BAFA0028EFD09DED010AE7E70000A6
:1060C00000F5C04393F84823FFF7D2BF10B54B68E3
:1060D000516800F5C0448B42D8BF0A46D4F840034B
:1060E000CCBF1A46194623F0BBFCC4F8400310BDD0
:1060F00010B504464E4867F073FA10F0080217BF57
:106100004C4BDFED4D7A93EDC77AD3EDC97A1FBFC3
:1061100077EE877A9FED497A012267EE877A10F051
:10612000010317BF434B9FED447AD3EDC96A93ED4A
:10613000C67A1CBF37EE667ADFED406A04F514516B
:1061400018BF27EE267AD1ED046AF5EEC06A18BFB3
:106150000123F1EE10FA34DD394A9FED386AD2EDB1
:10616000006A66EE866A0122F4EE676AF1EE10FAC2
:1061700058BFF0EE667A04F5C04090F8481329B392
:1061800073B1D0EDD36AF8EEE66AF4EEC76AF1EEC9
:1061900010FA58BFF0EE476AFDEEE66AC0EDD36A2A
:1061A0009AB190EDD37AB8EEC77AB4EEE77AF1EE11
:1061B00010FAD8BFB0EE677ABDEEC77A80EDD37A19
:1061C00003E0002AD7D1002BD5D110BDB3B1D0F850
:1061D0000C33D3ED016AF8EEE66A76EE876A90ED4D
:1061E000D07AB8EEC77AF4EEC76AF1EE10FAD8BFEB
:1061F000B0EE667ABDEEC77A80EDD07A002AE4D0A0
:10620000D0F80C3393ED017AB8EEC77A77EE277A9F
:1062100090EDD07AB8EEC77AF4EEC77AF1EE10FAC4
:1062200058BFB0EE677ABDEEC77A80EDD07ACCE782
:10623000204F0020104C0020000000000000C84249
:106240002051002000F5C0400023C0F844337047BF
:1062500073B51646044600236A463046009311F093
:1062600077FB48B1DDED007A9FED277A67EE877AFC
:10627000FDEEE77A17EE900A04F5C045C5F8440331
:1062800033785B0718D595F84833ABB104F5B240C5
:10629000012201A95C304CF0C7F968B1D5EDD37A81
:1062A000DDED016A9FED187AF8EEE77AE6EEC77A3F
:1062B000FDEEE77AC5EDD17A04F5A043D3F8203896
:1062C000042B1FD004F50054B4F94225002A16DD32
:1062D000D5F844339FED0D7A83EAE371A1EBE371C6
:1062E00007EE901AF8EEE77A67EE877A07EE102A43
:1062F000B8EEC77AF4EEC77AF1EE10FA02D50023B1
:10630000C5F8443302B070BD0000C8420AD7233C30
:1063100037B50B785A0704460D461DD500F5B24037
:10632000012201A95C304CF07FF9A8B1D5ED017ACA
:106330002B78DFED1B6AF8EEE77ADB0767EEA67ACB
:1063400019D59DED017AB4EEE77AF1EE10FACCBFE3
:106350000120002003B030BD2B78D5ED017A13F079
:10636000010FF8EEE77A04F5C0440FD194EDC97A35
:10637000B8EEC77AE7E704F5C044D4F80C3393EDE0
:10638000017AB8EEC77AE7EE667ADAE7D4F80C332A
:1063900093ED017AB8EEC77A77EE877AE6E700BF29
:1063A0000AD7233C00F50053B3F9F23400EE103A5B
:1063B00000F5A0431A46D3F89C1168329142B8EE1A
:1063C000C00A0CD1D3F82028042A02D093F8CD3784
:1063D0002BB100F5C040D0ED7E7A30EE270A704731
:1063E00010B5044604F5C044FFF7DCFFD4EDC97ACC
:1063F0009FED057AF8EEE77AE0EE477AFDEEE77A70
:1064000017EE900A10BD00BF0000C84237B500F576
:10641000C045044695F84833DBB100F5B24001228F
:1064200001A95C304CF000F998B1D5EDD37AD5EDE7
:10643000D46A9FED0B7AF8EEE77AE6EE877ADDED27
:10644000016AE6EEC77AFDEEE77A17EE900A03B02E
:1064500030BD2046FFF7C4FFD5F84033181AF6E7E1
:106460000000C84210B5044604F5C044FFF79AFF87
:10647000D4EDD77A37EEC00ADFED047A20EE270A92
:10648000FDEEC07A17EE900A10BD00BF0000C842B2
:106490002DE9F04100F5C64700F5C64520373035F7
:1064A00004462946384611F0C7FC04F5A04804F517
:1064B000C64608F2B47310362A46314683ED000A08
:1064C000384611F0EFFB08F5F763DFED220A83EDA4
:1064D000000AB7EE001A762023F022FA04F53F53A3
:1064E00083ED750A2046FBF7D1FDD8F89C010368BF
:1064F0005B6898470B280DD008D80A2811D004F5FE
:10650000C0440023C4F84433BDE8F0810E38C0B263
:106510000128F4D829462046FFF7FAFE0028EED0DD
:1065200011E029462046FFF7F3FE30B90A484FF440
:106530008041FCF711F80028E1D12046FFF792FFD7
:10654000B0F5FA6FE6DD2A4631462046BDE8F04157
:10655000FFF77EBE00000000102C002010B52DEDCE
:10656000028B00F5C043D3EDCD7A93F83033DFEDE5
:106570001D8AB8EEE78ADA0728EE288A82B0044638
:1065800009D400F5805202F5D662D2ED007AF8EE19
:10659000E77AA7EEE88A5B070FD504F5B24001223F
:1065A00001A95C304CF040F838B19DED010A30EEA5
:1065B000480A02B0BDEC028B10BD204604F58054A1
:1065C000FFF70EFF04F5D66393ED000A07EE900A7D
:1065D000B8EEC00AF8EEE77A28EEC00AA7EEA80ADD
:1065E000E5E700BF0AD7233C70B52DED028B00F51F
:1065F000A0463346D6F89C2144339A4204464DD1F6
:1066000000F58053D3F8405600F50053B3F94035F8
:10661000002B66DD04F5C25292ED017AF7EE007AA6
:10662000B4EEE77AF1EE10FA5BD404F53F52D2ED06
:106630000E7AF6EE006A67EEA67A87EE871AB5EE56
:10664000C01AF1EE10FA4CD907EE905A9FED278A46
:10665000B8EEE70A07EE903A04F5B24004F5C044FC
:10666000F8EEE70A20EE080A5C304CF0E9F8D4F8BE
:1066700044339FED1F1ADFED1F0A002BBCBF07EE4E
:10668000903AF8EEE77A4FF42970B8BFA7EE880A7F
:10669000BDEC028BBDE8704023F042B905F0E0FD8F
:1066A000F8B904F5405306F2B476D3F80809036844
:1066B0001B69984704F50053DFED0E0AB3F9403526
:1066C00096ED000A01EE103A0546B8EEC11A40F206
:1066D0007F2023F025F9BDEEC00A10EE103A1BB260
:1066E00096E7BDEC028B9FED030A70BD0AD7233CF1
:1066F00000007A440000000010B5044681F088FDD7
:1067000004F50053D3F85C2F801A41F2883290428E
:106710000FD802212046FFF79FFC50B104F5A0449A
:10672000D4F82028042A04D103F5756393ED000AF8
:1067300010BD9FED010AFBE70000000030B52DED14
:10674000028B00F5C045DFED278A95F8483383B00A
:1067500004465BB3D5EDD37A9FED230AF8EEE77AD2
:1067600000F5B24027EE800A012201A95C304BF00F
:1067700093FFD8B12046FFF737FFDDED017A85EDB5
:10678000D40A37EE800A20468DED010AFFF7B4FFE8
:10679000DDED017A30EE270A20EE280ABDEEC00AB0
:1067A00010EE100A03B0BDEC028B30BDD5F80C23FF
:1067B000D5F8403352689B1A08EE103A2046FFF78E
:1067C000F1FDB8EEC88A2046A0EE288AFFF794FFB4
:1067D000BDEEC88AB8EEC88AA0EE288ABDEEC80A07
:1067E000DEE700BF0000C8420AD7233C10B500F521
:1067F000A0430446D3F89C0103685B6A984718B12C
:1068000004F5C04494F8D00410BD000038B500F57C
:10681000C0440D46D4F840330B44C4F8403394F8D8
:1068200048333BB1FFF7E2FF20B9D4F84C132944B9
:10683000C4F84C1338BD000030B500F50050D0F856
:106840003C25D3070FD4094B08201D785C688D4286
:1068500004D1224214BF0120002030BD013803F1D1
:106860000803F2D1F9E70120F7E700BF04DC0C08C8
:1068700010B500F5A0430446D3F89C0103685B689B
:10688000984701462046BDE81040FFF7D5BF0000FD
:1068900037B500F5C0440546D4F82433C4F8403376
:1068A0000023C4F84433FFF7E3FFD0B105F5B2404D
:1068B000012201A95C304BF0B7FE90B12846FFF7EA
:1068C00095FF70B9DDED017A9FED087A67EE877A62
:1068D0000123FDEEE77A84F84833C4EDD37A03B0A0
:1068E00030BD002384F84833F9E700BF0000C842F8
:1068F00038B504460D46FFF7BBFF30B103212846EB
:1069000011F002F880F00103D8B204F5C04484F815
:10691000490338BD73B500F5C0444A68C4F8402344
:106920000B780D46D90741BFD4F80C335B689B1830
:10693000C4F8403394F84933064623B100F5C64104
:106940003031FFF7D5FF2B785B070FD506F5B24046
:10695000012201A95C304BF067FE38B1012384F8B5
:1069600048336B68C4F84C3302B070BD002384F820
:106970004833F9E7F0B52DED028B044683B004F5FA
:10698000C0450E468DED010AFFF7C4FFDFED350A65
:106990009DED010A40F24310B7EE001A22F0C0FF4D
:1069A000D5F844335B4207EE903AF8EEE77A04F507
:1069B000155767EE807A2046FDEEE77AB0EE408A02
:1069C00017EE901AFFF722FFD7ED017AF5EEC07AA5
:1069D000F1EE10FA07F104073FDDD5F84433002B40
:1069E0003BDD2046FFF712FD07EE900ADFED1E6A41
:1069F000B8EEE77AD7ED007A67EEA67AB4EEE77ADA
:106A0000F1EE10FA29D531462046FFF783FF04F551
:106A1000C641324620312046FFF71AFCD5F84433F0
:106A20005B4207EE903AF8EEE77A204667EE887A06
:106A3000FDEEE77A17EE901AFFF7E8FEB5EEC08A92
:106A4000F1EE10FA09DDD5EDD17AB8EEE77AC7EEAE
:106A5000087AFDEEE77AC5EDD17A03B0BDEC028B82
:106A6000F0BD00BF000000000000C8C2F0B500F596
:106A7000C04487B094F8303303F00503052B074674
:106A80000BD04CF051FE4FF4AE724FF480114CF02D
:106A900003FE0025284607B0F0BD1E486A460321C4
:106AA00010F042FF0028F4D01B4801AA032110F087
:106AB0003BFF05460028ECD0184BDFED190A93ED9B
:106AC000000A40F26D10B7EE001A22F029FF04F51B
:106AD0004C730FCBB0EE401A02AEDFED111ADDEDB4
:106AE000010A9DED000AB7EE002A86E80F0022F0A9
:106AF00049FEDFED0C7A20EE270A3046FDEEC07A23
:106B0000032217EE901A10F03BFE31463846FFF78D
:106B100001FFBFE7208F0020408F0020C8830020A6
:106B2000000000000000C842F7B50E4602210446EE
:106B3000FFF792FA70B304F5A045D5F82038042B7E
:106B400028D12046FFF794FE20B304F5B2475C3706
:106B500004F5C64101236A46203138464BF04EFC0D
:106B6000C0B104F5C641012301AA303138464BF0CB
:106B700045FC78B19DED017ADDED007A77EEC77ABC
:106B800096ED007A37EE277A05F5FB6586ED007AFB
:106B9000C5ED007A03B0F0BDF0B52DED048B00F526
:106BA000005489B000F5736694F8121F03910546EE
:106BB000304645F07DFC03990746304645F08AFC97
:106BC000042F0399B0EE408A1FD1002305A88DED54
:106BD000050A0693079325F073FA05A905F5BB503E
:106BE00023F07AF9DFED9A7A8DED050AB4EEE71A13
:106BF000F1EE10FACDED060A8DED071A05DB05F56D
:106C0000805393F8BC36DF070CD494F8483F002239
:106C100062F3000384F8602F84F8483F09B0BDECAC
:106C2000048BF0BD94F8483F98075CBF43F0020323
:106C300084F8483F04F6647758BF04F64C7305F5B2
:106C40003D5158BF83ED008A243187ED001A284654
:106C5000FFF76AFF94F8603F092B00F2898004F681
:106C60006873D3ED000A9FED7B9AB0EE480A22F0DC
:106C700045FD00BB04F64C7394F8121FD3ED008A57
:106C8000304645F045FC07EE900A9FED737AF8EE2A
:106C9000E77A78EEC88A67EE877AF0EEE88A67EEE0
:106CA000897AF4EEE78AF1EE10FAC2BF94F8603FF9
:106CB000013384F8603F04F6687394F8121FD3ED33
:106CC000008A304645F024FC07EE900AF8EEE77A99
:106CD0009FED627A67EE897A78EEC88A67EE877AE6
:106CE000F0EEE88AF4EEE78AF1EE10FA02DD002316
:106CF00084F8603F04F6687383ED008A94F8483F97
:106D0000DA078BD5284605F5C046FFF727FC04F6C1
:106D1000647393ED008A96F8483330EE488A002B6E
:106D20004CD005F5B240012205A95C304BF07CFC4B
:106D3000002849D181F06CFAD4F85C2F41F28831F7
:106D4000821A8A42034604F5756204F6547144D9E6
:106D500082ED008A284681ED008A0221FFF77CF946
:106D600018B1D6F80422C6F80022C4F85C3F55E7F3
:106D700094F8483F43F00103590784F8483FB9D4D9
:106D800005F5A042D2F82028042AB3D102212846D2
:106D9000FFF762F90028ADD043F0040384F8483FC0
:106DA0003868F9F7B1FB05F55B562036CDE90001EF
:106DB0002B4A0621304651F013FC9BE72846FFF78B
:106DC00057FD0028ADD1B5E704F6647393ED000AD2
:106DD0009DED058A38EE408AACE79FED200A92EDE2
:106DE000007ADFED207A28EE008AA7EE278A82ED6E
:106DF000008AC4F85C0FD1ED007A38EE678AF3EEB2
:106E00000E7AB0EEC88AB4EEE78AF1EE10FA7FF798
:106E100005AF94F8483F5B070ED504F6647405F59A
:106E20005B562068F9F770FB2036CDE900010E4A69
:106E30000621304651F0D4FB05F53D5024220021B7
:106E4000083009B0BDEC048BBDE8F040ACF060BE8A
:106E5000000000340AD7233CCDCC4C3DCDCC4C3E79
:106E6000C4DB0C08CDCC4C3FE1DB0C0838B52DED74
:106E7000028B0D460446FFF771FB002320462B7062
:106E8000B0EE408AFFF738FC0221204638EE400A77
:106E9000FFF7E2F828B104F5005494F8480F00F029
:106EA0000100BDEC028B287038BD000070B50B7876
:106EB00003F00503042B05460C46164615D105F5CF
:106EC000C0454CF031FCB2B24FF480114CF0E4FB01
:106ED000D5F80C23636852689B1A13F5FA7FC8BF74
:106EE0006360237843F00103237070BDF8B500F5AB
:106EF000805300F5A047D3F8B066D7F8DC57B54209
:106F0000044619D00E4A1268D26A92F89C209AB1AF
:106F100000F5C641751B25223031FFF7C7FF07EE8C
:106F2000905AB8EEE70ADFED077A04F53F5020EEFD
:106F3000270A10307CF026FDC7F8DC67F8BD00BFDB
:106F40000C2C00200AD7233CF8B500F5A04C00F526
:106F5000C0449CF8CFE705460F4604F54476BEF1E1
:106F6000000F53D004F54C730FCB86E80F000123BC
:106F70008CF8D03797E80F0004F54C7686E80F00C0
:106F8000D4F8383305F5C646303693B9D4F83C33D7
:106F90007BB9D4F82833D4F83423C4F83833D4F880
:106FA0002C33C4F83C3322B9D4F82413304610F003
:106FB000E7FB314628222846FFF778FF94F8301384
:106FC00011F0040102D1304610F09EFC05F5C641D7
:106FD00005F5C64032461031203010F099FE38B128
:106FE00004F5447604F5487494E80F0086E80F0031
:106FF000284604F08DFD2846FFF74AFA284605F09A
:10700000F3F82846BDE8F840FEF7FCBF04F54873E6
:107010000FCB86E80F0001238CF8CF378CF8D0E730
:10702000A8E70000F8B500F500530446B3F99A3418
:10703000002B0D4635DB0B7813F0020F14BF4FF019
:10704000FF33012304F5C04606F5447786F8E8329D
:1070500006F548730FCB87E80F0095E80F0006F59B
:107060004C7787E80F0004F5C6415722303120469F
:10707000FFF71CFF2046FFF70BFC2046FFF708FA3E
:10708000204605F0B1F804F5A042002382F8D0377D
:10709000C6F8EC3282F8D5372046BDE8F84004F057
:1070A00037BD4FF0FF33CDE72DE9F043354B1B687B
:1070B00085B00546D86AFAF737FA00285FD105F59A
:1070C000005393F9C03E5A1C52D0002B05F58C6634
:1070D00011DD95F87124242107EE903A01FB02623C
:1070E00092ED0B7AF8EEE77AB0EEC77AB4EEE77A73
:1070F000F1EE10FA3CDC05F5805305F5A25793F844
:10710000BC3613F0010429D0C3F340089B0732D4E6
:1071100095F8141495F858444FF0B00909FB015143
:1071200091F8F1314CBB022B18D9684610F022FBC4
:10713000694638460AF06CFE044678B195F8143476
:1071400009FB03534246D3F80012684610F018FBBF
:107150000BF020F969460AF049FD044630460DF06F
:10716000E1FB38460AF060FC2846FBF7C9F92046E7
:1071700005B0BDE8F0830024F0E74446EEE70020C8
:10718000F6E700BF0C2C002038B50C4B1B680546F9
:10719000D86A0C46FAF7C8F910B10024204638BD69
:1071A0000BF0F8F821460AF021FD04460028F4D03F
:1071B00005F5B040443025F071FDEFE70C2C0020C0
:1071C000F0B500F5A04300F5C046002283F8CF27B4
:1071D00083F8D02706F54873044600EE101A0FCB4B
:1071E00087B006F5447585E80F0002AD04F5C64288
:1071F000B8EEC00A28461749203244F017FF95E838
:107200000F0006F54C7787E80F0004F5C64140F201
:107210005712303120460191FFF748FE0199204670
:10722000FFF766FB01992046FFF774FB04F5005356
:107230002046B3F99A34002BB4BF4FF0FF3301233B
:1072400086F8E832FFF724F9204607B0BDE8F040A1
:1072500004F0CABFDC65002010B50349044644F0C1
:10726000E5FE204610BD00BFDC650020F8B500F546
:10727000C04505F5487304460E460FCB05F5447727
:1072800087E80F0006F108012046FFF75DFEB2888F
:1072900002EB820202EB8202920012B204F5A043DA
:1072A000002AD8BF4FF4C872A3F8CA27D5F80C2318
:1072B000D5F834135068091AC3F89C1791680A313D
:1072C000C5F83813D2680A32C5F83C230022C3F847
:1072D000B02783F8CC2783F8E027C3F8A02703F270
:1072E0009472002111604FF0FF32C3F88C2794F89C
:1072F000711404F58C62242000FB012203F2C47394
:10730000D26A1A60F8BD000070B50E460831044616
:10731000FFF71AFEB38804F5A04543B3642213FBBC
:1073200002F3C5F89C37B5F9CA37002BD8BF4FF424
:107330007A7304F53D50D8BFA5F8CA37242200213E
:107340000830ACF0E5FB04F5C04304F5C34093ED11
:10735000D70A314678307CF083FED5F82038072BE9
:107360000CD120460421BDE87040FAF73FBED5F8A5
:107370009C37002BD7DC40F6B833D2E770BD000055
:107380000B7A00F5C04013F0020F14BF4FF0FF332B
:10739000012380F8E83270477FB501F10803054604
:1073A0000E460FCB6C4684E80F0005F5C641203130
:1073B000204610F049FB21462846FFF7C5FD31461F
:1073C0002846FFF7DDFF04B070BD00007FB501F176
:1073D000080304460E460FCB6D4685E80F0004F502
:1073E000C6412031284610F02FFB29462046FFF7E2
:1073F000ABFD20463146FFF7C3FF337907EE903AE5
:10740000337E9B0748BF9FED0B7AF8EE677A04F551
:10741000C04448BF67EE877A9FED077A67EE877AA8
:107420000123FCEEE77AC4F80033C4EDB87A04B067
:1074300070BD00BF0000803B00A00C477FB501F18C
:10744000080304460E460FCB6D4685E80F0004F591
:10745000C6412031284610F0F7FA29462046FFF7AA
:1074600073FD20463146FFF78BFFB38804F5C04417
:107470004FF47A725343C4F8F8320123C4F800334E
:1074800004B070BD2DE9F34100F5C6450446303522
:1074900000F5C6400E461030294610F095FA04F566
:1074A000A047D0B94FF0FF33C7F88C3706F1080773
:1074B000384610F08FF9032802463CD1F16828467F
:1074C00010F05EF9B28804F5C0432046C3F80023EB
:1074D00002B0BDE8F041FEF7B5BE1AF039F8FAF790
:1074E00019FB012812D94FF0FF33C7F88C371AF077
:1074F0002FF890F8F432DFED150AB02202FB0300FA
:1075000090ED3C0A284610F00DFDCFE704F58058B9
:10751000D8F8400622F0D8F904F5B253C7F88C0722
:10752000D3ED007A9FED0A0ADFED080AF8EEE77A5C
:1075300027EE800AE6E701AA0021384610F056F946
:107540000028BFD001990022B9E700BF00007A44AB
:107550000AD7233C7FB501F1080304460E460FCB42
:107560006D4685E80F0004F5C6412031284610F02D
:107570006BFA29462046FFF7E7FC20463146FFF725
:10758000FFFE04F5C0440023C4F8003304B070BD0E
:1075900037B504460D4680F03BFEE060D5ED027A3B
:1075A000F5EEC07AF1EE10FA15DD9FED127A67EE76
:1075B000877AFCEEE77AC4ED027A57F0E9FEA2681A
:1075C0004FF47A73B2FBF3F30B4A062103B0BDE824
:1075D000304051F005B865F051FE0023009395F955
:1075E0000D2095F90E3095F90C1065F0E3FDA060C3
:1075F000E3E700BF00007A4444DC0C082DE9F043C7
:107600002DED028B85B004460AF0C4FE09F0F2FFAE
:1076100004F5805304F5A04693F838390BB90028D7
:1076200077D0D6F88C37013373D1D6F8B037002B2A
:107630004BD080F0EDFDD6F8B037C01AB0F5FA6F38
:1076400067D394F81424DFED607A9FED608A4FF0E1
:10765000B00808FB024292ED840A20EE270A22F0CD
:107660004BF906F29479D9ED007A30EE670A22F0F0
:1076700043F9DFED577A20EE080A04F55B5720EE58
:10768000270A22F0E1F8FDEEC07A203717EE905A73
:10769000C6F88C57D9ED007A67EE887A17EE900A13
:1076A000F8F732FFCDE9020194F8143408FB0343E4
:1076B000D3F80C02F8F728FF464ACDE900012B4623
:1076C0000621384650F08CFF23E004F59070FAF75D
:1076D00021FA02281DD994F81434B02202FB034386
:1076E00093ED837AF1EE047AB4EEE77AF1EE10FAD4
:1076F0000FDD394B1B68D86A0368DB69984701289E
:1077000003D080F085FDC6F8B007D6F8B037002B5F
:107710008FD104F54053D6F88C17D3F808094A1CCA
:10772000036848D01B6B98472C4807F0B9FD20B17F
:1077300004F5B040443027F033FD2046FEF792FEBA
:10774000D6F89C378342054638DA07EE905A9FED0B
:10775000247AF8EEE77A04F55B5767EE877A2037EC
:1077600017EE900AF8F7D0FE1E4ACDE90001384620
:10777000062150F035FF04F5C0444FF0FF330125DA
:10778000C6F88C3786F8CC5704F548730FCB04F550
:10779000447704F54C7487E80F0084E80F00124822
:1077A00065F0E8FE002386F8CF37284605B0BDEC2B
:1077B000028BBDE8F0835B6B9847B5E7074807F09D
:1077C0004FFD0028C1D1F1E735FA8E3CE02E65422D
:1077D0000000C84254DC0C080C2C0020102C0020A7
:1077E0000AD7233C78DC0C08204F00202DE9F04F0D
:1077F00000F5A0492DED028B4FF0FF3300F5C04A94
:10780000C9F88C370AF54C730F4606460FCBBC8877
:1078100097F8048089B004AD240A85E80F001FD0D2
:1078200006F5C64710372946384610F005FB2946AD
:107830003846B0EE408A10F0CFF9DFED577AB4EE5B
:10784000E78AF1EE10FA0BDBE3B200EE903ADFEDDF
:10785000537AF8EE600A20EE270A284610F062FB01
:1078600006F5405B99F8D027DBF808099FED4C0A34
:10787000036806F5C6479B6A203732B306F5C64152
:107880002A461031984706F50051B1F9CA34002B49
:107890001EDD07EE903A09F2B472F8EEE77A92ED47
:1078A000007AB4EEE77AF1EE10FA11DD06F5C64182
:1078B0002A461031384610F02BFA00BB002420462F
:1078C00009B0BDEC028BBDE8F08F2A463946D9E7F6
:1078D000B8F1000F1DD1002C3DD1B1F9C824DBF85F
:1078E000080900EE102A026809F5F563126AD3ED63
:1078F000000AB8EEC00A9047B0EE408A0DE0002CB6
:10790000DCD10AF548730FCB0AF5447585E80F0002
:10791000D5E707EE908AB8EE678A2946384610F018
:107920008BFAB4EEC08AF1EE10FA17DBB9F88038A2
:1079300003932946384610F07FFABCEEC00A06F5DC
:107940005B50039B174A8DED000A0621203050F052
:1079500047FE0124B3E79FED128ADEE706F5C64134
:107960002A461031384610F0D3F904460028A5D035
:10797000B9F8803803932946384610F05DFABCEE1A
:10798000C00A06F55B50039B074A8DED000A0621ED
:10799000203050F025FE92E700000034E02E6542D2
:1079A0000000000094DC0C08B2DC0C0838B500F5CF
:1079B000005500F5C043B5F9CC140029ACBF012235
:1079C0004FF0FF320029B8BF4942044683F8E8224D
:1079D00089B204F02BFD04F5AF4393ED0D7AB5F9B0
:1079E000C834002BCABF07EE903ADFED0E7AF8EEEE
:1079F000E77AFCEEE77AF8EE677AB4EEE77AF1EE32
:107A000010FA08D804F55B502030074A062150F0E0
:107A1000E7FD012038BD204604F022FC0028F1D10A
:107A2000F8E700BF00000000D0DC0C08F8B500F556
:107A3000C64600F5C6451036303504462946304660
:107A40000FF0C2FF04F5405750B304F5A043D3F83C
:107A50008C174B1C24D0D7F8080903681B6B984778
:107A600004F5C045D5F80033012B47D0D5F80033D5
:107A7000022B06D12046FEF7B3FCD5F834339842EA
:107A800043DD2046FEF7ACFCD5F83433C01A00289D
:107A9000B8BF4042B0F5FA7FCCBF0020012035E0EE
:107AA00004F5C6402946203010F0C6F9DFED187AFB
:107AB000B4EEE70AF1EE10FA16D53046294610F07A
:107AC0008BF89FED147ADFED140AF6EE007AE0EE03
:107AD000077A28469FED110AFDEEE77AF8EEE77A7D
:107AE00027EE800A10F01EFAD7F808099FED0C0A5D
:107AF00003682A469B6A31469847B1E72046FEF75D
:107B00006FFCD5F834339842B0DB0120F8BD00BFDC
:107B100000004843A00CB345000096430AD7233C1D
:107B20000000000073B5374CD1ED026AD4EDC97A7C
:107B30009FED357AF8EEE77A0546D7EE876A0E466E
:107B4000F5EEC06AF1EE10FA08DD57F021FC2F4A7D
:107B5000062150F045FD012002B070BDD1ED037A41
:107B6000F5EEC07AA4F65404F1EE10FA94ED006A32
:107B700012DDF4EEC67AF1EE10FA0DD557F008FCDE
:107B800005462068F8F7C0FC214ACDE9000106212E
:107B9000284650F025FDDEE7DFED1E7A337CB4EE9B
:107BA000E76AF1EE10FA54BFB0EE677AB0EE467AAB
:107BB0000BB90020D0E7B5EEC06AF1EE10FA0CDC8C
:107BC00086EE876A03EB830307EE903AF8EEE77AD6
:107BD000F4EEC67AF1EE10FAEBD52C7C002CE8D14D
:107BE00080F016FB6B69C01A337C4FF47A725343F2
:107BF0009842DED901232B7480F00AFB686120468D
:107C0000AAE700BF108C00200AD7233CE8DC0C0850
:107C1000F9DC0C080AD723BC38B5054677F0E4FE3A
:107C200076F076FC044640B980F0F2FAEB68C01AB0
:107C3000AB68984284BFAC600124204638BD000088
:107C400038B504460D4680F0E3FA04F5C0439FEDD5
:107C5000067AC3F80403D5ED027A67EE877AFDEE63
:107C6000E77AC3EDC07A38BD00007A4410B5044607
:107C700080F0CEFA04F5C043D3F80423801AD3F879
:107C8000002390424FF0000084BFC3F8000301209E
:107C900010BD000000F5C04300F5AF41D3F800234C
:107CA00091ED0D7A22EAE27207EE902AF8EEE77A79
:107CB0000020B4EEE77AF1EE10FA44BFC3F80003F7
:107CC0000120704710B500F5005300F5C040B3F92E
:107CD0009A34002BB4BF4FF0FF33012380F8E83211
:107CE00000F54C7400F548700FC884E80F0010BD13
:107CF00038B504462DED028BF0EE408AB0EE608A76
:107D000009B301295CD0B5EEC08AF1EE10FA67DD47
:107D1000DFED347AB4EEE78AF1EE10FA60D8FCEECB
:107D2000C87A04F55B5017EE903A2F4A06212030AE
:107D300050F056FCFDEEC87A04F5005417EE903A68
:107D400084F867343AE0F8EE000A21F0D7FC40B13D
:107D500004F5A0444FF0FF33C4F8CC31BDEC028BE6
:107D600038BD04F50053B3F9702407EE902AF8EEFD
:107D7000E77AF4EEE87AF1EE10FAC4D8B3F9723487
:107D800007EE903AF8EEE77AF4EEE87AF1EE10FAC0
:107D9000B9DBDFED147A154A68EEA77A04F5A04343
:107DA000FDEEE77A04F55B50C3ED737AFCEEE87AFA
:107DB000062117EE903A203050F012FC0120CDE75A
:107DC000FCEEC07A00F55B5017EE903A084A0621A7
:107DD000203004F5115450F003FCC4ED0F8AEDE798
:107DE0000020BBE70000C8423FDD0C0818DD0C088E
:107DF0002CDD0C08D1F80D3000EE903AD1F80930A6
:107E0000097A00EE103AFFF773BF000070B58B8857
:107E1000012B04460D4611D100F590763046F9F756
:107E200079FE02280AD994F81414B02303FB0161E7
:107E30002046DC31BDE87040FFF7A6B90AF0AAFA87
:107E400005F10801BDE8704009F0D0BEF0B500F5BD
:107E5000A0460027A14B86F8D57789B0044608468E
:107E60000D4683F8497324F02BFD50B3012386F8A7
:107E7000CC3704F54053D3F808090368DB6B984707
:107E800004F5C04386F8D37703A8C3F8EC720FF06B
:107E900071FCB6F880184FF6FF73994208BF394657
:107EA000013104F5B04001AA89B2443026F0FAFC51
:107EB00028B1BDF80600A0F115035842584186F8D4
:107EC000CD076B885D2B00F0028132D81F2B29D89B
:107ED0000F2B01D800202AE0103B0F2BFAD801A26B
:107EE00052F823F0D77F0108ED7F0108F77F0108E2
:107EF0000180010815800108E37F0108C57F0108A2
:107F0000D57E0108D57E0108D57E0108D57E010801
:107F1000D57E0108D57E0108D57E010823800108A1
:107F20000B800108532BD5D1012086F8D30709B067
:107F3000F0BDBD2B18D8BB2B4BD8B22B7BD00CD8A7
:107F4000702B73D0722BC5D1D5ED027AFDEEE77A96
:107F500004F5C044C4EDC07A3BE0B32BBAD1294646
:107F60002046FFF753FF34E0C33B9AB2112AB1D841
:107F7000112BAFD801A252F823F000BF7180010885
:107F8000D57E010871800108D57E0108D57E0108E3
:107F9000D57E010871800108D57E0108D57E0108D3
:107FA000D57E0108AD800108D57E0108D57E010887
:107FB000D57E0108D57E010841800108D57E0108E3
:107FC00061800108002386F8093829462046FFF71A
:107FD0004DF90120ABE705F108012046FEF7B4FF9B
:107FE000F7E729462046FFF78FF9F2E729462046B2
:107FF000FFF7D2F9EDE729462046FFF7E7F9E8E772
:1080000029462046FFF71AFAE3E729462046FFF7FC
:10801000A1FADEE7292204F5A141204606F024FB5F
:10802000D7E729462046FFF72DFAD2E72946204612
:10803000FFF706FECDE729462046FFF7DBFEC8E73F
:10804000AB88012BC5D803F0010386F8CE3704F5C1
:108050005B50AB88224A0621203050F0C1FAB8E7C5
:10806000A988003918BF0121204600F0A7FBB0E71E
:1080700004F5C746EB6804F5C044283694F821148B
:1080800073B92B6963B96B6953B930465CF068F812
:1080900004289ED194F8211430465CF06BF898E7E0
:1080A00005F1080230465CF0A3F992E704F5C043FD
:1080B00004F5C74095ED041AD5ED020A95ED030AC3
:1080C00093F82114002228305CF076F881E704F55B
:1080D000A04029466830FFF75BFA7AE7108C002051
:1080E00050DD0C0800F5A0421346D2F89C216833FD
:1080F0009A4201D1FFF7AABE0120704710B500F5E2
:10810000A0421346D2F89C2168339A4204460DD10E
:10811000082200F5A14106F0A7FA04F55B50044AD5
:10812000BDE810400621203050F05ABA10BD00BF03
:1081300060DD0C0870B58EB009AD044628460E46C9
:108140000FF018FB04F5A0434FF6FF72B3F8803828
:10815000934208BF0023013304F5B04007AA99B247
:10816000443026F09FFBB0B104F5C04416B10023A3
:10817000C4F8E43295E80F0001AE86E80F00D4F8A9
:108180003C33009304F54C7494E80E00034802F06D
:10819000A7FD0EB070BD0120FBE700BF987C00205A
:1081A00070B5054605F5C046002104F03FF9D6F844
:1081B000EC427CB9284604F053F810B9002420465C
:1081C00070BDD6F8E432012BF8DD80F021F8C6F856
:1081D000EC02F4E7D6F8001361B180F019F8D6F894
:1081E000EC32C01AD6F8F8329842E7D90023C6F824
:1081F000003301212846FFF79DFF04460028DDD00B
:1082000005F55B50054A0621203005F5A04550F0E4
:10821000E7F9002385F8D537D1E700BF88DD0C08E2
:1082200038B50A468B88190A137EDB0748BF01EB75
:108230008101044648BF490004F0F8F804F5A04362
:10824000002583F8D557204604F00AF810B9002518
:10825000284638BD04F5C043D3F8001341B1D3E933
:10826000B8128A42F3DD012AF1DDC3F8005301217F
:108270002046FFF75FFF05460028E8D004F55B5075
:10828000024A0621203050F0ABF9E1E7A0DD0C08EE
:1082900038B5054605F5C044898804F0C7F8D4F818
:1082A000003383BBD4F8E432002BB8BF5B42012B10
:1082B00002DC0024204638BD94F8E92294F8EA3222
:1082C00072B9002BF5D005F55B50D4F82423642354
:1082D000062192FBF3F320300C4A50F081F901E0C3
:1082E000002BF0D10121C4F800132846FFF722FF2C
:1082F00004460028DDD005F55B50054A06212030F4
:1083000050F06EF9D6E70021EFE700BFB8DD0C08AA
:10831000D6DD0C082DE9F0474B881F2B8AB00446A8
:108320000A4631D80F2B07D804F55B50984A042130
:10833000203050F055F988E0A3F110010F29F3D84F
:1083400001A050F821F000BF5B84010829850108D5
:1083500035850108438501085D85010869840108A8
:108360004F84010829830108298301082983010812
:108370002983010829830108298301082983010829
:10838000698501084F850108702B00F0FB800CD82F
:10839000532B00F0EF805D2BC6D100F5A040683074
:1083A0000AB0BDE8F047FFF737BCB32B08D8B12BB4
:1083B0004BD8722BB8D10AB0BDE8F047FFF76ABCC2
:1083C000D42B3BD8BB2BAFD9A3F1BC02182AABD816
:1083D00001A151F822F000BF4B8401084B84010831
:1083E00029830108298301082983010829830108B9
:1083F000298301084B840108298301084B84010863
:108400002983010829830108298301084B84010875
:108410002983010829830108298301084B84010865
:108420004B8401084B840108298301082983010832
:108430004B840108298301084B840108DF2B04D0F9
:1084400040F6B83293427FF46FAF01202FE0204610
:108450000AB0BDE8F047FFF7D1B8114620460AB090
:10846000BDE8F047FFF7C2B904F5A04504F5C346DF
:10847000D5F8203804F5C64704F5C64804F5C649C2
:10848000072B06F1780607F1100708F1300809F10B
:1084900020090FD104F5B04418340194D5F89C3765
:1084A000009342464B46394630467BF09DFE0AB06B
:1084B000BDE8F0870DF12701002336488DF82730FD
:1084C000FEF7D4FC05F5FB63D3ED007AD5F8BCA725
:1084D00005F2AC73D3ED000A05F5F76330EE670AD9
:1084E00093ED001A8DED070A04F5C8402C30CDED50
:1084F000060A8DED051A76F001F80546204600F0D3
:108500009DFE9DF827309DED051ADDED060A9DEDD7
:10851000070ACDE90203CDE900A54B46424639469C
:1085200030467BF0B7FDC2E72046918803F07EFF1E
:108530000020BCE7114620460AB0BDE8F047FFF72F
:108540006FBE20460AB0BDE8F047FFF729BE1146CE
:1085500020460AB0BDE8F047FFF79ABE20460AB0B1
:10856000BDE8F047FFF722BA20460AB0BDE8F04761
:10857000FFF75CBA00F5A04068300AB0BDE8F047EC
:10858000FFF7D0BA0AB0BDE8F047FFF76FBB00BFF6
:10859000F0DD0C08102C002070B500F5A042134649
:1085A000D2F89C2168339A4205460E4602D0002438
:1085B000204670BDFFF7AEFE04460028F7D005F553
:1085C0005B503188203054F0FBF9F1E721F0400393
:1085D000152B04D0A1F15E03584258417047012089
:1085E0007047000018294DD8DFE801F00D1115196A
:1085F0001D2125292D4C313538443C3C404C4C4CF8
:108600004C4C4C4C480000F5A1402430704700F51C
:108610009F407C30704700F5A0400430704700F563
:10862000A0400C30704700F5A0401430704700F5B2
:10863000A0403C30704700F5A0404430704700F542
:10864000A0404C30704700F5A0406030704700F506
:10865000A0406830704700F5A140704700F5A14088
:108660000830704700F5A1401030704700F5A14078
:108670001C30704700F5A1402C30704700F5A14038
:10868000543070470020704700290DDB074890F8F0
:10869000442FCBB29A4207D3D0F8403F0122595C15
:1086A000A0F5005006F0B8B8704700BF104C00208D
:1086B0002DE9F34100F5005300F55B5593F8103FA9
:1086C00003F0010603F0020803F004075B07044609
:1086D00005F1200535D01F4A062128464FF080FFBE
:1086E00026B104F54950143077F08CFFB8F1000F33
:1086F00004D004F54E502C3077F000FD27B104F57E
:108700005450043078F0A8FB04F5C044012384F8E9
:10871000D134114A114B1249B8F1000F08BF1A4663
:10872000002F08BF1946CDE900210E4A0621002E70
:1087300018BF134628460C4A4FF052FF02B0BDE85E
:10874000F0810A4A0621284602B0BDE8F0414FF008
:1087500047BF00BF1DDE0C0812DE0C0860BF0D080D
:1087600019DE0C080CDE0C082EDE0C0840DE0C08AE
:1087700010B5044600F54950143077F06FFF04F54A
:108780004E502C3077F0E6FC04F55450043078F06D
:108790009DFB04F5C04393F8D1245AB1002283F81D
:1087A000D12404F55B50044ABDE810400621203076
:1087B0004FF016BF10BD00BF60DE0C0809B1FFF717
:1087C00077BFFFF7D5BF000000F5A0420848D2F8F8
:1087D0009C11814209D092F8A90138B91346683337
:1087E000994203D192F8CE0770470020704700BF2E
:1087F000B47C002010B504467FF00AFD054BD3F889
:10880000BC31C01A642804D82046BDE8104058F096
:108810002DBA10BD107C002010B500F53C54D4EDED
:10882000007AF5EEC07AF1EE10FA8AB04FF000034C
:1088300044D907930893099306AB019307AB0093C0
:1088400003AA05AB04A900F5A25009F055FA30B30C
:10885000DDED080A9DED070AA8F0C4FDDDED090A6B
:10886000A8F0C0FDD4ED007A9DED047A77EEA76AFA
:10887000B4EEE70AF1EE10FAF4EEC76AACBF0120DD
:108880000020F1EE10FA0CD802309DED037AF4EEE0
:10889000C77AF1EE10FA0CD8003818BF01200AB0E0
:1088A00010BDF4EEC77AF1EE10FA9CBF0130C0B2F1
:1088B000EBE7012894BF00200120F0E70020EEE75D
:1088C00010B5074B1A7A4AB901241C724CF03EFDD0
:1088D00022461121BDE810404CF0F0BA10BD00BF97
:1088E000F890002010B5074B1A7A4AB100241C7288
:1088F0004CF02CFD22461121BDE810404CF0DEBAB0
:1089000010BD00BFF8900020F0B5054685B0684660
:1089100005F5A2560EF02EFF6946304609F040FBE1
:10892000A0B13348334C344F75F0E8FD40B105F544
:108930003C53D3ED007AF5EEC07AF1EE10FA07D889
:10894000002328462380FB73FFF7CCFF05B0F0BD62
:108950002846FFF761FFA0B363787BBB2378013320
:10896000DBB2082B237002D1304609F031FA2378AC
:10897000092B02D1304609F023FA2378092B1DD99F
:108980004FF4857323804CF0E1FC022210214CF05F
:1089900095FA7FF03DFC6368C01A47F23053984265
:1089A00009D905F55B50154A022120304FF018FE19
:1089B0007FF02EFC60602846FFF782FF6378FB7330
:1089C000C4E72678002EF9D0013E6378F6B226700F
:1089D000002BF3D0002EF1D166704CF0B7FC32467C
:1089E00010214CF06BFA2846FFF77CFFE6E700BF4A
:1089F0003C900020F89000209D91002074DE0C082F
:108A000000F5A040D0F82038042B14BF90F84C0893
:108A10000120704773B500F5A0450192A5F8B41187
:108A200004467FF0F5FBC5F8B801D5F89C01036852
:108A30005B68984785F8B201D5F89C0103685B68CC
:108A400098470F28019A0BD80F2827D8DFE800F0A5
:108A50001C261C1C1C1C1C1C1C2650260A260A0A30
:108A600018281BD104F50056019296F9DC34ABB1FD
:108A7000D5F89C0103685B68984785F8B20196F9C0
:108A8000DC34019A022B29E0204B93F8D23403B353
:108A900004F5A0413C31204605F0E6FDD5F89C01E7
:108AA00095F8B26103685B68984704F55B548642A9
:108AB00004F1200422D0D5F89C0103689B689847F4
:108AC000134A03460421204602B0BDE870404FF02F
:108AD00087BD04F5005393F9DC34022BD8D0042B66
:108AE0000BBF04F5A04104F59F4144317C31D2E72E
:108AF0002046FFF785FF0028D0D1B3E7054A0421BF
:108B0000204602B0BDE870404FF06ABD108C0020D6
:108B100084DE0C08A6DE0C08F0B5044604F5A04679
:108B200085B00F46154658F027F8D6F89C01A6F8F0
:108B3000B47103685B68984718281ED8DFE800F016
:108B40000D0D0D0D0D0D0D0D0D1D53680D0D58580E
:108B50001D1D1D1D1D1D1D1D0D00314BD3F8202891
:108B6000012A21D104F5005393F8DD34023B012B97
:108B70001AD904F5405383F8DC26D6F89C01294A1B
:108B8000294B052D18BF134602680393926890473E
:108B900004F55B5420340090039B244A04212046B2
:108BA0004FF01EFD05B0F0BD214B93F8D2343BB120
:108BB00004F5A0412A463C31204605F055FDDCE78E
:108BC00004F5005393F9DD34032B03D1204603F061
:108BD00089FCD2E7022BEBD0042B15D104F5A04180
:108BE0002A466831E8E72046FFF70AFF0028C4D18B
:108BF00004F5005393F9DD34032BE7D0022BD7D0D3
:108C0000042BEBD0012BB8D12A4604F5A141D3E7C0
:108C100004F5005393F9DD34042BAED1DEE700BF39
:108C2000107C0020BCDE0C08B5C20C08C4DE0C08A9
:108C3000108C002070B500F55B5504462035124AB3
:108C40000421284604F5A0464FF0CAFC0023A6F8EC
:108C5000B43104F5005393F82434032B12D196F861
:108C6000B2113022204605F0D7FDD6F89C010368EA
:108C70009B689847054A034606212846BDE8704090
:108C80004FF0AEBC70BD00BFD8DE0C08EFDE0C08A4
:108C900000F5405310B500220529044600F55B504D
:108CA00083F8DC2600F120000CBF054A054A0421A8
:108CB00004F5A0444FF094FC0023A4F8B43110BD97
:108CC00008DF0C0819DF0C0830B50B4687B00446E6
:108CD000052A19D8DFE802F0182C0352185F00F5B6
:108CE000A043D3F82038042B22D02D4D95F8C53160
:108CF000F3B105F5995105F6440026F0A5F928B120
:108D0000274B012283F84C2807B030BD05F5995157
:108D100005F6440026F098FC50B104F5A041042269
:108D20006831A5F5A04007B0BDE8304005F09CBC17
:108D300004F5A043D3F82038042BE5D004F5005304
:108D400093F9A734022B0BD1154890F8C5313BB1EC
:108D500000F5995100F6440026F076F90028CFD1AD
:108D6000042204F5A141204605F07EFC04F51150D3
:108D7000273007B0BDE8304042F0C4B9094A11219C
:108D800001A87EF0FBFA04F5C54001AA01210430D8
:108D900078F04EF9B8E707B0BDE8304003F0A2BB69
:108DA000107C002034DF0C0870B52DED048B0446D8
:108DB0007FF022FA4F4BB4F8BE101A884E4E8A420A
:108DC00005464E4A06D01980002330601370BDEC72
:108DD000048B70BD33684A49C31A8B4276D901238C
:108DE000137057F0C9FF57F081FE356057F0C4FF8C
:108DF00057F07CFE04F5405393F8DB3623B104F5BD
:108E0000C540043078F068F857F098FE0428DED9A1
:108E100057F0B2FE0021204603F08EFE00212046CE
:108E2000F0EE409A03F092FE01212046B0EE409A07
:108E300004F052F800212046B0EE408A03F090FE84
:108E400004F5C8402C30F0EE408A75F061FBDFED90
:108E50002D7A0028B0EE690A4FF0040008BFB0EE8A
:108E6000678A59F009FBB0EE490A132059F004FB58
:108E7000B0EE680A152059F0FFFA04F5C545B0EECA
:108E8000680A1A2059F0F8FA04354620B0EE480A6C
:108E900059F0F2FA284678F0ADF808BB01210846EF
:108EA00059F0ECFD9FED170A022059F0E5FA9FED0D
:108EB000150A032059F0E0FA204604F027FABDEC29
:108EC000048B2046BDE8704005F052B91278002AA4
:108ED0003FF47DAF44F6206293427FF678AF80E79F
:108EE0002846FDF71FF804F5C04393F98E322B2B6B
:108EF000D4D06CE704910020089100200691002056
:108F0000400D03000000000000F5A0431846D3F810
:108F10009C216830824202D193F84C08E8B10F4B93
:108F200093F8240403F58043A0F12702012A93F863
:108F3000E0340FD92C2809D00A2809D0A0F1310239
:108F4000504250410A2B18BF002070470120F9E71A
:108F5000012070470A3B584258417047104C00208E
:108F600008B500F5005393F8102342B193F84C3341
:108F70002BB1FFF7C9FF80F00100C0B208BD01208E
:108F8000FCE700002DE9F04700F50055A54F95F8E6
:108F90004C83044600F5C8408AB02C3075F0AEFA18
:108FA000D7F82038042B06464FD000284DD0B7F80C
:108FB0008218A7F5A040FFF709FB014620B197F8FA
:108FC00048184B1E5942594104F50C57DFF868A266
:108FD0001037384664F034FE9AF8E0340A2B8146A4
:108FE00003D1A6BB00238AF8E03495F81033002B98
:108FF00039D195F916338C4D012B03D0063BDBB2EA
:10900000012B11D895F824340A2B0DD104F5A04674
:10901000D6F89C0103681B6A984728B1D6F8A011BE
:109020002B22204605F020FB9AF8E0340A2B04BFDF
:1090300037238AF8E03495F824340A2B02D13723F9
:1090400085F824340AB0BDE8F0870121BCE740EA86
:109050000803DBB2002BC8D1AAF5C04000F0EEF83F
:109060000028BFD0C1E7002EECD004F5C340783013
:109070007AF086FF0028E5D12046FFF745FF00285B
:10908000E0D1B9F1000F00F0BC8068494A4638468B
:1090900064F0AEF995F91683B8F1010F06D040F3EC
:1090A0008280A8F10603DBB2012B7CD85FFA88F836
:1090B000B8F1010F4AD104F5A0421346D2F89C1131
:1090C0006833994207D192F84C3823B195F8A73408
:1090D000013B012BB6D90A2204F5A141204606AE78
:1090E00005F0C2FA30460EF045FB95F9292392BBF4
:1090F000B8F1010F2FD004F5C048B5F92A33D8F8DC
:109100000C13DFED4B5AD1ED017A002BF8EEE77A24
:1091100052DD07EE103AF8EEC76AE6EEA57A304661
:10912000FDEEE77A17EE901A0EF02AFB0023384680
:10913000CDE9043364F020FE04A965F061FB00284A
:1091400059D0049B0893059B099317E004F5A141AE
:109150000A221031C2E72046FCF75CFF07EE900AB6
:109160006F4604F5C642203221463846B8EEE70A7B
:10917000FEF772F897E80F0086E80F0095F91633AE
:10918000012B10D031462046FDF7B2FB3146204678
:10919000FDF748FF95F91633072B04D104F5405429
:1091A000012384F8DA364CF0D1F84A4609210AB096
:1091B000BDE8F0474BF082BED5EDC66A95EDC95AC1
:1091C00095EDC77A35EE076A36EEC57AB4EEC67A03
:1091D000F1EE10FA8DBF37EE067A05F5A16393ED37
:1091E000007A27EE257A8ABFF6EE006AE7EE257A46
:1091F000E7EE267A93E7D8F80C339A680892DB6892
:10920000A2E7B8F1000F3FF41DAF95F84C33002BE7
:109210007FF418AF04F55B50064A052120304FF06B
:10922000DFF9C0E7107C0020104C002040DF0C0864
:109230000000C84249DF0C08108C002010B504461D
:1092400000F5C8402C3075F063F904F5A04404F62D
:10925000240494ED007A48B1DFED067AB4EEE77AA3
:10926000F1EE10FAACBF0120002010BDDFED027A54
:10927000F4E700BFCDCCCC3D6666663F10B500F587
:10928000A04200F5A141D2F89C412C318C4203460A
:1092900002D192F8180888B903F5A04368339C42BC
:1092A0000DD192F8180848B1D2F82038032B06D116
:1092B000B2F88208A0F116035842584110BD0020B0
:1092C000FCE700002DE9F84F00F5A0463346D6F83C
:1092D0009C2168339A42054604D100F5005898F95C
:1092E000803433B90023C6F80C3886F80938BDE855
:1092F000F88F7EF08DFFD6F8C047814634B1041B4D
:1093000040F6C3139C4294BF002401242846FFF773
:1093100095FF834620B1002486F8084800273FE0E7
:1093200005F5C8402C3075F0E9F882460028F2D0E7
:1093300005F5C347783738467AF022FE002840D03A
:1093400096F80878C7BB44B305F5805141F27072B6
:10935000D1F83836002BB8BF5B42934206DCD1F817
:109360003C36002BB8BF5B42934228DD05F5B14186
:1093700005F5C640083120300EF05EFDDFED457A80
:10938000C6F80C98B4EEE70AF1EE10FA4FF00003BD
:109390004CBF01270027C6F81038012386F808388B
:1093A00005F59070F8F7B6FB022835D9002C44D1AA
:1093B0000023C6F80C389AE75C465F46EDE73C466A
:1093C000EBE738467AF0C4FD074638B1002CA5D04B
:1093D0004FF4FA73C6F8103854469FE7D6F8203891
:1093E000012B03D0032B0FD03C46D9E708F5A4632B
:1093F000D3ED007AF5EEC07AF1EE10FAF4DD96F8CE
:109400001838002BF0D1E3E72846FFF737FF002894
:10941000EAD1002CDCD1C3E705F5055A98F88E1285
:10942000504606F059FE0028C2D098F88E125046D9
:1094300006F04AFF0028B9D1BAE7D6F80C3813B9BC
:10944000C6F80C9853E7D6F81028A9EB030393420B
:10945000FFF44DAF96F80938002B7FF448AF012296
:1094600086F8092898F88034DB0705D505F5C8404B
:109470000C212C30F8F786FA05F55B5020302FB11F
:10948000054A0221BDE8F84F4FF0AAB8034A394611
:10949000F8E700BF0000964260DF0C0876DF0C089A
:1094A0002DE9F04F2DED028B054685B0002305F523
:1094B000005803937EF0ACFE08F27C43D3ED007AB3
:1094C000F5EEC07AF1EE10FAC4BF9FEDC07A67EEF8
:1094D000877A05F5907BC8BFFCEEE77A07465846C9
:1094E000CCBF17EE906A9626F8F714FB022840F2DC
:1094F000FB8095F814349FEDB67AB02202FB03533B
:10950000D3ED837A67EE877AFCEEE77A17EE903A2E
:109510009E428CBF00260126B8F97034022BB8BFDA
:10952000022307EE903AB8EEE78A03A9F6EE087A2E
:1095300005F5A25028EE278A08F010FD044640B138
:10954000DDED037AF4EEC87AF1EE10FAACBF012437
:1095500000245846F8F7DEFA05F5C849012809F154
:109560002C0905F5A04A18D8484674F0C7FFA0B1E9
:109570009CB90AF6240292ED007ADFED967AB4EEF9
:10958000E77AF1EE10FA08DDDDED037AF4EEC87A41
:10959000F1EE10FAACBF01240024484674F0AEFF8F
:1095A0000090002800F0FE8095F8142405EB0212CC
:1095B000D2F8C02172B158460192F8F7ABFA0128EF
:1095C00000F29480019A41F28731BA1A8A428CBF24
:1095D00000220122DAF8BC1701B11AB9002C40F0C0
:1095E00087803446DAF89C1105F5A0426832914232
:1095F0001AD198F9A824002A40F0828000228AF823
:109600000A28DAF82028042A00F0AA80072A00F0A5
:10961000BD80032A08D12846FFF730FE20B1002480
:109620008AF80948CAF8C0479AF80A2802B18CB9E2
:1096300007EE904A9FED687AF8EE677A0AF6240200
:1096400067EE877AD2ED006A9FED647AE6EE877A5C
:10965000C2ED007A2846FFF7F1FD044698B19AF86A
:109660002808CAF8BC7708B9CAF82C78DAF89C112F
:1096700005F5A0426832914205D1DAF8C02702B15F
:1096800008B9CAF8C0779AF850298AF8284864F3CC
:10969000C3028AF850296FF06BF821466FF044F846
:1096A0004F4A28465471FFF70DFE2846FBF73AF95A
:1096B00034B198F826241AB97EF0AAFDC8F8280417
:1096C00088F826442846FFF7B9FD00287BD1484694
:1096D00074F01EFF80F00100C0B28AF8300805B0B7
:1096E000BDEC028BBDE8F08F002615E7002271E784
:1096F0001FF094FB1EF088FB00287FF472AF71E727
:10970000524207EE902A05F61862F8EEE77A92EDDB
:10971000007AF4EEC77AF1EE10FA13DD01228AF82E
:109720000A28CAF814780AF62402DFED2E7A92EDA0
:10973000007AB4EEE77AF1EE10FA7FF762AFC2ED8D
:10974000007A5EE79AF80A28002A3FF45AAFDAF85E
:10975000142840F6B831BA1A8A423FF64FAF50E7A4
:1097600005F5C34078307AF0F3FB00283FF45CAF96
:109770000AF2AC7292ED007ADFED1A7AB4EEE77A73
:10978000F1EE10FA7FF750AF009C4DE70AF2AC7291
:1097900092ED007AFEEE007AB4EEE77AF1EE10FA7E
:1097A000F2D441E7DAF82028002C18BF3446012A09
:1097B00007D005F5C34078307AF0C0FB00283FF4AD
:1097C00033AF002430E7002087E700BF0000B44239
:1097D0000000C8429A99993E9A99193E9A99593F20
:1097E0009D910020CDCC4C3E00207047002070475A
:1097F000012070470020704701207047034BD3F8C9
:109800002008431E58425841704700BF107C00207A
:1098100030B587B002A80DF0ADFF3B487AF08EFB63
:1098200020B13A493A48FDF775F81FE036487AF01A
:109830008FFBE8B1374C04F12405234604F11002F4
:10984000A4F11001A4F5947000957AF0A7FBCDE97E
:109850000045A4F66C3292ED000A2F4904F1100382
:10986000A4F11002A4F594707AF05AFB07B030BD51
:10987000254802A97AF0AAFB08B102A9D2E7274C31
:10988000D4F8A83E002B0CDD94F8483E4BB1A4F56B
:1098900000502049FDF73EF8A4F50050FCF7D2FC3B
:1098A000E4E71B4802F0DCFC0028BAD11C4C94F819
:1098B00030335B0720D4D4F84433002BB1D0134AA3
:1098C000A2F12001A2F110000EF022FA0028A8D186
:1098D000144C0F48D4ED007AB7EE000A04F6783144
:1098E00030EE670AFDF746F8094804F6583204F6E8
:1098F0007831FCF7EBFBB9E7A4F5C040FDF7B6F80B
:109900000028B3D1D7E700BF088E0020408F002089
:10991000102C0020308F0020585B0020104C0020BD
:10992000108C0020C883002008B50A4890F819352B
:10993000013B012B03D8A0F50050F9F74BF906487D
:10994000F9F772F80448F9F70BF9BDE80840024846
:10995000F9F726BC104C0020102C0020124A90422F
:1099600008B50ED002F1080188420AD002F11001B8
:10997000884206D002F13801884202D05C3290421F
:1099800006D10A4B93F9D104B0FA80F0400908BD22
:1099900003681B6A984728B1054B93F8DA0680F0F4
:1099A0000100F4E70120F2E7147C0020104C0020B5
:1099B000105C0020104A904208B518D002F108014E
:1099C000884214D002F11001884210D002F138010F
:1099D00088420CD05C32904209D003681B6A9847D9
:1099E00038B1064B93F8DA0680F0010008BD00207C
:1099F000FCE70120FAE700BF147C0020105C002087
:109A0000024A0260024A4260704700BFC8DF0C0889
:109A10005040002008B503681B6E98470648D0F8F0
:109A20009C2100F160039A4205D0BDE80840A0F5F2
:109A3000A040FEF79DBE08BD107C00202DE9F84334
:109A4000484C04F2947300221A6004F16803C11AAE
:109A50004B42A4F500584B4188F87C3904F2A473BA
:109A6000002584F87857A4F8CE5784F8D25784F8A4
:109A7000905784F8095884F80A58C4F8F857C4F87D
:109A8000F457C4F8F057C4F800581A604368D3F884
:109A9000FC31A4F8C83704F5995306460FCB04F5FA
:109AA000805909F5447787E80F0084F8D15784F886
:109AB000E057C9F8EC527EF0ABFBC4F8A401336860
:109AC00030465B6998474FF0FF3384F8D40784F839
:109AD000D55788F8DC5689F8495384F8D357C4F829
:109AE000CC3133683046DB6D98470546002836D0C8
:109AF000336830469B6B984784F81808D8F80809F3
:109B00000368DB6B984708F5CF6076F0E3FEA4F5B9
:109B1000A04002F07DFFA7F5804064F0F7F894F8CC
:109B20004C38CBB1A4F5A040FFF788FBA0B907F5EE
:109B30008E7074F0EDFC78B9D4F89C0103685B6B0F
:109B4000984748B955F024FC074A06214EF048FDD5
:109B500004F6440025F024FB0448F8F797FA284659
:109B6000BDE8F883107C002088DF0C08102C002052
:109B700070B503685B6E0E4615469847044650B9AB
:109B800095F900303BB90548054B00683246C06A7C
:109B900029461BF0E7FF204670BD00BF0C2C0020BB
:109BA000ACDF0C0810B50E4C204676F08FFC04F5A7
:109BB000AC7076F007FA04F52C7077F035F9094BA4
:109BC00003F5A042002182F8901702F2947200215E
:109BD00003F540531160012283F8A02110BD00BF9E
:109BE000645E0020102C002008B52DED028B15209E
:109BF000B0EE408A58F040FCB0EE480ABDEC028B53
:109C00001A20BDE8084058F037BC000008B50848E5
:109C100090F9D1340121A0F5005033B103F05CF983
:109C2000BDE80840462058F027BC03F07DF9F7E76F
:109C3000104C00200420704700487047BA230E08DB
:109C400000487047BA230E08037A73B1D0ED037A47
:109C5000FDEEE77A17EE903A084AC2F83438437AB4
:109C60003BB10369C2F8383870474368D3F8F8311C
:109C7000F2E74368D3F8FC31F4E700BF107C002022
:109C800008B50023038100F11401406808F07CF955
:109C9000012008BDF8B56D4E2DED048B0446012161
:109CA000304606F5A04797ED799ADFED699A02F004
:109CB00043FF0121B0EE408A304602F047FFC8EE74
:109CC000297A06F500556068B5F9F43404F11401F9
:109CD00008EE903AF8EEE88AB5F9F63468EEA78A0D
:109CE000C0EE297A08EE103AB8EEC88A28EE278A24
:109CF00008F04AF995F9FA345BB39FED567AF0EE25
:109D0000E87AF4EEC77AF1EE10FA22D5227A636887
:109D1000002A54D1012222720022E26094ED037ADB
:109D2000DFED4D7AD3F8F8314C4867EEC77A9FEDF6
:109D30004C7A67EE877A0122FDEEE77AB0EE490AA7
:109D400017EE901A0B44C7F83438002376F04EFB18
:109D500008E0002341482372F0EE490AB0EE680A99
:109D600076F040FB042058F087FB95F9FA3443B1B4
:109D70009FED387AF0EEC87AF4EEC77AF1EE10FA79
:109D800028D4002337486372F0EE490AB0EE480A3F
:109D900075F082FF132058F06FFBB5F9F834002BF3
:109DA00003DD314E96F91A355BBB28482021F8F7C0
:109DB000D3FB002842D1254802F0FAFC41E0D3ED64
:109DC000C56A96ED467AD4ED037AE6EE877AC4ED5D
:109DD000037AA3E7637A2BB9012363726368D3F82C
:109DE000FC3123612169C7F838186368D3F8FC0196
:109DF0000023091A1A461B48B0EE490A76F032F8D9
:109E0000C8E70121A6F5405002F0AAFE80EE297AAB
:109E1000B5F9F834002106F2045007EE903AF8EE56
:109E2000E77AF0EE490A27EE870A76F0FDFEBDECF0
:109E3000048B2046BDE8F840FFF7D6BE0348F9F78B
:109E40001BF807EE900AB8EEE70AF0E7102C0020A6
:109E500000A08C4500000034E02E6542645E0020C6
:109E60000000C842BC5F0020105C00202DE9F04FCC
:109E70002DED0C8BDFF8A0A39FEDDCDA9FEDDC9AD3
:109E800097B000F114050AF5A04B04460121504695
:109E90009BED79BA02F050FE01215046F0EE408A67
:109EA00002F054FE01215046B0EE408A02F058FE06
:109EB000DFEDD07A88EEA77A0AF5005601A8B6F948
:109EC000F4340AEE903AF8EEEAAAB6F9F634DFED89
:109ED000CA8A6AEE87AA88EE277A0AEE103AB8EEA6
:109EE000CAAAB6F9F8349FEDC58A2AEE07AA80EE11
:109EF000277A09EE903AF8EEE99A6AEE8D7A69EEE1
:109F0000879AF0EEEACAF4EEC8CACDED017AB0EE57
:109F1000CACA6AEE0D7AF1EE10FAF0EEE9BAB4EEC2
:109F2000C8CACDED027A58BF4FF0010969EE8D7AAB
:109F300048BF4FF00009F1EE10FAF4EEC8BA9AEDFE
:109F4000460ACDED037A54BF4FF001084FF00008E8
:109F5000F1EE10FA54BF0127002721F0B7FF01A945
:109F6000284621F0BDFA284621F0ACFB284621F016
:109F700023FB20EE090A284620EE280ABDEEC00A7F
:109F800010EE103ACBF8343821F030FB20EE090AFD
:109F900020EE280ADFED9A8ABDEEC00ACDED0D8ACB
:109FA00010EE103ACBF838380DF1280B4FF07E53F5
:109FB000594660680A93CDED0C8ACDED0B8A07F007
:109FC000E3FF0021504602F087FFB0EEC00AB4EE76
:109FD000C80AF1EE10FA16D55046FFF72FF990B9DE
:109FE000F4EEC8CAF1EE10FA0DD5B4EEC8CAF1EE1F
:109FF00010FA08D5F4EEC8BAF1EE10FA44BF9BE8A7
:10A000000F0085E80F000AA821F0C0FB294612A81E
:10A010008DED141A8DED120ACDED130ACDED151A42
:10A0200021F0C6FB0DF1100A51460EA88DED101A55
:10A03000CDED048ACDED058ACDED068A8DED0E0AB3
:10A04000CDED0F0ACDED111A21F084F9B6F9F434F3
:10A05000DFED6C7A01EE103AB6F9F63409EE103AFB
:10A06000B6F9F83408EE903AB8EEC11AB8EEC99ACB
:10A07000F8EEE88A21EE271A29EE279A68EEA78AD9
:10A08000F4EEC8CAF1EE10FA21EE0D1A29EE0D9A7F
:10A0900068EE8D8A07D594F82430DFED597A002BCD
:10A0A00018BFB0EE671AB4EEC8CAF1EE10FA07D5C1
:10A0B00094F82530DFED527A002B18BFB0EE679A86
:10A0C000F4EEC8BAF1EE10FA07D594F82630DFEDB9
:10A0D0004C7A002B18BFF0EE678A9AE8070007AEAB
:10A0E00086E80700F1EE410AC2209DED070A1FF045
:10A0F00017FCC3208DED070AB0EE491AF1EE490AAC
:10A100009DED080A1FF00CFCB0EE681AF1EE680A2B
:10A110008DED080AC4209DED090A1FF001FC51468F
:10A1200030468DED090A21F067FE12A928468DED13
:10A13000120ACDED130A8DED141A21F0D1F928463B
:10A1400021F0C0FA304BDDED076A93ED967A9FED72
:10A15000280AC6EE877A3046DDED086ACDED077A2B
:10A16000D3EDEC7A86EEA77ADDED096A8DED087AFB
:10A1700086EEA77A8DED097A21F0A8FEB9F1000FDD
:10A1800001D0CDED07AAB8F1000F01D08DED08AADE
:10A190000FB1CDED099AF0EE4B0A9DED070A1B4871
:10A1A00076F020F9042058F067F9F0EE4B0A9DEDA7
:10A1B000080A174875F070FD132058F05DF900216A
:10A1C000F0EE4B0A9DED090A124876F02DFD20466F
:10A1D000FFF70AFD84F8249084F8258084F826701F
:10A1E00017B0BDEC0C8BBDE8F08F00BF35FA8E3C8C
:10A1F000E02E654200A08C450000C84200000034FB
:10A2000000000000CDCC4C3E105C0020645E0020BD
:10A21000BC5F002014610020102C002010B5044603
:10A22000FFF7F4FC0B4B93F9FA24022A0DD1B3F992
:10A23000F824002A09DD03F5805393F91A3523B178
:10A240002046BDE81040FFF711BE2046BDE8104093
:10A25000FFF720BD104C00200A20704700487047CF
:10A26000E9EB0C0800487047E9EB0C080120704747
:10A27000012070470120704701207047012070477E
:10A28000034BD3F82008031F58425841704700BFC2
:10A29000107C0020F8B51C4E06F599530FCB06F53F
:10A2A000805505F5447405F54C7584E80F0085E884
:10A2B0000F00002706F6440086F8D47725F0B0F9A1
:10A2C000124B1C68E56A2B6828465B689847A8B162
:10A2D00095F84D3093B1E36A9B8F7BB155F058F8F8
:10A2E000E36A0B4A9B8F06214EF07AF9E36A06F681
:10A2F0004400998F24F080FFE36A9F8705487AF035
:10A30000B5FD0120F8BD00BF107C00200C2C002002
:10A31000A0E00C08D058002010B50A4C94F848383A
:10A32000012B0AD104F6440022F03EFAB4F8823838
:10A33000152B02D1044879F0E1FE0023C4F8C037A0
:10A3400010BD00BF107C0020088E002008B508F06A
:10A3500021F890F87C32DB0704D5BDE808400248BC
:10A3600024F0FABF08BD00BF5484002010B52F4C64
:10A3700094F84838012B0ED004F180010822A4F58E
:10A38000A04004F071F955F003F8BDE81040284AE8
:10A3900006214EF025B9B4F88238162B05D0152BBE
:10A3A00034D1D4F82038072B0AD1224804F0E6FC37
:10A3B000204804F02DFEBDE810401E4804F040BDCA
:10A3C000A4F5A040F9F75CF8A4F5A040F8F756FF13
:10A3D000A4F54053D4F8341893F93825164864236B
:10A3E0005A4379F0E7FDC4F83408134879F024FFA4
:10A3F00030B1BDE810409FED110A462058F03CB83E
:10A40000A4F5A040BDE81040F8F71EBD1E2B18BFF4
:10A410004FF0FF33074818BFC4F88C37F9F730F80E
:10A420000448F8F72BFF0348ECE700BF107C00203E
:10A43000B8E00C08102C0020088E0020000000005E
:10A4400010B5144BB3F88238532B04461ED103F0D9
:10A4500033F99FED110A462058F00EF89FED0E0AD1
:10A46000492058F009F89FED0C0A4A2058F004F8EA
:10A47000462058F0E1F8492058F0DEF84A2058F01C
:10A48000DBF82046BDE81040FFF78CBBBDE810406C
:10A49000FFF74ABA107C0020000000000820704737
:10A4A0000048704754E10C080048704760E10C0810
:10A4B0000120704708B50248FEF7FAF8012008BDF0
:10A4C000102C0020014800F061B900BF4C7C002036
:10A4D00010B50446FFF728FA2046BDE81040FFF704
:10A4E00095BB00000120704700487047D8E10C0878
:10A4F00000487047E0E10C080120704701207047D8
:10A5000010B5054B03F54C7403F548730FCB84E885
:10A510000F00012010BD00BF108C002008B50B48B3
:10A5200000F5A04200F500530321D3F8383F93FB18
:10A53000F1F3C2F83438F8F709FF0448F8F79EFE43
:10A54000BDE808400148F8F77FBC00BF102C002090
:10A55000072070470048704772C40C0800487047D5
:10A5600058E20C0801207047012070470120704715
:10A570007047000010B5064C0023037203612046AB
:10A580007AF074FCA4F53350FCF782F9012010BD79
:10A59000D058002010B5194CD4F8203FB3F908303A
:10A5A00023B9D4F82C3FB3F90830F3B10023037278
:10A5B0000361D4F8200F56F0CFFC04F63873D3EDC6
:10A5C000007A0F48F8EEE77A27EE800ABDEEC00A5F
:10A5D00010EE103AC0F83438A0F5A040F8F7B6FEF7
:10A5E000BDE81040074801F037BD037A002BE0D0EA
:10A5F000A4F50050F8F744FFF2E700BF104C00202C
:10A60000107C0020102C002070B54E4DDFED4E7AEE
:10A6100095F814349FED4D7A2DED048BB02606FB92
:10A62000035393ED848A9FED4A9A28EE278A05F515
:10A63000B253BDEEC88A93ED030AF8EEC87A044619
:10A6400067EE897A97EE870A1FF056F9237AF0EEC3
:10A65000408A002B62D105F50053D3F8203FB3F9AF
:10A660000830002B5AD1284602F0A2F8002855D114
:10A6700095F8143495F8581406FB035393F8F12118
:10A6800000294BD1012A49D993ED837AF0EE087A5B
:10A69000B4EEE77AF1EE10FA40DBDFED2E7AB0EEA1
:10A6A000E80AB4EEE70AF1EE10FA37D5236993B35E
:10A6B0007DF0AEFD2369C01AB0F5FA7F32D8237A57
:10A6C000002B3CD0244DA5F1200696E80F0085E82C
:10A6D0000F0094ED038AA5F110013046B8EEC88A48
:10A6E0000DF0AAFB28EE098ADFED1C0A284670EE61
:10A6F000200AB0EE480A0DF015FC194B9FED190A1F
:10A70000D3F80809BDEC048B03682A4631469B6ADE
:10A71000BDE8704018477DF07BFD20612369002B68
:10A72000CDD0C5E7104D84ED038A012323720023A9
:10A73000236105F110030FCB85E80F00BFE7BDECE7
:10A74000048B70BD102C00200000C84235FA8E3CEE
:10A750000AD7233CDB0FC93F408F002000007A441A
:10A76000105C002000000000208F0020C3680B60F8
:10A77000007A70470520704700487047D0E20C0807
:10A7800000487047E0E20C080120704738B52DED15
:10A79000028B4D4C9FED4D8AD4F8200F56F0DCFB18
:10A7A000D4F8383F07EE903AF8EEE77A04F54055D2
:10A7B00027EE800AA4F50050BDEEC00A10EE103A54
:10A7C000C5F83438F8F7C2FDD4F8240F56F0C4FBAE
:10A7D000B5EEC00AF1EE10FACBBF04F5916304F6B2
:10A7E0003C73D3ED007AD3ED007A3948CBBF20EE2D
:10A7F000270A20EE270A20EE080A28EE400ABDEEBE
:10A80000C00A10EE103AC5F83838F8F769FD04F5BB
:10A81000916393ED007AD5F8380804F63C7327EE7F
:10A82000087AD3ED007A27EE888AFDEEC77A17EE14
:10A83000902AFDEEC87A17EE901A1FF011F9C5F8AC
:10A8400038082348FDF7C0FF20B1D5F838385B42FF
:10A85000C5F8383895F8B03163B194F9DC34022B7F
:10A8600008D1002301214620C5F83438C5F838380E
:10A8700058F05CF956F080FA5F2157F0AFFAF8B162
:10A8800057F07CFA02281BD195F8D137C3B905F2ED
:10A89000A47304F5A56493ED007AD4ED007AB4EEC8
:10A8A000E77AF1EE10FA0BD5012385F8D137BDEC2C
:10A8B000028B084A0848BDE8384004214DF090BE9C
:10A8C000BDEC028B38BD00BF104C00200000C84218
:10A8D000102C0020E8E20C08F062002010B50446BD
:10A8E000FFF722F82046BDE81040FFF78FB90000BF
:10A8F000062070470048704768E30C08004870471E
:10A9000078E30C0801207047012070470120704750
:10A91000012070477047000010B5054C20467AF0C2
:10A92000A5FAA4F53350FBF7B3FF012010BD00BF1B
:10A93000D058002038B50F4C04F50055D5F8200F3D
:10A9400056F00AFB05F63872D2ED007AF8EEE77A97
:10A9500004F5A04327EE800A2046BDEEC00A10EEA3
:10A96000102AC3F83428F8F7F1FC2046BDE8384037
:10A9700001F072BB102C00200F2070470048704778
:10A98000F0E30C0800487047F8E30C08012070471A
:10A990000120704701207047012070470120704757
:10A9A000012070477FB50B4D05F54053002283F819
:10A9B000DA2605F5C643203306460FCB6C4684E8FD
:10A9C0000F0000232846B3602146FCF72BFB012033
:10A9D00004B070BD102C002010B53C4CD4F8F037FA
:10A9E000002B2CDD7DF014FCD4F8F037C01A40F6B3
:10A9F000B733984223D8A4F54053D4F8E407D3F8EA
:10AA0000382F51421FF02CF8C4F83408A4F5A040A8
:10AA1000F8F79CFCD4F8F437002B14DC2C48F8F73A
:10AA20002DFC2C4890F8DA3693B30121A0F5405064
:10AA300002F052FABDE81040462057F01DBD2448F0
:10AA4000F8F71EFDE6E77DF0E3FBD4F8F437C01A13
:10AA500040F6B7339842E1D81F4BDFED206A93ED03
:10AA6000007AD4F8E80703F6B423D3ED007A27EE92
:10AA7000267A67EEA67ABDEEC77AFDEEE77A17EE84
:10AA8000102A17EE901A1EF0EBFFC4F83808C8E73A
:10AA9000A0F5805090F96734012B04DCBDE810402C
:10AAA0000B48F8F7D1B9D4F80038002BF6D07DF078
:10AAB000AFFBD4F80038C01A40F6B7339842EDD84F
:10AAC00004F2FC7494ED000AB4E700BF107C00208F
:10AAD000102C0020105C0020985000200000C8427C
:10AAE000D0ED027A0348FCEEE77A17EE903A99B27D
:10AAF00001F09CBC102C002084B010B503AC84E89D
:10AB00000E000B4821466F22FCF7D0F99DF80C107F
:10AB100011F0040102D120460CF0F6FE0448214653
:10AB2000FCF780FABDE81040012004B0704700BF78
:10AB3000102C0020B0EEC00AFDEEC07A38B54FF6FA
:10AB4000FF7205460C4617EE900A00211EF088FFA2
:10AB500007EE900A002CF8EEE77A054BC5ED027A75
:10AB600014BF4FF0FF32012283F8E82238BD00BF46
:10AB7000108C0020FEF74CBE0C2070470048704738
:10AB800070E40C0800487047A9230E0801207047A4
:10AB90000120704701207047012070470120704755
:10ABA00008B50C48FDF78EF80A480B49FBF7A0FEE4
:10ABB0000848F7F7C7FE40B106484FF48051F7F751
:10ABC000CBFC10B10348FBF763FE024800F0A0FF86
:10ABD000012008BD102C0020408F002008B50D4832
:10ABE000F8F74EFC0B48F7F7ADFE50B109484FF4AB
:10ABF0008051F7F7B1FC20B1BDE80840054801F0ED
:10AC00002BBA0448F8F73AFBBDE808400148F8F7CA
:10AC10001BB900BF102C002008B50A484FF4805122
:10AC2000F7F79AFC38B108480022D0F8401300F535
:10AC30004C700CF0A5FDBDE808400248002101F071
:10AC4000F5BB00BF102C0020108C0020881A10B516
:10AC50001EF02EFE104BD3F8E4220028B8BF40426D
:10AC6000002AB8BF524248F6A041B2FBF1F24FF4BD
:10AC70007A7102FB011188420CDC93F83023D20672
:10AC800006D503F54C7403F548730FCB84E80F0029
:10AC9000012000E0002010BD108C002013B50446F8
:10ACA0004068019100F57F7020F04AFFDFED0A7ADD
:10ACB00020EE270A1EF09EFDDFED087A019920EEB6
:10ACC000270A2046FDEEC07A17EE902A02B0BDE8B2
:10ACD0001040FFF7BBBF00BFE02E65420000C84236
:10ACE00084B070B52DED048B86B00FAD85E80E00F5
:10ACF0004D4CDFED4E8A0646D4F8080904F5405461
:10AD000094EDBF0A0368B0EEC00A5B6A9847B4EEE0
:10AD1000E80AF1EE10FAB0EE408A07DA012006B038
:10AD2000BDEC048BBDE8704004B070474049284634
:10AD30000CF08EFF02A8CDED030A8DED020A20F083
:10AD4000A3FF04A88DED040AB0EE480ACDED050A74
:10AD500020F094FE13A928468DED000ACDED010ADE
:10AD60000CF076FF02A88DED020ACDED030A20F06B
:10AD700031FFB4EEE80AF1EE10FACFDBB4EEC08A90
:10AD8000F1EE10FA9FED2B9ADFED2B8ADFED2B9A77
:10AD90002BD802A8694620F061FE04A88DED040AB4
:10ADA000CDED050A20F0CCFE684620EE098A20F0A1
:10ADB000C7FE94F9E83207EE903AF8EEE77A28EE0B
:10ADC000288AA7EEA90A1EF097FD20EE090ABDEE1B
:10ADD000C88A20EE280A18EE101AFDEEC07A304616
:10ADE00017EE902AFFF732FF99E738EE400A38EE67
:10ADF000088A80EE080AA6F05DFC02A8B0EE408A40
:10AE000020F09EFE94F9E832F0EE007AB0EE697A16
:10AE1000A8EE677A07EE903AF8EEE77AA7EE270AEF
:10AE20001EF06AFDC0E700BF105C00200000003487
:10AE3000308F0020E02E65420000C842DB0FC93F82
:10AE400010B504460848F7F77DFD20B92046BDE857
:10AE50001040FEF7DDBC04484FF48051F7F77CFB4F
:10AE60000028F3D010BD00BF102C00200020704738
:10AE700000487047E8E40C0800487047F0E40C080C
:10AE8000002070470020704738B5154C054600215A
:10AE9000204601F051FE042057F0EEFA0021204632
:10AEA00001F054FE132057F0E7FA0021204601F08C
:10AEB00057FE2846FEF798FE2046012102F00CF8C6
:10AEC000462057F0D9FA6B6804F5A044D3F8F8315E
:10AED000C4F834386B68D3F8FC31C4F8383838BD5E
:10AEE000102C0020FEF75EBE0B2070470048704714
:10AEF00016E80C080048704768E50C080120704708
:10AF000001207047012070470020704770B50B4E3C
:10AF100006F5C04505F548730FCB05F5447484E884
:10AF20000F003046FBF776F801463046FCF748F94B
:10AF3000002385F8A033012070BD00BF102C002035
:10AF400038B53148F8F79CFA2F48F8F797F92E48AA
:10AF5000F7F77AFF2C481021F7F7FEFAE0B12B4AF9
:10AF6000D2F82433D2F834239342D4BF00230123F0
:10AF7000264C94F8A02372B973B304F548730FCB31
:10AF800004F5447585E80F00A4F5C040FBF780FA8E
:10AF9000012384F8A03338BD1D4AB2F9041F0029EB
:10AFA000F9DD02F580429FED1B7AD2F82433D2F806
:10AFB00014239B1A07EE903AF8EEE77A67EE877A49
:10AFC00007EE101AB8EEC77AF4EEC77AF1EE10FA6F
:10AFD000CCBF01230023CBE7A4F58043642193F980
:10AFE000382512FB01F2D3F8381FA4F580548A42A9
:10AFF000A8BF0A46D4F83408C3F8382F51421EF0CF
:10B000002FFDC4F83408C6E7102C0020108C002057
:10B01000104C00200AD7233C38B52A4DB5F9CC3462
:10B0200083EAE371A1EBE37189B241B1002B05F52D
:10B030008043B4BF4FF0FF32012283F8E822224C54
:10B04000224801F0F3F994F8D237DBB995F9A73427
:10B05000022B18D194F8C5318BB11D49A1F6DC2023
:10B0600024F0F2FA58B101231A49184884F87D38BF
:10B07000282203F0F9FA28B9002384F87D38012347
:10B0800084F8D23738BD012B0ED1A4F5A04001F0D1
:10B09000E7F848B1A4F5A040FBF7B8F90028B8BF1D
:10B0A0004042B0F57A7FD5DB95F9A734042BE9D17E
:10B0B00094F8C531002BE2D00549A1F6DC2024F03C
:10B0C0003FFBCFE7104C0020107C0020102C00200C
:10B0D000308F0020787C00200220704700487047A5
:10B0E000E0E50C08004870479E230E08034B002241
:10B0F000C3F83428C3F83828704700BF107C0020FC
:10B1000038B5094D04462846F7F78EFC2846F7F770
:10B1100027FD2046F7F73CFD2846F8F741F8204682
:10B12000BDE83840FEF772BD102C00200D2070479E
:10B13000004870475CE60C080048704764E60C085D
:10B140000120704701207047012070470023C3741D
:10B1500080F82430012070470148002101F066B9D1
:10B16000102C00202DE9F041B44CD4E9CA322DED69
:10B17000088B1343D4F82423134388B005460FD11A
:10B18000AF48F8F77DF9AE48F8F778F89FEDAD0ACB
:10B19000462008B0BDEC088BBDE8F04157F06CB913
:10B1A00007F0F8F890F87C32DB07E9D5B5F90830FC
:10B1B000E97C09EE103AB5F9103008EE903AB8EE95
:10B1C000C99AF8EEE88AA4F58056002940F0D780A5
:10B1D0009FED9DAA29EE0ABA0122FDEECB7AA4F5D5
:10B1E000C04017EE903AC6F89C37FAF741FF6868FE
:10B1F00000F57F700790B0EE408A20F0A1FCDFEDF3
:10B20000937A20EE270A1EF0F5FA0798F0EE409A9E
:10B2100020F0E0FCA4F5C040F0EE40AAFEF70EF8E6
:10B22000002878D104F5487797E80F0005F1140C51
:10B230008CE80F0097E80F0004F5447C8CE80F00C1
:10B2400004F54C7C8CE80F00D4EDCD7A8048F8EE04
:10B25000E77AF0EE680A77EE8B7AB0EE690AFDEED7
:10B26000E77AC4EDCD7A0CF05DFE002386F809384C
:10B2700095F91230724803EB830303EB83039B00C1
:10B280000121A6F8CA37F6F7B1FE96F81888B8F18A
:10B29000000F74D16F4B9FED707AB3F9703407EEE5
:10B2A000903AF8EEE77A67EE877AF4EEE7AAF1EEE5
:10B2B00010FA64DD54F06CF8074619EE900AF5F7C1
:10B2C00023F9CDE9040118EE900AF5F71DF9CDE94F
:10B2D000020119EE100AF5F717F9604ACDE90001ED
:10B2E000062138464DF07CF97CF092FFC6F888873D
:10B2F000C6F874077CF08CFF0123C6F8840729EE9A
:10B300008A0AEB741EF0A0FABDEEC00A10EE103AE5
:10B31000C6F88C3733E07CF07BFFD6F82C38C01AA7
:10B3200042F2107398427FF67DAFF0EE087AF4EEA9
:10B33000E7AAF1EE10FA7FF775AFBCEEC88A04F504
:10B340004C7718EE103A9BB208EE103AB8EEC88A65
:10B35000B4EEC89AF1EE10FA47D854F019F8404A02
:10B3600006214DF03DF904F548730FCB87E80F0037
:10B370000123EB740321A4F5C040F6F737FE3048F3
:10B3800003F08EFF28B12E480321F6F72FFE00238D
:10B39000EB74D6F82038012B40F0B180D4F8243378
:10B3A000AA699FED29AA9B1A07EE903AD6F88C3726
:10B3B0000133F8EEE79A5BD0DFED2A7AE9EE0A7AFC
:10B3C000F4EEE79AF1EE10FA0ADA274905F11400D3
:10B3D0000CF032FDF4EEC08AF1EE10FA00F28F802C
:10B3E00017480321F6F702FE89E053F0D1FF1F4A08
:10B3F00006214DF0F5F804F5487C9CE80F0005F1B6
:10B40000140E8EE80F009CE80F0087E80F00D4EDC3
:10B41000CD7A39EE488AF8EEE77AF0EE680AE8EE7F
:10B420000A7A3846B0EE690AFDEEE77AC4EDCD7AC5
:10B430000CF078FD0121E9749DE700BF108C00201D
:10B44000102C0020000000000000C842E02E6542E1
:10B45000408F0020104C00209A99993EADE60C08D0
:10B460006CE60C08000048C3308F002088E60C080A
:10B47000B5F90A3007EE903AF8EEE77A05F11407CD
:10B4800067EE8A7AF4EEE79AF1EE10FA51DB424960
:10B4900038460CF0A1FBDFED417AB6EE008AA0EE53
:10B4A000278A97E80F00BDEEC88A9FED3D0AB8EEE7
:10B4B000C88A04F54C7C28EE008A8CE80F00F0EE78
:10B4C000680A3848B0EE480A0CF02CFDD4EDCD7A6D
:10B4D000F8EEE77A28EE0A0AE9EE0A7AFDEEE77A54
:10B4E000C4EDCD7A1EF0B0F9BDEEC00A10EE103AF0
:10B4F000C6F88C37D6F82038012B3FF45DAF2A48C8
:10B5000003F0AEFE18B128480321F6F76FFDD6F818
:10B510002038012B17D1244803F030FC224803F0D7
:10B5200077FD214808B0BDEC088BBDE8F04103F081
:10B5300087BC194938460CF07FFCF4EEC08AF1EE66
:10B5400010FAA4D9D6E795F824302BB9174862F041
:10B5500011F8012385F824301348F7F791FF1248BA
:10B56000F7F78CFE1048F7F76FFC114890F8DC36BF
:10B570006BB1002380F8DC3633220221A0F5405065
:10B5800008B0BDEC088BBDE8F041FDF7C5BA08B0C6
:10B59000BDEC088BBDE8F081308F0020A00CB345D6
:10B5A0000AD7233C408F0020102C0020204F002081
:10B5B000105C002010B50446FEF722FA2046054B29
:10B5C00040F8143B0CF0D6F8204603493FF0C4FC89
:10B5D000204610BD60E70C08F8E60C0818207047FC
:10B5E00000487047C8E70C0800487047D0E70C08CF
:10B5F00001207047012070470120704708B50548B9
:10B60000F7F73EFF0348F7F739FEBDE80840014869
:10B61000F7F71ABC102C002010B5074C204679F023
:10B6200093FEBCEEC00AA4F5335010EE103ABDE80C
:10B63000104099B200F0FABED058002010B50D4C61
:10B64000D4F8A83E002B12DDA4F50050FCF73AFB1D
:10B65000A4F5005000F05CFA04F54C6079F0BEFFF0
:10B6600004F54C60044979F057FB012010BD00201F
:10B67000FCE700BF104C0020408F002070B5274C25
:10B68000D4F8A00103688EB05B689847072838D0CB
:10B690000A2809D0062805D106F07CFE90F87C32F5
:10B6A000DB071BD4012017E004F508640FCC07ADBD
:10B6B0000FC594E8070085E8070009AB0FCB01AD83
:10B6C00085E80F00D4F8AC3A009304F52A630ECB5A
:10B6D000A4F60800FFF704FB0EB070BD06F05AFE9A
:10B6E00000F51B700FC801AD85E80F0004F580560A
:10B6F00004F18800D6F83C33009306F54C730ECB6A
:10B70000E8E707A904F14C00FFF730F80028C9D09A
:10B71000079904F18800FFF7C1FADDE7107C0020EB
:10B72000F0B585B00E4E0391144653F031FE06F588
:10B73000A0470546D7F8A001026892689047039B8E
:10B740000090084A284606214CF04AFFD7F8A0117D
:10B750002246304605B0BDE8F04002F085BF00BF8C
:10B76000102C0020D8E70C082DE9F0432DED028BBA
:10B77000DFF8C48197B000250746404679F00EFEF9
:10B7800005950695079506F005FE05A906F04CFB04
:10B7900058B398ED797AB5EEC07AF1EE10FA08F563
:10B7A0000D5927DBDDED067ADDED056A67EEA77A38
:10B7B00027EE077AE6EEA67AF4EEC77AF1EE10FAF3
:10B7C00018DDD9F8A00103685B6898470A2811D0F2
:10B7D00053F0DEFD544A06214CF002FF262208F504
:10B7E0000F51A8F5335002F03FFF17B0BDEC028BAC
:10B7F000BDE8F083D9F8A0414C4B01959C420295DD
:10B800000395049517D104F618040FCC08AE0FC6A3
:10B8100094E8070086E8070011A80BF0ABFFB9F821
:10B82000D8180FAAA4F14C0023F03CF890BB029565
:10B830000195049503959FED3E0A3E4E01A820F028
:10B8400029F903A88DED080A9FED390ACDED090A03
:10B8500020F020F938488DED0F0AB0EE401AF0EED6
:10B86000601ACDED100A9DED080ADDED090A79F0A8
:10B87000EFFC062804461AD10023C6F8E4327CF017
:10B88000C7FC06F54C71C6F8CC04A6F54D5079F00E
:10B8900043FAAAE701A911A80CF04AF90028C6D07A
:10B8A00003A90AA80CF044F90028C0D0C3E77CF033
:10B8B000AFFCDFED227A98ED508AD6F8CC6428EE02
:10B8C000278ADFED1F7AB4EEE78AF1EE10FA05461B
:10B8D000384658BFB0EE678AFFF7D0FE48B9022C51
:10B8E00016D0BCEEC88AAD1B18EE103A9D42FFF48C
:10B8F0007CAF013C062C0ED8DFE804F0040A0D0DE5
:10B90000100D13000F4924223846FFF709FF6CE79A
:10B910000D492522F8E70D491622F5E70C492622A4
:10B92000F2E70C490122EFE7F4E70C08787C0020ED
:10B930000000C842108C0020D058002000007A443B
:10B9400000409C461AE80C082FE80C0844E80C0854
:10B950005CE80C0873E80C08032070470048704747
:10B96000F8E80C080048704704E90C08F8B52B4DBE
:10B9700006460027A5F54050A5F8D876F7F7E6FC6F
:10B980007368A5F58052D3F8F811D2F8383F994280
:10B9900005F5005423DBC4F8343873689FED206A42
:10B9A000D3ED7F6A02F5916393ED007AF8EEE66AD3
:10B9B00027EE067AF4EEC76AF1EE10FA18DBBDEE58
:10B9C000C77A17EE103A1748C4F83838FCF7FCFE6F
:10B9D00020B1D4F838385B42C4F83838F8BD5B423F
:10B9E0009942D8DD012385F8D836C4F83478D4E7F5
:10B9F00002F63C72D2ED007A67EE867AF4EEE76AE0
:10BA0000F1EE10FA93BFFDEEE77A012385F8D936FF
:10BA100017EE903A88BF0023D5E700BF105C0020E6
:10BA20000000C842102C002070B500212DED028BC3
:10BA300004463448344D01F07FF832480021F0EEDE
:10BA4000408A01F083F895F8D836B0EE408AD3B139
:10BA5000B0EE680A042056F00FFD95F8D93693B37E
:10BA6000B0EE480A132056F007FD2648002101F0E9
:10BA700077F82046FEF7B8F8BDEC028B2046BDE80B
:10BA80007040FEF7C3B805F50056A5F54050F6F72F
:10BA9000CBFFD6F83438002B0CDCD6F83438002B2A
:10BAA000DBDA042056F0FCFCB4EEE80AF1EE10FA02
:10BAB000CED4D2E7042056F0F3FCB4EEE80AF1EE5F
:10BAC00010FAEADDC4E7114D0E48F7F749F8D5F84A
:10BAD0003838002B0CDCD5F83838002BC5DA1320A9
:10BAE00056F0DEFCB4EEC80AF1EE10FAB8D4BCE7AA
:10BAF000132056F0D5FCB4EEC80AF1EE10FAEADDD8
:10BB0000AEE700BF102C0020105C0020107C00204D
:10BB100000F5C0400023C0E9B83380F8E93280F86E
:10BB2000EA32704700F5A043D3F8CC31002BCBBFED
:10BB300007EE903A00F51150B8EEE70ADFED037A10
:10BB4000DCBF90ED0D0A20EE270A70470000C842C6
:10BB50002DE9F0412DED028B00F5A25784B09FED49
:10BB6000D98A054603A938468DED038A06F0F6F911
:10BB700005F5A044B0B19FEDD47ADDED037A04F56C
:10BB8000046367EE877AD3ED006A9FEDD07AE6EE24
:10BB9000877AF4EE487AF1EE10FA48BFF0EE487A70
:10BBA000C3ED007A2846F6F71DFEF0EE000AB0EE6F
:10BBB000408A9FEDC40A1DF08BFFD4ED797A94F88A
:10BBC000B03138EE678A05F50056E0EE087AC4ED2C
:10BBD000797A002B40F02681D4F89C2105F5A0430A
:10BBE00044339A4205D005F5A0434C339A4240F0C5
:10BBF000198108212846F6F7AFFC804640B106F2CD
:10BC00007443D3ED007A9FEDB27A67EE877A04E150
:10BC100002212846F6F7A0FC0146002800F0E68045
:10BC2000D6F8283F1B8B2846414608EE103A01F013
:10BC300053F9D6F8280F4369B8EE488AB0EE401A97
:10BC4000002B00F0B480012B00F0B680DFEDA17A6C
:10BC5000F0EE671A06F2744393ED000A9FED9C7AAA
:10BC6000F4EEC17AF1EE10FA20EE070A4FF064010B
:10BC7000C0F2AF80B6F8702412FB01F2B0EE672A72
:10BC800007EE902AF0EE400AB8EEE70A1DF07AFDC2
:10BC9000BDEEC00A84ED720AD4F89C0103689B6B68
:10BCA0009847002852D094F8DC31002B4ED0D4F8BD
:10BCB0009C3105F59F457C35AB4247D0D4ED727A77
:10BCC0009FED857AF8EEE77A384627EE878AD4ED3D
:10BCD000767AF8EEE78A68EE878A06F04BFBC8EEC4
:10BCE000807A9DED037A77EE877AB6EE007AB4EE2D
:10BCF000E78AF1EE10FA4CBF77EEC87ADFED757A7D
:10BD000077EE877A94ED787AFDEEE77AF8EEE77AC7
:10BD1000B4EEE77AF1EE10FA0ADD37EE676ADFED8E
:10BD20006F6AB4EE666AF1EE10FA48BFF0EE477A39
:10BD300094ED727ADFED666AC4ED787AB8EEC77A70
:10BD4000A7EEA67ABDEEC77A84ED727AD4F89C018C
:10BD500003681B6B984740B1B4F9D421002AC2BFD5
:10BD6000D4F8C8319B18C4F8C831B6F97224B6F9B2
:10BD70007014D4F8C80164235A4359431DF070FE6F
:10BD8000C4F8C80106F57D63D6F8E00F93ED4A8A42
:10BD900006F0F0FAC8EE007A9DED037A77EEC77AE6
:10BDA000C4ED747A04B0BDEC028BBDE8F081DFED28
:10BDB000497AF1EE481A4DE78DED010A55F03EF84B
:10BDC00007EE900ADFED431A9DED011AF8EEE77ACF
:10BDD00040E7B6F8723413FB01F300EE903AB0EE90
:10BDE000482AF8EEE00AF0EE671A4FE7B6F9702439
:10BDF000B6F972349B1A07EE903A2846B8EEE78AF5
:10BE000001F06AF8B6F87034642213FB02F307EE0F
:10BE1000903AF8EEE77AE8EE007AFDEEE77AC4EDC4
:10BE2000727A39E7D6F8A83E002B17DD96F8483E1F
:10BE3000A3B1D4F89C2105F5A14354339A4219D1FA
:10BE400005F5335079F09AFBB5EEC00AF1EE10FA21
:10BE5000DFED1F7A19DD20EE270A19E7D4F8203824
:10BE6000042B17D105F5C340783078F0B1F8C4F849
:10BE7000C80111E705F5A04368339A427FF40CAF7F
:10BE800005F5335079F07EFBDEE706F2744393ED5F
:10BE9000000AE0E7D4F89C2105F5A14310339A424B
:10BEA00006D1D4F8CC31002B02DDC4F8C831F3E65A
:10BEB00005F5A04368339A427FF4A1AE2846FFF708
:10BEC00031FEE5E6CDCCCC3DCDCC4C3ECDCC4C3F8F
:10BED0000000C842000000000AD7233C9A99993F0D
:10BEE00030B500F5A25587B00023044628460393D9
:10BEF0000493059305F0E0F8002846D003A92846EE
:10BF000006F05AF8002840D004F5BB5393ED007AB0
:10BF1000DFED226A8DED017AB0EEC77AD3ED037AB8
:10BF2000B4EEE67AF1EE10FACDED027A06D5F0EE37
:10BF3000E77AF4EEE67AF1EE10FA2DD401A81FF0BC
:10BF40009BFE03A901A81FF0DFFD04F5115393ED3B
:10BF50000F7AB5EEC07AF1EE10FAC4BFDFED107AB9
:10BF600027EEC00A04F5A044C8BFA7EE270A03F1D4
:10BF70003C03CABF01230023FDEEC07A84F8DC3104
:10BF8000CCBF17EE903A002304E004F5A044002350
:10BF900084F8DC31C4F8D83107B030BD000000347B
:10BFA0000000C8422DE9F04100F5C0472DED028B9D
:10BFB00007EE901AD7F8EC3200F5C645B8EE678A5E
:10BFC0000446303500F54056B3BB00F5A042134699
:10BFD000D2F89C116833994204D000F5A143103384
:10BFE000994229D192F8D03733B304F5C640294697
:10BFF00020300BF021FFD6F808090368F0EE408AE4
:10C000005B6AB0EE480A9847F0EE087A60EE277A4D
:10C01000F4EEE78AF1EE10FA0EDDBDEC028BD6F8F5
:10C0200008099FED0C0A036804F5C6412A469B6A7D
:10C03000BDE8F04110311847B0EE480ABDEC028B64
:10C04000D6F8080997F9E82203682946DB6ABDE8B3
:10C05000F04118470000000070B504462DED048B38
:10C0600004F5C0457CF0C8F8D5F85833544AC31AD3
:10C070009342064676D907EE903AB8EE670ADFEDAE
:10C08000517A9FED511ADFED510A20EE270A40F256
:10C0900095101DF045FCC5F8586304F50056DFED1A
:10C0A0004C7AD6F8243FB3F9083008EE103A96F9E6
:10C0B000CE34B8EEC88AF0EE408A28EE278A0BB15B
:10C0C000B1EE488A9FED437ADFED437AB4EEC78A3A
:10C0D000F1EE10FA6CDAD5EDD56AF4EEC76AF1EE3E
:10C0E00010FAB4EEE78AACBF01230023F1EE10FA98
:10C0F0005BD995EDD57AB4EEE77AF1EE10FA54D823
:10C100002046FAF7C5FB96F9CF349FED349A00EE3E
:10C11000103A04F54052D2ED000AB8EEC00A06F615
:10C12000F87393ED001A40F2A710F1EE600A20EECA
:10C13000080A1DF0F5FB28EE800A204620EE090AC9
:10C14000FDEEC07A17EE901AFAF760FBD6F8A83E1B
:10C15000002B05DD96F8483E8BB12046FAF798FB98
:10C1600085EDD58A2046F9F7C3FF2046F6F76CFE29
:10C17000BDEC048B2046BDE87040F7F77FB8184B44
:10C18000DFED187A93ED007AE7EE097AF0EE678A30
:10C1900006F000F9D0ED9C7AF8EEE77A77EEA87A0F
:10C1A000FDEEE77AC5EDD07ADAE7002BA8D1AAE751
:10C1B000B4EEE78AF1EE10FAA5D9002399E700BFA3
:10C1C0009F860100BD3786359A99193ECDCCCC3D6E
:10C1D0005304693900000034000000B40000C84274
:10C1E0009C5A002000007A4470B5054600F5B04026
:10C1F0004FF0FF31443022F0ABFB431C064605F5FF
:10C20000A04404D104F5F564124B236070BD05F51C
:10C21000C64105F5C640303110300BF0DDFC9FED16
:10C220000E7AF6EE007AE0EE077A04F5F564FDEE9C
:10C23000E77A17EE900A301A1DF03AFB07EE900AE3
:10C240009FED067AF8EEE77A67EE877AC4ED007A1A
:10C25000DCE700BF0000B442A00CB3450AD7233C82
:10C2600000F54050D0F8080903689B6B18470000A0
:10C27000F7B500F540530546D3F8080903681B6974
:10C28000984707462846FFF7EBFF05F5C0440646EA
:10C29000D4F8E402002860D13EB1D4F82433C4F8C5
:10C2A000F0323D4BC4F8F4320120C4F8DC721DF0CA
:10C2B000FFFAD4F8E43294F9E82200FB0230C4F823
:10C2C000E4022EB30023019394F84833002B48D0A6
:10C2D00094F8F431022B44D105F5B240012201A9B2
:10C2E0005C3046F0A1F900283BD0D4EDD37ADFEDE5
:10C2F0002B6AB8EEE77ADDED017AE7EE667AB1EE09
:10C30000047AF0EEE77AF4EEC77AF1EE10FA33D45D
:10C3100094F8E932002B3DD1D4F8E432D4F8F42279
:10C32000002BB8BF5B42934234DBD4F82413D4F81B
:10C33000F032C4F8F012CB1A03F2F31340F2E630F5
:10C34000834202F5D2328CBF0023012302F5F07242
:10C3500084F8EA32C4F8F4221CE0D4F8DC32F81A8B
:10C36000A3E7D4F84023D4F824339B1A03F2F31341
:10C3700040F2E6329342CBD8012384F8E93200231D
:10C3800084F8EA32D4F8E43203F5D23303F5F073DB
:10C39000C4F8F43203B0F0BDE0A501000AD7233C95
:10C3A0002DE9F04100F5A045044695F8C531C3B329
:10C3B00000F5C043D3F8382312B9D3F83C3383B324
:10C3C00004F5C64604F5C647204620363037FAF74E
:10C3D0008DFD394630460BF02FFD05F2B47304F5A0
:10C3E000C6413A461031304683ED000A0BF05AFC44
:10C3F00005F5F763DFED0C0A83ED000A7620B7EE52
:10C40000001A1DF08DFA04F53F53204683ED750A9E
:10C41000FFF72EFFD5F89C010368BDE8F041DB6A09
:10C420001847BDE8F08100BF00000000012970B589
:10C43000044600F5C04512D800F5005395F83023A6
:10C44000B3F99A3483EAE371A1EBE37189B201296C
:10C4500098BF3C21920731D5FF2385F8E83207EEDB
:10C46000901AF8EE677A2046C5EDBF7AFFF79AFD7D
:10C47000D5F8EC3243BB2046FFF7F2FE04F5A046A8
:10C4800050B906F5F76393ED007AF7EE007AB4EE53
:10C49000E77AF1EE10FA17DD7BF0BAFEC5F8EC0290
:10C4A000D6F89C0103681B6A984768B104F55B5095
:10C4B0000021BDE87040203050F082BA002BB4BF9C
:10C4C0004FF0FF330123C8E770BD000010B500F541
:10C4D000B2443C3420465CF0A9FC2046BDE8104044
:10C4E0005CF014BD10B500F5A043044693F8503934
:10C4F0009A0717D45B0700F55B504FF002014CBF61
:10C50000094A0A4A20304CF06BF804F5B2403C303E
:10C510005CF060FC04F53B500121BDE810400C309C
:10C5200062F0EABF10BD00BF7CE90C0896E90C0878
:10C5300070B500F5A046054696F93C499CB196F8C1
:10C540005039C3F380045B0729D4B6F94239002B74
:10C550000BDC2846FFF7C6FF05F53B5001210C30E8
:10C5600062F0CAFF0124204670BD2146F9F7A8FDFC
:10C57000B6F9423907EE903AF8EEE77AB4EEE70AF8
:10C58000F1EE10FAE5D5D6F8BC37002BE1D005F571
:10C590005B50044A042120304CF022F8E3E70024E9
:10C5A000E1E700BFACE90C0808B52DED028B08EE01
:10C5B000901A30B3F2B1B0F9083008EE103AB8EE84
:10C5C000C88AF8EEE88A9FED100ADFED100A28EE1F
:10C5D000800ADFED0F8A4FF4D470B7EE001A1DF019
:10C5E0009FF9C8EE280A1DF0F7F820EE280ABDECE6
:10C5F000028B08BD54F0A6FC07EE900AB8EEE78A5D
:10C60000DFE79FED020AF2E70AD7233C00000000B3
:10C6100000A08C4537B500F50054054694F9FB346D
:10C62000002B52D054F0A8FB54F09CFBC4F8200F10
:10C6300054F0A2FB54F082FBC4F8240F54F09CFB8E
:10C6400054F086FBC4F8280F54F096FB54F08AFB94
:10C6500041F29411C4F82C0FD4F8200F54F0D6FBFB
:10C66000D4F8240F41F2941154F0D0FBD4F82C0FDD
:10C6700041F2941154F0CAFB284600F027FC48BB55
:10C68000D4F8280F642154F0BDFB54F075FBD02181
:10C6900055F0A4FBC4F8300F54F06EFBD22155F0D6
:10C6A0009DFBC4F8340F05F5225024304921019038
:10C6B00056F022F901984A2156F01EF901984621B8
:10C6C00003B0BDE8304056F017B954F055FB54F0B4
:10C6D0002BFBABE705F5C043D4F8280F93F8D4340F
:10C6E000642173B154F08EFB6421462055F0FCFFA9
:10C6F0006421492055F0F8FF64214A2055F0F4FFE9
:10C70000C3E754F083FBEFE710B500F500541E219A
:10C71000D4F8200F54F07EFBD4F8240F1E2154F0DF
:10C7200079FBD4F82C0F1E2154F074FBD4F8280F99
:10C730001E21BDE8104054F06DBB000007B500F0AD
:10C74000C5FB014658B90190462055F0EFFE01990E
:10C75000492055F0EBFE01994A2055F0E7FE0021F3
:10C76000042056F0B5F90021132056F0B1F900214C
:10C77000462056F0ADF90021492056F0A9F90021D4
:10C780004A2056F0A5F90021152003B05DF804EB0E
:10C7900056F09EB910B5044656F0E0FB56F030F85E
:10C7A000204601F0E5FCBDE8104056F0DFBA00007D
:10C7B00038B500F50055044695F9FB340BB100205F
:10C7C00038BD0121F5F7C8FE90B104F5A043D3F8B8
:10C7D0009C2104F5A14324339A4209D004F5A043D7
:10C7E00004339A4204D004F5A04314339A42E6D1AC
:10C7F0002046F6F7A7F80028E1D0D5F82C3FB3F98A
:10C800000800DDE738B52DED028B00F5A04393F865
:10C81000B031002B40F0B9805D4A00F5A143D2F859
:10C820009C21243300F55B549A4204F1200408D083
:10C83000584A0321BDEC028B2046BDE838404BF03E
:10C84000CFBE00F500559FED546AD5F8202FB2F900
:10C850000830002BB8BF5B429BB207EE903A138BB7
:10C8600006EE903AF8EEE66AF8EEE77A66EE866A49
:10C87000F4EEE67AF1EE10FA17DCD5F8242FB2F9CF
:10C880000830002BB8BF5B429BB207EE903A138B87
:10C8900007EE103AB8EEC77AF8EEE77A27EE067A96
:10C8A000F4EEC77AF1EE10FA01DD3C4AC1E700F57B
:10C8B000BA5014301FF018FFDFED397A20EE270A46
:10C8C000F3EE0E7AB4EEE70AF1EE10FA01DD354A26
:10C8D000AFE7042056F0B4F8132056F0B1F8152055
:10C8E00056F0AEF84D2056F0ABF84E2056F0A8F8B2
:10C8F0004F2056F0A5F8502056F0A2F8152055F01C
:10C90000CFFD9FED298AB0EEC00AB4EEC80AF1EE61
:10C9100010FA0BD5102056F093F8562056F090F8E8
:10C92000112056F08DF8572056F08AF8032055F064
:10C93000C7FDB0EEC00AB4EEC80AF1EE10FA0FD58A
:10C94000022055F0BDFDB0EEC00AB4EEC80AF1EE0B
:10C9500010FA05D5182056F073F8192056F070F823
:10C96000D5F8200F811D0C303FF0BCF9D5F8240F0D
:10C97000811D0C303FF0B6F9D5F82C0F811D0C301D
:10C980003FF0B0F9094A052154E7BDEC028B38BDF0
:10C99000107C0020C0E90C08CDCC4C3EE0E90C082E
:10C9A000E02E654208EA0C080000003424EA0C0876
:10C9B00010B500F5005494F9D2349BB1D4F8280F87
:10C9C00054F036FAD4F8282FB4F9D43430B1B2F98F
:10C9D00006009842ACBF0020012010BDB2F906004D
:10C9E0008342F7E70120F8E710B50446FFF7E0FFC0
:10C9F00060B104F5A0447BF00BFCD4F8BC31C01A44
:10CA0000B0F57A7F94BF0020012010BD0120FCE723
:10CA100070B50546FFF7E8FF05F5005408B3D4F8F4
:10CA2000203F9A89DA80D4F8243F9A89DA80D4F8B2
:10CA30002C3F9A89DA80D4F8203F00261E81D4F852
:10CA4000243F1E81D4F82C3F1E8105F5A043D3F866
:10CA50009C01C3F8D46103685B689847D4F8283F09
:10CA60001E8105F5C8402C3071F048FD80B30026CA
:10CA700054F082F9437A13B954F07EF9837A94F929
:10CA8000D224012A23D106B10BB32846FFF7ACFF0D
:10CA900005F5A04494F8B63138B30133DBB20A2B64
:10CAA00084F8B6310CD105F55B501F4B1F4A0421A9
:10CAB00020304BF095FD1E4A012384F8B03193726B
:10CAC00094F8B6310A2B02D90A2384F8B63170BD26
:10CAD0002846FCF7B3FB0028C9D154F04DF954F0B7
:10CAE0000FF9061E18BF0126C2E7002BEFD0013B4D
:10CAF000DBB2032B88BF032384F8B63194F8B63138
:10CB0000012B09D105F55B500A4B084ABDE870407E
:10CB1000042120304BF064BD002BD8D1044A84F8A6
:10CB2000B0319372D3E700BFAB480E0834EA0C086B
:10CB30009D9100203FEC0C0800F500500A4690F94A
:10CB4000061FD0F8200FFFF72FBD000000F50050A2
:10CB50000A4690F9071FD0F8240FFFF725BD000003
:10CB600000F500500A4690F9081FD0F82C0FFFF787
:10CB70001BBD000010B54FF480610446F5F7ECFCD6
:10CB800004F5005328B1BDE81040D3F8280F54F045
:10CB9000D5BABDE81040D3F8280F54F0D9BA000038
:10CBA0002DE9F04100F500530546D3F82C3FB3F9C9
:10CBB000088000F5C044B8F1000F02D1012384F8C9
:10CBC000703405F5C8472C37384671F097FC064697
:10CBD000F8B9B8F57A6F2EDD7BF01AFBD4F86C3417
:10CBE000804693B1C31A40F6B73293420FD905F588
:10CBF000A045012231463846F4F79EFEC4F86C6425
:10CC000084F87064C5F8648701E0C4F86C04BDE87A
:10CC1000F08118F57A6F0EDA7BF0FAFAD4F86C34FA
:10CC20006BB1C01A40F6B7339842F0D90122002107
:10CC30003846F4F7A7FE0023C4F86C34E7E7C4F8DD
:10CC40006C04E4E770B52DED028B044654F094F8C3
:10CC500053F04CFF30B9BDEC028B2046BDE870406C
:10CC6000FFF7D6BE04F5A04595F8B0311BB97BF0AF
:10CC7000CFFAC5F8C0012046FFF79AFE18B17BF045
:10CC8000C7FAC5F8BC012046FFF7C2FE2046FCF7F4
:10CC900067F904F500560023C5F8D43196F9D63467
:10CCA0006BB3D6F8283FB3F90830322B27DD30B309
:10CCB000323B1BB207EE903AB8EEE78ADFED227AFC
:10CCC00004F5A25028EE278A04F030F948B3B6F9EB
:10CCD000723407EE903A06F2744696ED007AF8EE5A
:10CCE000E77A77EEC77A27EE888ADFED187A28EEA2
:10CCF000278ABDEEC88A18EE103AA5F8D43120462E
:10CD0000FFF74EFFD5F89C0103685B689847BDECC0
:10CD1000028B014604F5C8407830BDE8704056F0FB
:10CD20009BBB96F9653496F967249B1A07EE903AF7
:10CD3000F8EEE77A27EE888ABDEEC88A18EE103A38
:10CD4000A5F8D631DBE700BF0AD7A33C0000C842F4
:10CD500070B500F50054D4F8D8340BB9002042E087
:10CD600094F96434002BF9DA00F5A045D5F89C015C
:10CD700003685B6898470138172833D801A353F834
:10CD800020F000BF7DCE0108B9CE0108E5CD010835
:10CD9000AFCE0108A5CE010891CE010887CE0108CB
:10CDA000E5CD0108E5CD0108E9CD010873CE010804
:10CDB00069CE01085DCD01089BCE01089BCE01081C
:10CDC000E5CD0108E5CD0108E5CD0108E5CD010877
:10CDD000E5CD0108E5CD0108E5CD0108E5CD010867
:10CDE000C3CE0108012070BDB5F88268162EB5D0FB
:10CDF000D4F8D81411F0020301F0010205D0A6F115
:10CE0000150CDCF1000343EB0C0311F0040043EAC2
:10CE1000020303D0A6F11F046042604143EA00020E
:10CE200011F0080007D01F2E1AD0A6F11100022819
:10CE30008CBF0020012011F0100340EA020005D051
:10CE4000102E0FD0A6F1520253425341034311F466
:10CE5000006014BF95F84C18014643EA0100C2E790
:10CE60000120E8E70123F1E7D4F8D804C0F340102B
:10CE7000B9E7D4F8D804C0F38010B4E7D4F8D804E4
:10CE8000C0F3C010AFE7D4F8D804C0F30020AAE77D
:10CE9000D4F8D804C0F34020A5E7D4F8D804C0F3F0
:10CEA0008020A0E7D4F8D804C0F300309BE7D4F882
:10CEB000D804C0F3403096E7D4F8D804C0F38030EB
:10CEC00091E7D4F8D804C0F3C0308CE700F50050E7
:10CED00090F86404C009704738B504460D4653F015
:10CEE0004BFF0368DB689847C8B104F50053D3F8DB
:10CEF000280F6DB154F026F807EE900AB8EEE70A55
:10CF000004F5C04494F8D3340BB1B1EE400A38BDF7
:10CF1000B0F9083000EE103AB8EEC00AF0E79FED25
:10CF2000010AF4E70000000038B52DED028B04463D
:10CF30000D4653F021FF0368DB68984700283FD077
:10CF4000214BD3F8283F5B69012B07D0BDEC028B46
:10CF500029462046BDE83840FFF7BEBF4FF4806148
:10CF60002046F5F7F9FA0028F0D004F50053DFED7C
:10CF7000177AD3F8280F93F96734028B08EE903AAA
:10CF800000EE102AF8EEE88AB8EEC08A68EEA78AAA
:10CF900053F0E2FFB6EE001AA0EE011A04F5C04409
:10CFA000DFED0B0AB0EE680A1CF0E8FC94F8D3340D
:10CFB00028EE000A0BB1B1EE400ABDEC028B38BD81
:10CFC0009FED030AF9E700BF104C00200AD7233C6D
:10CFD0000000000073B500F5C046044696F8F43131
:10CFE000022B00F5736512D100F5B240012201A9B0
:10CFF0005C3045F019FB50B1019BC5F89C322846C6
:10D000003FF0FCFA2046F9F7C7FD02B070BD04F509
:10D01000A043D3F82038042B05D12046F9F79EFA17
:10D020008DED010AE8E7D6F85C330193E4E70000F0
:10D0300070B500F5A0450446D5F89C0103689B6BCC
:10D040000E46984748B9D4ED460A9FED1B0A642165
:10D050003046BDE8704055F005BBD5F89C0104F59D
:10D06000A04104F500526831884292F8663492F982
:10D0700030251DD195F8CC1741B93AB1D3B2D5F8C6
:10D0800020180139012998BFD3B209E004F5C04145
:10D0900091F9741261B1D5F82008042808D1CBB2F7
:10D0A00007EE903AD4ED460AB8EE670A6421CFE75E
:10D0B000002AF5D0E3E700BF000000002DE9F041B1
:10D0C00000F5A045044604F5A143D5F89C0124339E
:10D0D000984203D100263046BDE8F08103689B6B7F
:10D0E000984740B195F8506916F0010603D0012326
:10D0F00085F81838EFE704F5C340783077F09CF8EE
:10D10000064608B10126E6E795F81838002BE1D06D
:10D11000D5F89C0103689B6B984708B90023E7E7A3
:10D1200094F8143494F85874B02202FB034393F833
:10D13000F121BFBB012A0AD993ED837AF1EE047A7B
:10D14000B4EEE77AF1EE10FAACBF01270027D5F86C
:10D150009C2104F5A04368339A4202D195F8CC375C
:10D1600023B104F5A1432C339A4241D104F5005375
:10D17000204693F92485FCF761F8A8B9204601F010
:10D1800081FC0028BED0002385F8183894F871245B
:10D1900004F58C63242101FB023305F2C475DB6ABC
:10D1A0002B6098E73746D2E77BF032F8D5F82C3879
:10D1B0004FF4FA62C01A642313FB082341F2883249
:10D1C000934238BF13469842D8D92046F9F74AF916
:10D1D000B0F5FA7FD2DD04F5805341F26E72D3F8D8
:10D1E0003C3603F6B7339342C8D8002FC6D095E734
:10D1F00004F5C043D3EDD77AB2EE047AF0EEE77AC5
:10D20000F4EEC77AF1EE10FA88DA002F3FF47AAF25
:10D2100004F5A25003F08AFE00283FF47FAF04F526
:10D22000005304F5055093F88E1203F08FF8F1EED9
:10D23000047AB4EEE70AF1EE10FAFFF663AF6DE799
:10D24000F8B52DED048B0446084617461D46BDF97A
:10D25000286055F025F904F500543846B0EE408AB0
:10D2600055F01EF9B4F90025002AF0EE408A39DAAB
:10D27000C2F1640307EE903A9FED217AF8EEE77A67
:10D2800067EE877A60EE278A04F2FC44D4ED007AD8
:10D290009FED1C1ADFED1C0A38EEC80ABC2020EEF8
:10D2A000270A1CF03DFB38EE288AB0EE409A94ED38
:10D2B000000A9FED141ADFED140A28EE000ABD20C3
:10D2C0001CF02EFB2846B0EE408AB0EE490A55F01D
:10D2D000D3F8B0EE480ABDEC048B3046BDE8F84008
:10D2E00055F0CAB8D0D002F1640307EE903A9FED32
:10D2F000047AF8EEE77A67EE877A28EE278AC3E7A2
:10D300000AD7233C00A08C4500A08CC500B52DEDAC
:10D31000048B042083B055F0C3F80320B0EE408A9C
:10D3200055F0CEF8DFED189A9FED181ADFED180AC8
:10D330008DED011AF0EE408AB0EE480AA8EEA90A77
:10D34000CF20CDED000A1CF0EBFAB0EE409AB0EE23
:10D35000480A9DED011ADDED000AA8EEE90AD02089
:10D360001CF0DEFA1820B0EE408AB0EE490A55F003
:10D3700083F8B0EE480A192003B0BDEC048B5DF8C9
:10D3800004EB55F079B800BF0000344200A08C4592
:10D3900000A08CC5F8B52DED088B00F5005600F502
:10D3A000C04596F9EE3E13F0040F03F0010203F0BE
:10D3B000020440F0F580D5F8D8747B1E5F425F41CF
:10D3C000002A00F0EF804D2055F06AF84E20F0EE74
:10D3D000409A55F065F8B0EE408AB6F90235DFEDB7
:10D3E00087AA0AEE103A1520B8EECAAA55F058F8E6
:10D3F0002AEE2AAA20EE0AAA002C00F0DB80F0EE2A
:10D40000488AB0EE699AB5EEC0AAF1EE10FA40F380
:10D41000D6809FED7B1ADFED7B0A38EE0A0A4FF4C7
:10D4200080701CF07DFA9FED761ADFED760AB0EE83
:10D43000408A40F2011038EECA0A1CF071FAF0EE90
:10D44000408A96F9EF3E632B15DC07EE903A9FED8C
:10D450006E7AF8EEE77AB4EEC79A67EEAA7AF1EE42
:10D4600010FAF4EEC78A98BF29EE279AF1EE10FA67
:10D4700098BF68EEA78AD5F8D83496F9EC4E96F99D
:10D48000ED6E022B00F0B48024B2002C01DC002EE3
:10D490006EDD032055F014F8DFED5C7AB4EEE70A98
:10D4A000F1EE10FAB0EE40AA62DB002F00F0A2808D
:10D4B0009FED571ADFED570A40F2271030EE000AB1
:10D4C0001CF02EFA9FED541ADFED520AB0EE40BA6E
:10D4D0004FF494703AEE410A1CF022FA70EE007A92
:10D4E000B0EE4BAA07EE104AF8EEC7AA9FED4BBA72
:10D4F0009FED431ADFED430A6AEEA7AAB0EE690A70
:10D5000040F22B10AAEE8B0A1CF00AFA07EE906A82
:10D51000F0EE409AB8EEE70A9FED391ADFED390ACE
:10D520002AEE40AAB0EE490A4FF49670AAEE0B0A12
:10D530001CF0F6F9B0EE409AB0EE480A9FED301AB2
:10D54000DFED300A40F22D10AAEE8B0A1CF0E8F94C
:10D55000B0EE408AB0EE680AAAEE0B0A4FF497705C
:10D560009FED271ADFED270A1CF0DAF9F0EE408A6A
:10D57000B0EE690A102054F07FFFB0EE490A562041
:10D5800054F07AFFB0EE480A112054F075FFB0EE67
:10D59000680ABDEC088B5720BDE8F84054F06CBF1A
:10D5A00001270DE7042054F07BFFB0EE408AF1EE36
:10D5B000409A12E7DFED178AB0EE689A23E79FEDF5
:10D5C000101ADFED100A39EECA0A4FF482701CF00F
:10D5D000A7F99FED0B1ADFED0B0AF0EE409A40F22F
:10D5E000051039EE0A0A1CF09BF9B0EE409A28E7C4
:10D5F00000244CE7F0EE407A74E700BF0AD7233CE2
:10D6000000A08C4500A08CC5000000B400000034D0
:10D610000000C84200000000000048426666E63E86
:10D6200038B52DED028B00F500550446D5F8340FC2
:10D63000A0B304F5A04393F8B0217ABB93F8B631B8
:10D6400063BB53F045FD07EE900AB8EE678A4620AB
:10D6500095F9645454F024FF002DF0EE408A20DA4E
:10D6600004F5C340783076F069FCE8B99FED101AF4
:10D67000DFED100A40F25110B1EE680A1CF050F9CB
:10D68000B4EE408AF1EE10FAC8BFB0EE480ABDEC25
:10D69000028B6E20BDE8384054F0EEBE9FED058A47
:10D6A000D5E79FED040AEBE79FED010AE8E700BF2D
:10D6B0000000C8420000000010B52DED028B436948
:10D6C000002B4AD0037C0BB101330374037C002B85
:10D6D00041D0182B1FD803EB4303C3EB03139B006C
:10D6E0001CB2002307EE903AB8EEE78A0420B0EEB1
:10D6F000480A54F0C1FE07EE904A1320B8EEE70A3C
:10D7000054F0BAFEB0EE480ABDEC028B1520BDE81D
:10D71000104054F0B1BE4A2B02D8C3F13203DAE70D
:10D72000632B01D8643BD6E77C2B08D8643B03EB22
:10D730004303C3EB03139B001BB20024D2E7AE2BC1
:10D7400002D8C3F19603F2E7C72B01D8C83BEEE736
:10D7500000230374F1E71C46C4E7BDEC028B10BD47
:10D7600010B59FED1C7AD0ED017AF4EEC77A002354
:10D77000F1EE10FA044643722BDB90ED007AB4EE22
:10D78000E77AF1EE10FA24D908F042FB217A07F08B
:10D7900093FFD4ED010AF5EE007A60EEA77AB4EEBD
:10D7A000E70AF1EE10FA14D494ED001A40F2A51035
:10D7B0001CF0B6F8F7EE007AB4EEE70AF1EE10FAD4
:10D7C00007D494ED007AC7EE007A01236372C4EDAA
:10D7D000037A10BD00000034437A7BB391F9003026
:10D7E00090ED037A07EE903AF8EEE77A67EE877AE3
:10D7F0009FED137AF4EEC77AF1EE10FAD8BFF0EE8F
:10D80000477AFDEEE77A17EE903A0B7092F9003006
:10D8100090ED037A07EE903AF8EEE77A67EE877AB2
:10D820009FED087AF4EEC77AF1EE10FA58BFF0EEE9
:10D83000477AFDEEE77A17EE903A1370704700BF13
:10D840000000C8C20000C842437AF0EE407A5BB1E3
:10D8500090ED030A9FED051ADFED050A27EE800A19
:10D860004FF4E6701CF05CB8704700BF0000C8427F
:10D870000000C8C2F8B504460E4617467AF0C8FC48
:10D88000054604F5A340683008F0A0F804F5A0446C
:10D89000D8B3462054F004FEDFED3D7AB4EEE70A3B
:10D8A000F1EE10FA10DB97F9002094F91938193AC3
:10D8B000934209DAD4F81C28AA4205D0C4F81C58AF
:10D8C000013384F8193844E0462054F0E9FDDFEDD7
:10D8D000317AB4EEE70AF1EE10FA3AD896F9002060
:10D8E000002A36DAC2F1FF2294F91A3802F57F02D3
:10D8F000E73293422DDAD4F81C28AA4229D0C4F882
:10D900001C58013384F81A3823E0D4F81C38EB1A79
:10D91000B3F57A7F1DD3462054F0C2FD94F919382F
:10D9200007EE903AF8EEE77AB4EEE70AF1EE10FA75
:10D9300001DD002B22DC462054F0B2FD94F91A38A8
:10D9400007EE903AF8EEE77AB4EEE70AF1EE10FA55
:10D9500018D497F9000094F919280021821A1CF0B4
:10D960008FF8387096F90000002806DA94F91A1832
:10D97000002201441CF084F83070F8BDC4F81C5833
:10D98000013B9EE7002BE4DDC4F81C58013BB9E7DE
:10D9900000000034000000B410B52DED028B00F53E
:10D9A000005282B092F9643492F865248DF8063002
:10D9B000002B0446B0EE408A8DF8072004DAFFF70A
:10D9C000C7F908B98DF8060004F5A043D3F820285C
:10D9D000012A4CD0072A4AD004F5C340783076F0AB
:10D9E000ADFA002858D104F53B500DF106010DF1B8
:10D9F00007023030FFF7F0FE2046FFF73BFF9DF9AE
:10DA000006309DF90720DFED258A9342A8BF134613
:10DA100007EE903A04F53F54B8EEE70A103420EED2
:10DA2000280A20468DF8063075F080FC9DF90730F5
:10DA300000EE103AB8EEC00A204620EE280A75F033
:10DA40007FFC9DF9073001EE103A9DF9063000EE9B
:10DA5000903AB8EEC11AF8EEE00A40F24D20B0EE6E
:10DA6000480A1BF05DFF02B0BDEC028B10BD03F253
:10DA70007C73D3ED007AFDEEE77A17EE903A8DF8DD
:10DA8000073004F5AF43D3ED007AFDEEE77A17EEE9
:10DA9000903A8DF80630A6E70023FAE70AD7233C30
:10DAA00070B5044600F53B55303504F5A0462846D0
:10DAB000FFF756FED6F89C0103685B6D984740B1AE
:10DAC000462054F0EDFC2846FFF7BEFE462054F0F9
:10DAD000D3FCD6F89C0103681B6D984740B14620E3
:10DAE00054F0DEFC2046FFF757FF462054F0C4FCFC
:10DAF0002046FFF7E3FA10B304F5005595F9D0344A
:10DB000043B101212046FFF7E7F9BDE87040462008
:10DB100054F0B2BC04F5C3447834204676F00EFAD3
:10DB200050B1204676F092FB30B195F9643400EEA6
:10DB3000103AB8EEC00AE8E79FED010AE5E770BDCC
:10DB40000000000010B504462DED028B462054F075
:10DB5000A7FC2046B0EE408AFBF770FB80BB04F5C3
:10DB6000C8402C3070F0CAFC50B304F5A253D3ED7A
:10DB7000968A1BF053F990F8EC349FED137A0C223F
:10DB800002FB0300D0ED807AE8EEC77AF4EEC77AA4
:10DB9000F1EE10FA0CDC04F5005494F9673407EE4A
:10DBA000903AF8EEE77AF4EEC87AF1EE10FA07D57B
:10DBB000BDEC028B0548BDE81040012104F05EBEBB
:10DBC000BDEC028B10BD00BF0AE81C415040002094
:10DBD0002DE9F34100F500550646D5F8303F002BFE
:10DBE00041D1002706F5A048D8F89C0103689B6B3B
:10DBF0009847044600285FD006F5A25003F096F936
:10DC000000283DD0D8ED727A9FED487AF8EEE77A99
:10DC100067EE877AFDEEE77A17EE903A1BB295F938
:10DC200017250AB19A422EDA95F9154574BBD8F832
:10DC30009C2106F5A14354339A4209D105F56A6344
:10DC4000D3ED007AFDEEE77ACDED017A9DF904403F
:10DC5000D8F82038013B062B2ED8DFE803F01E2D24
:10DC600024612D2D1E0053F087F80368DB68984768
:10DC70000028B6D0D5F8300F53F02AFA47B2B1E7F2
:10DC800095F96734CBE795F91645D0E724B29C4265
:10DC9000ACBF95F914450024C9E795F91835002B58
:10DCA00018BF1C4608E095F918352BB13046FBF734
:10DCB000E5FA08B195F9184587EAE773A3EBE7732E
:10DCC000DBB2A342C8BF3C4607EE904A0320B8EE41
:10DCD000E70A54F0D1FB07EE907A0220B8EEE70A8B
:10DCE00054F0CAFB95F94935D6ED460A00EE103AD4
:10DCF0006421B8EEC00A032054F0B4FC95F949350C
:10DD0000D6ED460A00EE103A6421B8EEC00A0220B1
:10DD100054F0A8FC304602B0BDE8F041FFF7F6BA77
:10DD200006F5C04393F97332B9E700BF0AD7233C25
:10DD300070B504462DED048B462054F0B1FB5B4BCF
:10DD4000DFED5B7A93F9B83E08EE903AF8EEE88A98
:10DD5000152068EEA78AB0EE408A54F0A1FB9FED33
:10DD6000557A20EE280A04F5C045C0EE077A05F57D
:10DD7000996604F5C5400430C6ED007A73F03AF9AF
:10DD800008B100233360B5EEC08AF1EE10FA46D533
:10DD90002046FFF79BF8002800F083802046FEF71E
:10DDA000D7FF00287DD005F59965D5ED007A9FED68
:10DDB000429A9FED421ADFED420AB0EE480AA7EE02
:10DDC000890A4FF43B701BF0ABFDD5ED007A9FED57
:10DDD0003B1ADFED3B0AF0EE408A40F2ED20B0EE58
:10DDE000480AA7EEC90A1BF09BFDB0EE408A04F575
:10DDF000C8452C35284670F08BFBE0BB284671F0F7
:10DE00004DFC022829D10321492054F08FFEBDEC9E
:10DE1000048B0321BDE870404A2054F087BE40D9EE
:10DE200005F59965D5ED007A9FED239A9FED251AAA
:10DE3000DFED220AB0EE480AA7EE890A40F2F2208E
:10DE40001BF06EFDD5ED007A9FED1E1ADFED1B0A6B
:10DE5000F0EE408A40F2F320C1E79FED180A492016
:10DE600054F00AFBBDEC048B9FED140ABDE8704032
:10DE70004A2054F001BBB0EE680A492054F0FCFA85
:10DE8000B0EE480A4A2054F0F7FA20464921FFF73D
:10DE9000CFF8BDEC048B20464A21BDE87040FFF767
:10DEA000C7B89FED068AF0EE488AA0E7104C002024
:10DEB0000AD7233C00A08C45000048420000000027
:10DEC0000000C8C20000C842F8B52DED028B00F575
:10DED000C046044696F97132002B31DD00F5A042B0
:10DEE0001346D2F89C2168339A4229D196F97032B0
:10DEF000002B25DD00F5C340783076F091F8F8B1BD
:10DF000004F5C8402C3070F0F9FAC8B9124F9FEDF3
:10DF1000138A04463D682D190ED0B5F9080054F057
:10DF2000D1F848B196F97132012B0CD1B5F908003E
:10DF3000B0EE480A54F0A0FA1434B4F5A07FE9D149
:10DF4000BDEC028BF8BD022BF6D1B5F90800032118
:10DF500054F0ECFDF0E700BF2C960020000000001C
:10DF600037B500F5A043044693F878370BB39FED1F
:10DF7000120A15204F2554F07FFA204600955023B1
:10DF800013221521FFF75CF9152054F017FD80B915
:10DF9000284654F013FD60B99FED070A4E2054F057
:10DFA0006BFA9FED050A4D2003B0BDE8304054F0F8
:10DFB00063BA03B030BD00BF00000000704700002E
:10DFC000F8B52DED048B00F5A0440546D4F89C016E
:10DFD00003689B6B984730B9D4F89C2123463C33A7
:10DFE0009A4240F0C08005F5C8402C3070F090FA9D
:10DFF000002800F0B8802846FBF720F9002800F040
:10E00000B280D4F83438002BB8BF5B42B3F52F7F11
:10E0100000F3A980D4F83838002BB8BF5B42B3F5C1
:10E020002F7F00F3A08005F5C0477AF0F1F8D7F80C
:10E030009833C31AB3F5FA7F0646C0F0948005F50D
:10E04000C25393ED017AF2EE007AB4EEE77AF1EE84
:10E0500010FA00F1888004F5046494ED007AB4EEBF
:10E06000E77AF1EE10FA7ED405F5405393EDE38A9A
:10E0700005F5225403F59B63D3ED048A2434B0EEF6
:10E08000480A0421204654F06DFAB0EE680A1321C4
:10E09000204654F067FA78EEC89A4D21B0EE690A2E
:10E0A000204654F05FFA38EE289A4E21B0EE490A25
:10E0B000204654F057FAB0EE680A4F21204654F03B
:10E0C00051FAB0EE680A5021204654F04BFA05F59B
:10E0D0000055B0EE480A1821204654F043FAB0EE3D
:10E0E000480A1921204654F03DFA95F9EE3E03F016
:10E0F0000202DB075CBFF1EE489AB0EE489A6AB3C1
:10E10000B0EE498AF0EE698AB0EE690A1021204625
:10E1100054F028FAB0EE680A5621204654F022FA4C
:10E12000B0EE490A1121204654F01CFAB0EE480A1C
:10E130005721204654F016FAD7F89C33C7F8986355
:10E14000F31A42F2107293420DD9C7F89C63BDECEA
:10E15000048B2046BDE8F84054F0EABD9FED038AE9
:10E16000F0EE488AD0E7BDEC048BF8BD000000005B
:10E1700073B5044654F0F2FE054654F085FE204681
:10E18000FFF7D6FD4E23009313224D230421204692
:10E19000FFF756F84F2315211322009320465023F2
:10E1A000FFF74EF82046FFF7F5F82046FFF78CFE04
:10E1B0004FF400512046F4F7CFF910B12046FFF795
:10E1C000CFFE04F50056D6F8BC0E50B104F5A042BF
:10E1D00004F5A143D2F89C2124339A4201D154F092
:10E1E00025F954F0E7FD54F03BF8284654F054FE6E
:10E1F00096F9903C2BB1204602B0BDE87040FFF785
:10E20000DFBE02B070BD000073B5044604F5C5451D
:10E2100054F0A4FE043554F037FE284672F0EAFEAE
:10E22000002866D104F5A046D6F82038042B04D186
:10E2300004F5C340783075F0ADFE2046FFF730FCA2
:10E24000D6F89C2104F5A143243304F5C8459A422D
:10E2500005F12C0523D0284670F05AF9F8B99FED46
:10E26000320A462054F008F99FED2F0A492054F055
:10E2700003F99FED2D0A4A2054F0FEF8284671F06C
:10E280000DFA02280BD10321462054F04FFC032144
:10E29000492054F04BFC03214A2054F047FC20460F
:10E2A000FFF750FC2046FFF793FC2046FFF7B8F934
:10E2B00020464621FEF7BCFE284670F01FF990B9B3
:10E2C0000190284671F0EAF968B102281CD1019941
:10E2D000462054F097FB0199492054F093FB019993
:10E2E0004A2054F08FFB204602B0BDE87040FFF793
:10E2F0003FBF2846F7F716FE04F5C04393F98E3268
:10E300002B2B8FD002B070BD9FED070A462054F032
:10E31000B3F89FED050A492054F0AEF89FED020ACC
:10E320004A2054F0A9F8DEE700000000F8B500F537
:10E33000A046044696F84C18214876F05DFE04F598
:10E340000053D3F8A83E002B38DD04F5335528469A
:10E3500076F042FED6F89C7104F5A1465436B742D9
:10E3600008D12846012176F085FE3846BDE8F84000
:10E37000FDF7FAB93B6838469B6A9847014628463C
:10E38000C1B176F0E9FCC8B1284676F085FD284693
:10E3900076F024FD90B104F55B500A4B0A4A062141
:10E3A00020304AF01DF9314620461522BDE8F840DC
:10E3B00000F05AB9BDE8F84076F05CBEF8BD00BF89
:10E3C000D0580020C8E70C084CEA0C08F6F75EBBF2
